:020000040000FA
:1000000000F8020269340000F50F0000A1110000A1
:1000100000000000000000000000000000000000E0
:100020000000000090E00000D8E00000F50F0000A4
:100030000000000000000000F50F0000C5350000C2
:10004000E90D0000F50F0000F50F00008D340000F1
:1000500059120000B5310000850F00002510000086
:10006000810C0000BD0B0000F50F0000F90F00002F
:100070002D120000C53C000009340000353400009A
:10008000F50F0000F50F0000F50F0000E935000046
:1000900009360000F50F0000F50F0000F50F000015
:1000A000193A0000233A0000EB0D00001D33000058
:1000B000F50F00001D3200000000000000000000ED
:1000C0000348854600F04AFD004800477D77000060
:1000D00000F8020230B50B46014600202022012420
:1000E00009E00D46D5409D4205D31D469540491B6C
:1000F0002546954040191546521E002DF1DC30BDB5
:1001000070B500242546002801DA01244042002968
:1001100001DA01254942FFF7DDFFAC4200D0404241
:10012000002C00D0494270BDF8B5002425460029B6
:1001300004DA0E46012400214042B141002B04DACA
:100140001E46002352420125B34100F003FC8C46B9
:1001500017461E46AC4203D0002540428D41AC46B6
:10016000002C02D0002657429E4161463A46334653
:1001700001B0F0BD03460B439B0703D009E008C95B
:10018000121F08C0042AFAD203E00B780370401C47
:10019000491C521EF9D27047D2B201E00270401CD5
:1001A000491EFBD270470022F6E710B513460A46F7
:1001B00004461946FFF7F0FF204610BDF8B5024689
:1001C0004A40D40F42004B0052085B089A4202D2C8
:1001D0000246084611464A0023D0C30D4A00DDB24C
:1001E000120EAD1A202D35DA49020126490AF6050C
:1001F0008A19002C00D0524220214F1B1146B940D1
:100200002A411018C20D9A4221D0002C17D0012D7E
:1002100008DCDA05801AD20F8019D207DBB200F0B1
:1002200005FCF8BDDA05801A012340001B06C01842
:1002300080185A428018CA0F1043490007E0490845
:10024000C2071143DA05801A80194008801800F0AF
:10025000E5FBF8BD61000122511A001BF7E70122FE
:10026000D2075140AAE70122D2075040A6E7024632
:1002700070B54A40D30FDB0740002DD04A002AD08A
:10028000010E140E000212020919400A520A8418C3
:10029000E50104465443000A120A2E045043A419EF
:1002A0004219200CC543AA18120C0125AD03521C9B
:1002B000521912047F39240400D0521C104301D477
:1002C0004000491EC2B20C06C0092018401C40085C
:1002D000802A02D003E0002070BD400840000029C1
:1002E00000DA0020184370BD70B502464A40D50FB1
:1002F00040004A00ED0740085208002814D0002AA8
:1003000012D0C40DD30D41020120C0055202490A8A
:10031000520AE41A091812187D34914201D3641C60
:1003200000E04900002C01DA002070BD002391425A
:1003300001D3891A0343400849000028F7D1002956
:100340000AD0914202D10121C90705E0914201D2B0
:10035000012101E00121C943E005C018401900F066
:100360005DFB70BDF0B507460846584087B0C00F2A
:10037000049048000E46590040084908BC1A8841BC
:1003800005D2384631461E4617460B4602465800EF
:10039000400810434CD0300D039040055900400DEB
:1003A000490D0590401A0290402872DA1803012185
:1003B000000B09050843019004980092002805D01D
:1003C00001995242002088410092019002984021F8
:1003D0000A1A0199009800F0EDFA05460C466B46A2
:1003E00007CB00F008FBC0197141039A0E0D0023E2
:1003F000D71756401A467A40164344D0049A002A2A
:100400002DD0029A012A039A15DC1205C01A9141D7
:1004100001263605001C7141D20F059ED2070093BC
:10042000019202962A46234600F046FB07B0F0BD33
:1004300038463146FAE71605224A0F46B218C01A66
:10044000B74101210905001C4F4100187F411146A9
:1004500018187941E20F10436D19644113E0E20767
:100460006D0815436408C2071443039A0126120558
:10047000C01A91413605001C7141CE074008304337
:100480004908C01851412A46234600F008FBCDE731
:10049000FFE7049801224000C117121A00238B4184
:1004A00004983146C417381AA141EEE730B401244C
:1004B000E407634030BC55E730B40124E4076140F1
:1004C00030BC4FE70000E0FFF0B51FB488B00B99D7
:1004D0000998002448400999C00F4900490809912A
:1004E000C0070B990090490049080B910999089899
:1004F000A64608431CD00B990A98084318D00998BF
:1005000001244000420D4800410D099824050003D4
:10051000000B204309900B980003000B20430B9025
:1005200050181C494018002201901446104605E05E
:10053000002001460DB0F0BD032801DA034600E0BB
:1005400003239C46C11A0AAE0AE05F0008ADED5BCA
:100550004F00F75B7D430027AA187C41491C5B1EB6
:100560006145F2DD410004AB5A522104120C0A43EA
:10057000240C401C0828DFDB01980290009970468B
:1005800001910090059B049A0799069800F094FA4F
:10059000D0E700000DFCFFFFF0B50C465C4085B0D5
:1005A000E40FE40703944C000026640859009446C5
:1005B000490802460296224321D062460A431ED0D1
:1005C0006200570D4A000E032303550D0124024615
:1005D0002C492405781B1B0B360B4018234326435C
:1005E000614600901C46501AB44103D30098401C49
:1005F000009002E0921800985B41002803DA002086
:10060000014605B0F0BD00200121090507468646D8
:1006100011E064461D46141BB54106D36546521BC6
:10062000B341744607430C43A646CD07400849082A
:10063000284392185B4105460D43EAD11046184302
:1006400013D06046194650407140084306D06046BA
:10065000101AB34106D20122002306E00022012332
:10066000DB0702E00122D2435310009874460105D3
:10067000381C6141029C039D0019694100F00FFA8A
:10068000BFE70000FD0300000122D207002800DBC5
:10069000101A002900DB511A814201D8012070474D
:1006A000002070470122D207002800DB101A002921
:1006B00000DB511A814201D20120704700207047AF
:1006C0000122D207002800DB101A002900DB511A92
:1006D000814201D301207047002070470122D207D8
:1006E000002800DB101A002900DB511A814201D9D1
:1006F00001207047002070470122D207002800DB4C
:10070000101A002900DB511A814201D101207047E3
:100710000020704710B5002904DB0C460121C907F1
:100720004042A141002B04DB1C460123DB0752425F
:10073000A341801A994101D3012010BD002010BDB2
:1007400010B5002904DB0C460121C9074042A14134
:10075000002B04DB1C460123DB075242A341101A85
:100760008B4101D3012010BD002010BDC217C10F65
:10077000504010B54018CA079623002100F056F9E2
:1007800010BD10B500229623114600F04FF910BDA0
:100790000EB5C217C10F5040CA0740180021054BC3
:1007A0000293019200910A460B4600F085F903B0CE
:1007B00000BD0000330400000EB505490291002180
:1007C00000910A460B46019100F076F903B000BD96
:1007D000330400003EB5CA17CB0F002450405140EF
:1007E000C0186141DA07054B02930192009422463A
:1007F000234600F061F903B030BD0000330400006F
:10080000C20F410040020123400ADB05D207090E56
:10081000C0187F2901DA00207047962903DC96234F
:10082000591AC84001E096398840002AF4D0404265
:100830007047410040020122400AD205090E80188B
:100840007F2901DA00207047962903DC9622511A8D
:10085000C8407047963988407047000070B5CD0F8A
:100860004A0009030123090B1B0519430B4BED0734
:100870000024520D9A4201DA002070BD074B343338
:100880009A4203DC9A1A00F0A5F802E004495118D4
:1008900088402C43F1D0404270BD0000FF030000AF
:1008A000CDFBFFFF70B5CD0F4A0009030123090BF3
:1008B0001B0519430D4BED070024520D9A4202DA35
:1008C0000020014670BD094B34339A4203DC9A1A6A
:1008D00000F080F803E0064BD21800F06BF82C43D0
:1008E000F0D0002240428A41114670BDFF03000053
:1008F000CDFBFFFFC20FD207400040080BD0C10D57
:100900000723DB01C91840020905400A1143C20848
:10091000400711437047002001467047CB0FDB07AB
:10092000490010B5490802460A4307D00A0D0724BA
:100930000903E401090B121B002A01DC002010BD91
:10094000C900440F0C43C100E018D205801800F024
:1009500065F810BDF0B51FB40646002082B005460C
:100960004024019100901BE0019922460F46304639
:1009700000F030F8049A059B801A994110D3104674
:100980001946224600F016F8361A8F410197224682
:1009900001200021009F00F00DF838184D41009013
:1009A0002046641E0028DFDC019B00982946324661
:1009B00007B0F0BD10B5202A04DB0146203A914073
:1009C000002010BD914020239C1A0346E3401943A8
:1009D000904010BD10B5202A04DB0846203AD040D4
:1009E000002110BD0B46D340D0402024A21A9140D4
:1009F0000843194610BD10B5202A06DBCB17084660
:100A0000203A1041C1170B4306E00B461341D0407A
:100A10002024A21A91400843194610BD002904DA87
:100A2000401C490001D140084000704770B40024C8
:100A3000050C05D11024000402D1002921D0112475
:100A4000050E01D100020834050F01D10001241D5B
:100A5000850F01D18000A41C002801DB4000641C2C
:100A6000002908D020252E1B0D46F540A14000D0BE
:100A700001212943084301061B1B000ADB1D02D587
:100A8000002070BC7047DB05181880180029F8DAC0
:100A9000401C4900F5D170BC40084000704710B5BB
:100AA000002B08DA0024401C614192185B411A4374
:100AB00001D14008400010BDF0B51FB482B005461A
:100AC0000C0003D008460BF0B9FA02E00BF0B6FABE
:100AD00020300246009021462846FFF76BFF049B1A
:100AE000059A04460F4618431143084314D018468C
:100AF00010431BD0009840210A1A18460599FFF7A9
:100B000069FF05460E46009A05990498FFF752FFC3
:100B1000084305D0012004E02046394607B0F0BD67
:100B20000020C11705430E432C43374300990E980C
:100B30006305401A7905E40A00220C43FD0A0A30D5
:100B400002D500200146E9E70105101969410C9C16
:100B50000D9D00196941FFF7A2FFDFE7064C012553
:100B6000064E05E0E36807CC2B430C3C9847103455
:100B7000B442F7D3FFF7A8FA6CDB00008CDB00006F
:100B800030B58C180278401C13071B0F01D1037875
:100B9000401C120906D10278401C03E005780D7054
:100BA000401C491C5B1EF9D101E00B70491C521E10
:100BB000FBD1A142E6D3002030BD000010B5214892
:100BC000016A8A0715D44A0715D4C90732D01E49CD
:100BD0008A89002A15D0531E8B8182688C6904C4CF
:100BE0008C610A691B040DD0002A22D10121016009
:100BF00010BD022100E00421C16113488021416140
:100C000010BD0A69012A09D1026801239A430260D2
:100C1000C361FF20683099300C4A106001204861A0
:100C2000CA69002A05D0886909898B00C01A9047D3
:100C300010BD10BDFF226832054806A109A309F0C6
:100C400021F8C04608D001400095010280E200E092
:100C5000E4CA00004144435F49525148616E646CEC
:100C600065720000556E6578706563746564204137
:100C7000444320696E746572727570740D0A0000C9
:100C800070B582B000230193444801688A6A4C68B9
:100C900013252540132D02D1CB689B07DB0F436141
:100CA000930772D453070AD4D30711D1130724D55D
:100CB000048F838E1C1B102C0EDD102310E00420EB
:100CC00088620220032142A20AF03AF802B070BD05
:100CD0000120886202B070BD048F1B1B1C0610D05F
:100CE000DBB20024058FC66A75192D5D0D74641C76
:100CF000A342F7D1048FE3180387D20607D400215B
:100D00002FE04B6A0824A3434B62D206F7D5CB6889
:100D1000C28E448F141B5B04DB0EA34201D3438FAE
:100D2000D31ADAB2002A16D0097D438F046BE1543E
:100D30000199012A10D001231C46890145582D7DB7
:100D400041184E8F9B19096BCD54641CE3B2019975
:100D50009A42F2D800E000218B01C3185C8FA218E0
:100D60005A878A0181184B8FCC8EA3420BD3012363
:100D70000B61805800224262CA6B002A03D03A31CC
:100D8000098801A8904702B070BD0220886204481B
:100D900004A1084A08A308F075FFC046209001028C
:100DA000FDCA00004145535F49525148616E646C71
:100DB00065720000CE02000041455320696E7075D7
:100DC00074206F766572666C6F770D0A0000000004
:100DD000414553206F757470757420756E6465722B
:100DE000666C6F770D0A000070477047F0B587B0EA
:100DF00050480068FFF7CCFC04460D464E48406A58
:100E0000FFF778FD02460B4620462946FFF7C4FB54
:100E100002460B46002449492046FFF747FB039052
:100E2000029101200590400201904549454F06E09E
:100E3000534A10517F1C891C241D642C78D03878AB
:100E400064284148F4D10497069140480159404E26
:100E5000316240480359B3613F480059B0623F4A8C
:100E60001259326300275D1A3564736AF16999413A
:100E7000059B00DB3B46002B01D0019BC918344E7B
:100E80007164F36A716B101A9941059A00DB3A4656
:100E9000002A01D0019A8918FFF79CFC02460B46F4
:100EA00003980299FFF710FBFFF7FCFC284A9063B8
:100EB000D163401BC10F4018401010601546FFF76A
:100EC00067FC274A274BFFF7FFFAA864E964264A24
:100ED000264BFFF7F9FA3A46254BFFF7F5FA3A4663
:100EE000244BFFF73FFA05460E461948056141615C
:100EF00028463A46204BFFF70DFC00280699049F30
:100F000098D10022284631461C4BFFF719FC069960
:100F100000288FD1088800B2FFF73AFC02460B4642
:100F200028463146FFF71EFAFFF798FC06997FE73F
:100F300007B0F0BDF0960102F8C000000000F03FDD
:100F4000B098010218970102FFFF0100E498010226
:100F50003896010248990102FCB3010260B4010213
:100F6000699006699006903F52257997532ED33F9A
:100F70000000594000003E4000408FC0006AF84029
:100F800024A70102B0B582B0194C2068056801A9F8
:100F90000020087007E090470198401C01A90870E4
:100FA000C0B2082822D2012211048140294209D06E
:100FB0002268516080002018826A002AECD001A8C3
:100FC0000121E8E7130283402B4201D0022104E013
:100FD00082402A42E0D003211346226853608000F9
:100FE00020188268002AD7D001A8D4E702B0B0BD8B
:100FF00070920102FEE7000010B509480168CA6955
:1010000020231343CB610269032A08D101229305EF
:101010000C689C430C605102C26E0A43C26610BD4C
:10102000E0920102F0B581B05C4C2068856BE80766
:1010300007D0E168002904D00020884720680121FA
:101040008163A80707D52169002904D001208847BA
:10105000206802218163680707D56169002904D0EF
:1010600002208847206804218163280707D5A169E9
:10107000002904D003208847206808218163E806FE
:1010800007D5E169002904D0042088472068102191
:101090008163A80607D5216A002904D00520884766
:1010A000206820218163680607D5616A002904D081
:1010B00006208847206840218163280607D5A16A59
:1010C000002904D0072088472068802181630126F9
:1010D000E80507D5E16A002904D0370208208847CF
:1010E00020688763A80507D5216B002904D0770203
:1010F0000920884720688763680507D5616B002948
:1011000004D0B7020A20884720688763280507D5DE
:10111000A16B002904D0F7020B2088472068876361
:10112000E80407D5E16B002904D037030C20884779
:1011300020688763A80407D5216C002904D07703B1
:101140000D20884720688763680407D5616C0029F3
:1011500004D0B7030E20884720688763280407D58A
:10116000A16C002904D0F7030F208847206887630B
:10117000E80307D5E16C002904D037041020884724
:1011800020688763A80307D5216D002904D0750462
:10119000112088472068856301B0F0BD609301028B
:1011A00004217046084204D0EFF30983EFF308826C
:1011B00003E0EFF30883EFF309829BB004A8F0C0CB
:1011C00044464D4656465F4608A8F0C01846F0C84B
:1011D0006846F0C018690C90202018440D9058699A
:1011E0000E9098690F90D8691090EFF310801190CD
:1011F000EFF31480129009490868139008490868B1
:1012000014900849086815900749086816901793C4
:10121000189270461990684608F04EFF04ED00E001
:101220000CED00E010ED00E014ED00E080B50748A3
:1012300001210170064802680A43026005480268FD
:10124000002A02D000200146904780BDDEA60102A0
:101250001C100050E0A60102F0B599B0F548017BE2
:10126000C67A427B0E92F44C221F1368F34A12682E
:10127000069242780C9202790592C76A04931F4045
:1012800001200F907A0200D5BCE03A0200D5BFE001
:10129000FA0102D50F9802062260502508968A1995
:1012A0001826BB0102D50F984306236041230795FA
:1012B00069430A96354655431426FC0210D50F980B
:1012C000040538463746DC4E3460DA4CA469B46411
:1012D000D84CE4697464DA4C241D34603E460746F9
:1012E00090000B90D8040D90681809900E9B7343E2
:1012F0000F988203B902D04D22D50F98410529607D
:10130000CC480E961646024681692965C169696511
:1013100009990D9801430898000108180B99401885
:10132000C018C849098892794A4380180A301C4677
:1013300003F0DAFD234632460E9EC04988672A60D4
:101340000F98C404380300D52C60F80302D50F9819
:10135000000428600F984104B80300D529603804C0
:1013600000D4E4E1039402910E9308920D980B9936
:101370000C180A980C9941430C910F98C0030B90DC
:10138000286006F083FB002801D003F08FFD0C9845
:10139000005B410B43D1099800190E99401805993B
:1013A000090140180E90E74D287B079B4343E97ADB
:1013B0000A010D9C2243D21841188B00D2180A9BB7
:1013C0004B43D1186A7B564389190E9E2A7910180F
:1013D000DF4A12884243881816903068C000800D9A
:1013E00010A9C882002511957079C0077ED110A878
:1013F0000F998182069C00940020E8A2049B09F0CA
:101400009FFC78E00F98820522603A0200D43FE703
:101410000F98C2052260FA0100D53BE73DE707219E
:1014200049030840032149038842089A00D07EE11D
:10143000069705F0F5FF0020169009901590C14C15
:10144000E07A217B08180A99414380000D9A1043E5
:101450004118627B0E9672438A186178A379079EC1
:101460007343D718FA683F26324063789A420C9744
:101470006ED105960A9A4A4380580F210A07024006
:101480000398401EC04B1B68DB090340981810905E
:101490000F98C0020B90B868800767D42C46283C90
:1014A00008F0C2FB05462068000609D5C320840168
:1014B000786A400704D408F0B7FB401BA042F7D974
:1014C00005980002B96849080140B348036882687A
:1014D000B868C40C20202040DB0700D095E0002332
:1014E00010221D461C460E9E0B9FB1E010A885825F
:1014F000B0681190069C701D924B1979E20707D1D4
:10150000491C1971D97A1A798A4202D31D7100E0F7
:10151000D970017842781202511882781204891821
:1015200003229143017035715878401C5870D87A65
:10153000197B08185978884200D85D70D879401E08
:10154000D871596B002901D010A888477E4DEDE075
:1015500010A80B998182F8683040637800900020D1
:101560007CA20F9909F0ECFB0E9E94E0388A874A22
:10157000024010A8C2822022BA5C9307DB0F3C68AD
:10158000C3720F9B1A4082726205D20C0D9B1A43E4
:101590001692FA68130E0372BB69FC697C4D2D68C4
:1015A0002D0C05745204920F427211931394654CE2
:1015B000A07B002809980E9E0B9F5FD0754800689D
:1015C000007A0328099859D00C98007D0840092812
:1015D000099853D1C320840108F026FB05460C98D6
:1015E000406A41070BD4594909680906890F06D199
:1015F00008F01AFB401BA042F1D90C98406A410345
:101600000898884310A9888237E0D2070E9E0B9F66
:1016100003D108230022154619E00C9B9A68029C0E
:10162000224211D19A68520C02249443002213469C
:1016300015460DE0E8A6010228A000503CA100508C
:10164000FC1F0000E4A601020425002213461446F4
:101650000843104318432843204310A98882384286
:101660000BD10C9B198A494A0A4010A9CA821968F1
:101670004905C90C0D9A11431691324C2921615C20
:10168000002908D03037B84205D010A908461130DB
:10169000123107F0D7FDE77A2A48047BE51929487B
:1016A00000790E9027484078401C2946FEF712FD2D
:1016B00088000D9A10431890079961433801104330
:1016C00040182049497B4E4380191C21694340182A
:1016D0000E9909191B4B1E4A12884A43801817900D
:1016E000099A0C998A60987B002800D04A62987900
:1016F000401C9871187B99798142069F00D39A719A
:101700005978491C5970D97A0818597888420E4D71
:1017100000D85A70187A401E18722820185C0028C9
:1017200004D0996B002901D010A88847089A174265
:1017300002D00F98000328601C480449486019B083
:10174000F0BDC046E8A6010228A000503CA1005010
:10175000E4A6010248572045542069647820256496
:1017600020616E64204554206964782025642069D6
:101770006E2052582064657363206D69736D6174C7
:1017800063680D0A0000000038200040FF030000DD
:1017900094300040C8930102604000404D41432016
:1017A0004556542025782025780D0A00FFFFFF03B9
:1017B000F0B5A5B01E460C9208910024239422A9EE
:1017C0000C8016A90C8024A909250D80598C0D9137
:1017D000FEF780FC2A99012900D0DFE03189012938
:1017E00000D0DBE0318C012900D0D7E00D99002931
:1017F00000D1D3E0224607962C990B912B990691A4
:1018000080B205900F9415A8058090000E900C9959
:101810000C582E460025204629461746FEF734FF71
:101820000028119636D12C200A9778430899081879
:1018300017A90A4668C868C2E8C8E8C2E8C8E8C28A
:10184000079F119880B280000E5822AD019523A801
:10185000009020463946059A069B02F0C7FF0F9874
:10186000401C0F90288800282DD03B8A239913AC68
:10187000039416A8029014A8019015AE009617A81C
:1018800024AA03F08DF92588308811900120149E38
:101890000A9A05E013A8058014952E4628463A4674
:1018A0000E9F51000B9B119C5C52591808830D84AC
:1018B000D81986600F981885521C0D9882426DD0F9
:1018C00024A805889FE7099616A800250580149589
:1018D00024A80688239812902F46109503E06D1CCB
:1018E000A8B2B04213D8A8B2800017A90C5820465D
:1018F0001299FEF7D7FE0028F1D1002FEFD115A8DD
:10190000058016A80127078014941094E7E715A80E
:101910000288B01A012805D115A80680099F1497DE
:10192000119628E010200799095E0129119221DB08
:10193000551CA8B20C18109F0E9B099403E06D1C57
:10194000A8B2844218DDAAB2B242F8D8800017AA21
:1019500010581090394634461E46FEF795FE334621
:101960002646099C0028EAD115A80580109F1497E7
:101970001195E4E7109F0E9B1C463E46384612998F
:10198000FEF7B2FCFEF73CFF0546052800D305250F
:1019900013A8058001200A9A274682E725B0F0BDEA
:1019A000F0B58BB00243159A149C139E2BD00546BC
:1019B00001A856C0129CD869196A09900A911E465E
:1019C0009F6B0123009309A807AA0146059304F021
:1019D00061FF716C3846FEF787FC0746E06A616B71
:1019E000FEF782FC002D069613D00446119801994B
:1019F000012924D10921081A0421069A515E88423E
:101A000029D16425B1E000203080207010700BB027
:101A1000F0BDB08800226425002829D005926949CC
:101A20003846FEF75BFE0028049C039E6FD1664992
:101A30003846FEF753FE00281DD05A2567E03C25A6
:101A4000082800D191E05F492046FEF747FE0028B4
:101A500019D0502589E00A291DDB1D293BDC594995
:101A60003846FEF73BFE0022002854D05A253AE0C3
:101A70003346049C39E055493846FEF72FFE0028CE
:101A800021D0502543E050492046FEF727FE00288C
:101A90002ED0462569E03C25012866D049492046DC
:101AA000FEF71CFE0028D4D147492046FEF716FE5B
:101AB0000028EED145492046FEF710FE002854D1FB
:101AC000434920466EE042493846FEF707FE0028AB
:101AD0001CD128251BE03B493846FEF7FFFD0022BC
:101AE000002832D05025049C069B0299039E41E0B9
:101AF00036492046FEF7F2FD002836D1344920460B
:101B0000FEF7ECFD00282FD114252EE03725029991
:101B1000059A069B2EE005922B493846FEF7DEFD1E
:101B2000002896D129493846FEF7D8FD0028B0D1C3
:101B300027493846FEF7D2FD0028049C069B0299EF
:101B4000039E059A3BD11E2514E005921E49384696
:101B5000FEF7C4FD00289CD11C493846FEF7BEFDA7
:101B600000281DD03C2500E02325049C069B0299FB
:101B7000039E059A25803270002008703078002876
:101B80000CD118681349FEF79BFD002806D1208868
:101B9000102803D30F3820800BB0F0BD0BB0F0BD80
:101BA0000B493846FEF79AFD0028049C069B0299D3
:101BB000039E059A01D11425DCE72325DAE72D25BC
:101BC000D8E7C046CDCCCC3DCDCC4C3DCDCCCC3CEB
:101BD0000AD7233C0000204070B588B00C4606466A
:101BE0004088002820D0FEF7CCFD059005A804A968
:101BF00001252A4605F0B8F83088B188081AFEF7A2
:101C0000B5FD0390049903A807AA2B4605F06CF8CC
:101C10005249079D2846FEF761FD002808D0BF20E5
:101C20000006206008B070BD0020206008B070BDC4
:101C30004B492846FEF736FD002804D03F20000619
:101C4000206008B070BD47492846FEF747FD0028D0
:101C500001D0002010E000212846FEF73FFD0028BB
:101C600001D0022008E040492846FEF737FD002851
:101C700001D0042000E0062001957F21C9050291D2
:101C800080003A49091801A806AA022304F0E0FFDF
:101C90000698206008B070BDF0B587B00C460546C8
:101CA0004768002638463146FEF726FD002802D058
:101CB000266007B0F0BD049704A803A901263246A8
:101CC00005F052F8A8682968FEF7C9FA029003994E
:101CD00002A806AA334605F007F82049069D2846C3
:101CE000FEF7FCFC002804D0BF200606266007B0E3
:101CF000F0BD1B492846FEF7D5FC002804D03F2044
:101D00000606266007B0F0BD16492846FEF7E6FC39
:101D1000002801D0002010E000212846FEF7DEFC5C
:101D2000002801D0022008E00F492846FEF7D6FC23
:101D3000002801D0042000E0062000957F21C9057D
:101D40000191800009490918684605AA022304F098
:101D50007FFF059E266007B0F0BDC046CDCC0C3F8E
:101D6000295C0FBFCDCC4C3ECDCC4CBED0930102F4
:101D7000F0B587B00C4606467F270088002801D0C2
:101D8000FD0503E0B08800282ED0334DFEF7F9FCA6
:101D900003907088FEF7F5FC049003A802A90126C1
:101DA000324604F0E1FF029904A806AA334604F083
:101DB0009BFF2A49069E3046FEF790FC002802D081
:101DC0003F20010641E026493046FEF76BFC002823
:101DD00002D0BF20010638E022493046FEF77EFCE3
:101DE000002805D0002024E00020206007B0F0BDCE
:101DF0001D493046FEF772FC002801D0022018E091
:101E00001A493046FEF76AFC002801D0042010E091
:101E100017493046FEF762FC002801D0062008E092
:101E200014493046FEF75AFC002801D0082000E093
:101E30000A200096F905019180000F4909186846AB
:101E400005AA022304F004FF05992846FEF70FFABD
:101E5000206007B0F0BDC046000080BF00003843DE
:101E60003333733F0000C84200007042000020423C
:101E70000000A0410000C040F0930102F0B59DB009
:101E800015460B917F210391C9051C9102911B916D
:101E900019A900248C80199418941794598C0691D0
:101EA000198C0F91DE8B998B0791997805911F887A
:101EB0002B21CA432799914201DB7F0015E0402284
:101EC000D243914211DC4922D243914202DB79088C
:101ED000CF190AE05322D2439142EEDA5D22D24377
:101EE000914201DBBF0000E0FF000A971396269E97
:101EF000597E00290BD0002132460F46D1709170D7
:101F000051701170121D7F1C5C7EA742F6D30C939A
:101F100011952599149122990D91159041088C42A3
:101F200011D2FD4A2346A00084583454270A451C88
:101F30007755250C871CF555240EC01C34545B1CAA
:101F40009CB2A142EFD823981090012009900090F4
:101F500030463146149A159F3B4604F0A9FC0D9873
:101F600000060890400E139D00D186E068000490A2
:101F7000002F3FD0002210461146144606E01C46B2
:101F80001146159F401C82B2BA420ED283B2AB42B8
:101F9000F8D09200149B9A5E0FB2BA42034600DC5E
:101FA0002346BA42EBDC0A46E9E7002F25D000229F
:101FB00010461146129206E012931146159F401CDE
:101FC00082B2BA4214D283B2AB42F8D0A5B2AB42CD
:101FD0000CD09200149B9A5E0FB2BA42034600DC0A
:101FE000129BBA42139DE7DC0A46E5E7139DE6E73C
:101FF000129903E00024214600E00021129110987C
:102000000183C4828582049FF057FEF7AFFB7921DC
:10201000C9050E91FEF72BF91099C861099807437D
:10202000F057FEF7A3FB0E99FEF721F9109F3862D7
:102030002004C40B3057FEF799FB0E99FEF717F9F1
:102040007862601C3056FEF791FB0E9C2146FEF72D
:102050000EF9B86212980004C70BF057FEF786FB22
:102060002146FEF704F9109CE062781C3056FEF71A
:102070007DFB0E99FEF7FBF82063119805800C9804
:10208000407E410000278D4228463A46149E1ED3CA
:102090000A9880B28AB29300F45E84420BDA491C3B
:1020A0008AB2AA42F6D9002728463A4681B2691A6E
:1020B000012910D01BE0F018119B19800788080433
:1020C0000FD0500040008019001F0288084681B2DE
:1020D000691A01290BD1A800301811990D800788C1
:1020E00026E00020024681B2691A0129F3D00A993C
:1020F00089B2079B4B43BB421AD306998A4217D831
:102100000599002914D0401C82B2891803E0401CB4
:1021100082B291420CD983B2AB42F8D89200B35E3E
:10212000BCB2A342F3DDB218119B18801788EEE70A
:1021300012970B980580119800882B1A002B16DD3A
:1021400002210F9A1143032942D10E93411C421ED2
:1021500010B281420EDA0E98032824DB0C98808C92
:10216000012820D019A818A9FFF736FD1FE000208C
:1021700018902BE00026F443374608E0B8B2400040
:1021800019AD2B527F1C521C10B28142E3DB13B2FB
:10219000A3423346F2DD159B98423346EEDA8000C7
:1021A000149B1B5AEAE719A818A9FFF7E1FD149E32
:1021B000139D0F9A012A13D0032A11D0022A04D1A9
:1021C00011980088281A02280ADA0020179034E0B3
:1021D000022A01D1022BB8DA00201890012AEBD193
:1021E000681C691E0FB2B84208DA0C98808C01286E
:1021F0001DD119A817A9FFF7BBFD1CE00022D3438E
:10220000144608E0A5B26D0019AF7E53641C491C4A
:102210000FB2B842E9DB0DB29D421646F2DD159DC4
:10222000AF421646EEDABD00149E765BEAE719A8C7
:1022300017A9FFF7D1FC149E139D249F189C179992
:102240002046FEF70CF80F99012900D82046386087
:102250000D98002800D1CBE011990888109FB8860E
:102260000888281AB880129880B2FEF78AFA792175
:10227000CC052146FDF7FBFF2146FDF7F8FFB863CB
:10228000119F3888002849D081008919091F0988C1
:10229000129C0C191599884203D2800080198088FD
:1022A000041915984300534916AA304604F0DEFC81
:1022B000169810994864FEF7BCFAA4B2A04201D166
:1022C0004D480FE0001BFEF75CFA1C901CA81BA9F0
:1022D000012204F049FD2046FEF753FA01461B98FF
:1022E000FDF7C5FF109908603988491B4A1C92B256
:1022F000032A02D20021159F17E009B20229159F77
:1023000012DB3F210906FEF7E9F9002802990CD1FA
:102310000998810709E0C046402100400020129C36
:1023200015998842B9D3BCE73449109801610898DF
:10233000800E5DD0002F1CD000221146144610469E
:102340004B1B1DB2ED135B196B40139D1BB292002A
:10235000B25E53431818A418491C8AB2BA42EFD38C
:10236000FEF70FFA06462046FEF70BFA002C03D1C3
:1023700000E000260398C0051C901CA81BA901259D
:102380002A4604F0F1FC1B9C20463146FDF76FFF06
:10239000014610988160002F119422D00024274616
:1023A000264613951291B8B2FEF7EBF91299FDF794
:1023B00056FF0546A0001499085EFEF7D7F90146BE
:1023C0001398C00785432846FDF751FF0146304664
:1023D000FDF7F4FE06467F1CBCB215988442E2D39A
:1023E00000E0002611983146FDF741FF1099C860C2
:1023F0001DB0F0BD7CA00102000020410000404063
:10240000F0B58FB00692F74A09AF70CA70C770CAAC
:1024100070C70328079320D88800F3A10858F6490D
:10242000FDF7CCFE0446F549FDF7C8FE0D90F449D2
:102430002046FDF7C3FE0C90F2492046FDF7BEFE94
:102440000B90F1492046FDF7B9FE0A90EF4920466E
:10245000FDF7B4FE0990EE4969E0042822D0062871
:1024600020D88800EBA10858EE49FDF7A7FE0446E6
:10247000ED49FDF7A3FE0D90EC492046FDF79EFEC9
:102480000C90EB492046FDF799FE0B90E949204658
:10249000FDF794FE0A90E8492046FDF78FFE09906B
:1024A000FD4944E00838022821D88800FBA10858DB
:1024B000D149FDF783FE0446FC49FDF77FFE0D90F0
:1024C000FB492046FDF77AFE0C90FF20810520464F
:1024D000FDF774FE0B90F7492046FDF76FFE0A905A
:1024E000CA492046FDF76AFE0990FE491FE08800B0
:1024F000F1A10858F449FDF761FE0446F349FDF7E0
:102500005DFE0D90F2492046FDF758FE0C90F14912
:102510002046FDF753FE0B90EF492046FDF74EFE97
:102520000A90EE492046FDF749FE0990EC490094D7
:102530002046FDF743FEEC4909680E90EB4804681D
:10254000EB4801684808EB4F05463D400022002D4E
:1025500008922DD0CA01120E07D0280CE90D12D115
:102560004000E649085AE6490AE0C903090E0CD0C2
:10257000280AE90B10D14000E049085A8F21890050
:102580004018E4300DE0DC490AE081B27F2905D82B
:102590004800DA49085A04E0D94901E08F2189004E
:1025A000401800B2FEF7E2F8D649FDF760FE024699
:1025B0000292039507252606D34B1A68002A08982D
:1025C00040D0791C8A420BD21102090E13D0110C93
:1025D0001F46D00D1FD14800C849085AC84907E016
:1025E0001F46110E002A13D44800C449085AC24994
:1025F0004018E4301FE011041F46090E0ED0110AE6
:10260000D00B12D14800BD49085A8F218900EFE74D
:10261000BE4808180FE0B84808180CE091B27F29AE
:1026200006D84800B549085A05E0B548081802E040
:102630008F218900501800B2FEF798F8B149FDF7D4
:1026400016FE3B460590159F2C40F50E5B69B04980
:102650001940089810D0DA02D20E34D0C80B3E21AF
:102660000140A648405AA6494018E43000B2FEF79F
:102670007DF8A449FDF7FBFD0490149E6800A5A118
:10268000085EFEF773F80146A00009AA1058FDF78E
:1026900095FD0146B8B20128089F019102D1022C94
:1026A0000AD9A74F052C24D1189808900C2D20D8B2
:1026B0000B2D16D3A44918E00027022C089718D038
:1026C0008120C70515E01A04120E00D1CAE0080ADD
:1026D000C90B00D0CDE040008849085A8F218900FD
:1026E000C2E7092D00D2C7E096490898FDF766FDBC
:1026F000089001200021B542034600D30B46052C6B
:1027000000D308461799169A1A9C199D1843069BE0
:10271000012B12D1079B402B22D1002840D03846F4
:10272000FDF74CFD01460198FDF748FD0146009874
:10273000FDF795FD059A04998AE0079B402B1FD170
:10274000002838D03846FDF739FD01460198FDF7DD
:1027500035FD01460098FDF782FD059A049977E062
:10276000002833D03846FDF729FD01460198FDF7D2
:1027700025FD01460098FDF772FD059A049967E072
:1027800000285BD03846FDF719FD01460198FDF79A
:1027900015FD01460098FDF762FD059A049957E082
:1027A00002981146FDF75BFD0399002900D16748A7
:1027B000059A04994CE002981146FDF750FD0399E3
:1027C000002900D16148059A049941E00298114618
:1027D000FDF745FD0399002900D15C48059A04994D
:1027E00036E0C04688C00000000068C1000088C113
:1027F00066665EC1000084C1000084410000B441EF
:1028000000004841000020400000F0C0000084C1EA
:102810000000F841333323C1000050C19A9929C107
:102820009A9949C19A9949413333CB4166667641B9
:10283000CDCCAC40333393C09A9949C1029811462C
:10284000FDF70DFD0399002900D14048059A049930
:1028500028601046FDF703FD0899FDF700FD206094
:102860000FB0F0BD99B27F2911D848002349085A0A
:10287000FCE623494018F9E6C12001060898FDF757
:102880009DFC0890062D00D933E7002030E78F210A
:1028900089005818EAE6C0463333F341000058C1B6
:1028A0009A9961C19A9969C1000084C10000AC4144
:1028B00000003841000008C1CDCC80C1CDCC88C11A
:1028C00033338FC1333397C133339741CDCC8C41F0
:1028D0003333F3409A9919C0666646C1333397C1C2
:1028E000CDCCB4410000D4410C0000405030004039
:1028F00068400040FFFFFF007C08000000C40000AB
:102900005C050000919AF63C642000409C0B00009E
:10291000FFFF1F00FAFFFCFFFEFF000002000400A3
:10292000060008000A000C000E001000120014003F
:10293000160018001A001C001E00200022002400AF
:10294000000080BF0000A0C0000040C00000DCC24A
:10295000F0B5FFB0ECB017460E460D900021E9919E
:10296000E891DC9199919891979196911491139196
:1029700012919AA8F49DF39CF29A002E00D1E6E100
:102980000B938030F09B1180099529602546DBACC4
:10299000218095AC21800C952980DA917F24E40573
:1029A000B994B894B794B694B594B494B394B294DB
:1029B000B194B094AF94AE94AD94AC94AB94AA940B
:1029C000A994A894A794A694A594A494A394A2943B
:1029D000A194A0949F949E949D949C949B949A946B
:1029E000046644668466C466046744678467C46793
:1029F000046444648464C464046544658465C46593
:102A0000046244628462C462046344638463C46392
:102A1000046044608460C460046144618461C46192
:102A2000B0090B250B2800D3AE011095012B0B9D8F
:102A300000D070E12B89012B00D06CE1298C00299A
:102A40000E9200D18BE16B8C002B00D1FAE1AA8CA5
:102A50003021695C002900D188E10892109F5F4312
:102A60001196304639460F93FDF734FB0590FDF77C
:102A70007DFE01462046FDF737FC8321C905FDF7A1
:102A8000F6FB064696A8021D119887420A9200D8C6
:102A900079E155A811909AA9069196AF15463A4644
:102AA000059C234604F0D4F815A80F9006992A46F1
:102AB000234604F0CDF802230D93384631463A46BA
:102AC00004F012F9012308930093E8AA1092384603
:102AD000394603F0DFFEE898DD901198069D2946FF
:102AE0003A46234604F0B4F80F9829460A9A23463A
:102AF00004F0AEF8384631463A460D9B04F0F4F83F
:102B0000089B009338463946109A03F0C3FEE898B4
:102B1000DE9011982C4629463A46059D2B4604F036
:102B200097F80F9821460A9A2C462B4604F090F805
:102B3000384631463A460D9B04F0D6F8089B009380
:102B400038463946109A03F0A5FEE898DF901198B0
:102B5000069D29463A46234604F07AF80F982946FE
:102B60000A9A2346254604F073F8384631463A4619
:102B70000D9B04F0B9F8089B009338463946109A2B
:102B800003F088FEE898E0901198069C21463A46AA
:102B90002B4604F05DF80F9821460A9A2C462B46E6
:102BA00004F056F8384631463A460D9B04F09CF83E
:102BB000089B009338463946109A03F06BFEE8985C
:102BC000E1901198069D29463A46234604F040F8C4
:102BD0000F9829460A9A2346254604F039F83846C4
:102BE00031463A460D9B04F07FF8089B0093384627
:102BF0003946109A03F04EFEE898E2901198069C30
:102C000021463A462B4604F023F80F9821460A9AAB
:102C10002B4604F01DF8384631463A460D9B04F029
:102C200063F8089B009338463946109A03F032FE49
:102C3000E898E390119821463A462B4604F008F8AC
:102C40000F9821460A9A2B462C4604F001F8384684
:102C500031463A460D9B04F047F8089B00933846EE
:102C60003946109A03F016FEE898E4901198069DF4
:102C700029463A46234603F0EBFF0F9829460A9A65
:102C80002546234603F0E4FF384631463A460D9B7D
:102C900004F02AF8089B009338463946109A03F04E
:102CA000F9FDE898E5901198069C21463A462B4696
:102CB00003F0CEFF0F9821460A9A2B4603F0C8FF77
:102CC000384631463A460D9B04F00EF8089B0093B7
:102CD00038463946109A03F0DDFDE898E6901198E1
:102CE00021463A462B4603F0B3FF0F9821460A9A35
:102CF0002B4603F0ADFF384631463A460D9B03F0B4
:102D0000F3FF089B009338463946109A03F0C2FD42
:102D1000E898E7907AE010880C9A10809991989141
:102D2000DA9E08460F46099DF59CFDF798FA286043
:102D3000DC9827606060A6600C34DDA80EC80EC465
:102D40002EC82EC42EC82EC47FB06CB0F0BDFF209C
:102D500010800021296020807FB06CB0F0BD00227F
:102D600001233021695C002900D076E6DDAA1ACF64
:102D70001AC23ACF3AC23ACF3AC20B213046FDF7D7
:102D8000A9F9054642E000200690059D0796089F98
:102D90001190069801460D9C0F9A4A43D219109B38
:102DA0005A43119BD218D200A35889002E4655AD24
:102DB0006B503546121DA25815AB5A50401C01B23B
:102DC0008E42E9DC55A89AAE96AC314622462B4697
:102DD00003F03EFF15A831460A9A2B4603F038FF50
:102DE000022320460799224603F07EFF0123009329
:102DF000E8AA2046214603F04DFD119B9800DDA96D
:102E0000E89A0A505B1C0B2B1846C1D1F19EDDA835
:102E10009AA9DCAA0B2303F01BFF09210E980F913E
:102E200001800B98C168DC9C2046FDF720FA014622
:102E3000A8B2E69F0F281BD808280DD30846FDF737
:102E4000BDF914E0FF2010800021099A11600C994F
:102E500008807FB06CB0F0BD042803D381220846FF
:102E6000D10502E0412208461106FDF700FA0146AD
:102E70002B20C04386420D9704DB0846FDF79EF9E0
:102E8000014603E04020C043864244DD0E9A0C9C7C
:102E90000B98408A002811D00B98038A95A80390BC
:102EA000DBA80290DAA801900094DDA80D4601F09D
:102EB00077FE29462488DA9E099D68E011910F98D3
:102EC000208000273D46109705E00E9804887F1C5F
:102ED000B8B2A04211D8B8B28000DDA90C58204683
:102EE0001199FDF7DFFB0028EFD1002DEDD10C98F3
:102EF000078001250F971094E7E7DBA805800F9A5C
:102F000090B2201A012811D10C9804800D9FDA97F5
:102F10003E46099D3AE04920C043864200DA8BE0F4
:102F2000FF2208469105FDF7A2F9A9E710200B99A9
:102F30000E5E012E00DA90E0551CABB21846A1B22D
:102F4000AAB28A4217D805E00E990C88A1B2AAB29B
:102F50008A4210D88000DDA90C58204610991F46DF
:102F6000FDF792FB3B46002805D10C9805800B9895
:102F7000068A0F95109430B2C1186D1CA8B2814218
:102F8000E2DC109EDA960F9C099D0D9F1199304648
:102F9000FDF7AAF9FDF734FC052800D3052095A913
:102FA0000880A0B20E990988814218D9401C611E80
:102FB0000CB2A04218DA12A898A9FEF76DFE0E987E
:102FC0000188481C491E0CB2A04221DA12A899A916
:102FD000FEF762FE99999898099D0D9FA4E600213D
:102FE0009891999108469FE60022134608E09CB20A
:102FF000A40012AF3D515B1C491C0CB2A042DADBAD
:103000008DB20A2D1546F2D8A400DDAD2D59EEE79C
:103010000022134608E09CB2A40012AF3D515B1C95
:10302000491C0CB2A042D1DB8DB20A2D1546F2D854
:10303000A400DDAD2D59EEE75320C043864200DBEE
:103040001BE70E460B9881692046FDF71DFB002803
:103050000C9C08D10B98808B07E01446099D0D9FAE
:103060001199109E93E70B98C08BFDF78AFB0146E0
:103070003046FDF7FCF8119021E70000F0B58BB069
:103080001C4609930E46034600200A9040480088DB
:10309000224F05970AA9049103940292109C01946F
:1030A000012500950B21414389B230331C4A30463B
:1030B000FFF74EFC3868079078680890B86806906B
:1030C00033480088334F009501940297324E3036D2
:1030D0003249334A3346FEF76BFB0698F86207988D
:1030E000386308987863099800882E4905912E491D
:1030F00004912E4903910297019000962C4B28468B
:1031000029462A46FEF74CFC432001060A98FDF7A3
:10311000AEF8FDF775FB0BB0F0BDC04644A0010250
:10312000B8B30102F0B589B00F9F0E9C002815D0EE
:103130001098079016480088164E012500950191B9
:1031400002960893144B30331449154AFEF730FBAE
:10315000089BF76207983063746303E00D48476388
:10316000C462002518880F4905910F4904910F4941
:1031700003910849029101900748303000900121E5
:103180000B4B28460A46FEF70BFC09B0F0BDC046C3
:10319000DAA601027CA80102AC99010200980102A2
:1031A00088A70102749D0102D8A6010284A601022B
:1031B0008CA6010280B5124801681F220A400260F5
:1031C00003200840022812D10E480268D30D02D015
:1031D000FF231B06D2180C4B1A600C4A12680C4BCA
:1031E0001A6080680B4A1080000C0B4A10801A4845
:1031F0008268002A02D082680020904780BDC046C5
:1032000074200040644000409CA7010278300040D8
:10321000A0A70102109A010272A8010280B50D4810
:10322000016889070FD5052101600B48C178002985
:1032300008D00021C170C168002903D0C26841686C
:103240000020904780BD054805A10B4A0BA306F05E
:1032500019FDC0462C040040B89301027DCF000048
:103260005048595F54494D45525F49525148616E2B
:10327000646C6572000000008D0A0000556E657870
:1032800070656374656420696E74657272757074BC
:103290000000000070B50446401E012814D8032029
:1032A000084011D13F2040030818050B2819802839
:1032B0000AD8164E317801204840294602F09AFC7F
:1032C000641E6D1C002CF5D170BDC04680B5002079
:1032D000014602F0B3F9002800D080BD0B4801215F
:1032E000017080BD70B516460C460546FF22FCF7FE
:1032F00053FF0548311805480278012050402A46FE
:10330000234602F01FFB70BD00E007047CA201020F
:10331000012000037047012040037047F0B583B0DF
:1033200030480068C16B0901890F01D003B0F0BDBE
:10333000C16BC06B2C4D05404800400F082602961B
:1033400086400227384601F073F901907043C10BA3
:103350004A1B26485043FCF7D3FE044606F076FB92
:10336000032123A238461F4F0091234607F0E8FCB3
:10337000F88A002817D0019840012946FCF7AAFED8
:1033800046431822324001200F2A014600D800216E
:1033900073095B181B4CA3420DD8194DED1A6D052E
:1033A0000F2A0CD80CE038680021C160112001F010
:1033B0002FF903B0F0BD5D1C6D050F2A00D95642F0
:1033C0002A0C029D2E4009018919A34202D80098B7
:1033D000000400E04004081880183968086303B04E
:1033E000F0BDC04648940102FFFF1F0040420F009D
:1033F00052434F33324B2070706D2025640D0A000C
:10340000FF070000FE7F0000B0B582B015490868D4
:103410008269D2070CD00122C2610D69002D07D04C
:1034200000686C46214606F003F900212046A847B3
:1034300002B0B0BDB0B582B00A490868026C92070C
:103440000ED5026C012313430364CD68002D07D011
:1034500000686C46214606F0EBF800212046A8479C
:1034600002B0B0BD489401020748016803229143AD
:103470000160016801220A43026008F023FB00F0AA
:10348000ADF806F005FBC0462800004080B50D49A8
:103490000868002810D5224802680423032A01D0B6
:1034A0001A4300E01A460A601E490A68002A02D040
:1034B00041680020904780BD03A00CA19E2211A36B
:1034C00006F0E0FB2C100140696E636C7564652F9B
:1034D000647269766572732F6D6B5F736C6565706E
:1034E0005F74696D65722E6300000000534C4545A2
:1034F000505F54494D45525F49525148616E646C6A
:1035000065720000556E657870656374656420733C
:103510006C65657020696E746572727570740000F8
:103520000890010278A80102B0B582B00446007884
:10353000002811D0094D01A908702868416A0029A6
:10354000FCD101A901220020034608F045F9611CC5
:10355000607800280C46EED102B0B0BD6094010244
:10356000F0B50C784D782D022C198D78C9780902A8
:10357000491909040C1981000D4D6C509478D578C7
:10358000167852780B4F7B50120292192B021B199E
:103590001B049A18084B5A50059A13785278074C16
:1035A000079D65501102C9184000054A1152F0BD2F
:1035B000E498010260B4010248990102FCB30102DF
:1035C000B098010280B504480168491C0160006997
:1035D000002800D0804780BDE4B301020148F149D2
:1035E000016070471890010280B582B00E490868EA
:1035F0000022C2600192CA68002A02D0016801A8B4
:10360000904702B080BDC04680B582B006490869C7
:103610000022C26001220192CA69002A02D0016818
:1036200001A8904702B080BDB8920102F0B589B000
:1036300008F058FCD04C607808F058FACF498A88D6
:1036400007A882800A88498809048918079104F02C
:10365000F3F96078052804D00222C949092804D169
:1036600004E00122C649092800D089184979207848
:10367000621C08F0FFFA607A05F0E0FDC148C2491B
:1036800003F008FDC14F387800260028049609D0C1
:10369000BF491A31BF4A034610CA0C80891C5B1E01
:1036A000FAD14600BC4DA872B88D6871797829703E
:1036B000B978E970000AA871481CB87028460B3028
:1036C000B34C21464C3105913246FCF753FD70193D
:1036D0000B30069421461A313246FCF74BFD202070
:1036E00068720498787138896870000AA870C326D7
:1036F000B40105F067FA03193B63387881000D3196
:103700000122284608F03BFCB8623D6B05F0F0F959
:10371000401905F0F5FE05460C469748007B05F07C
:103720007BFD81B2C90B401800B2C11740102818A8
:10373000B8666141F96605F045FAB86103F01AFC14
:103740000028FBD105F03EFAF861386B9349401828
:1037500078637D2005010020049001462A4608F088
:10376000E4FBB86205F02EFA31023A784A438C49FC
:103770005118B863F9630918481C00D0084638642A
:1037800005F020FA7864396C884203D3854A891899
:10379000884279D905F016FA786405F013FAF861D1
:1037A00003F0E8FB0028FBD105F00CFA3862B87989
:1037B000022855D0012860D10020B8717A4B597A7F
:1037C000212946D159799A7912025118BA8D91421C
:1037D0003FD179781A788A423BD1039559789A7803
:1037E00012025118F9813A78002A0AD0684B4C33FA
:1037F00000201D888D4204D09B1C401C8242F8D1C1
:103800001046C0B238823B6FB96CBA6E664D223535
:103810000095654D0191029229461A312A461E32C1
:10382000FFF79EFE3978388A884208D34200584B09
:103830009A18FB894C2553535B4D491C3970642100
:10384000534A115496212846FCF7ADFC002078829B
:10385000039D002001462A4608F067FBB8620CE091
:103860000020B87101462A4608F05FFBB86205F0F7
:10387000A9F9386205F0A6F9B8613A6C786C494943
:103880005118904284D285E7B86EF96EFDF7AEFA12
:10389000049CFC703A78002A68D03E4B254608E02C
:1038A0000698401C06900599891C05911B1D521E07
:1038B0001AD0069801780029F2D0491E06980170A6
:1038C000A800C9B2394E3150641C0494FC706900E0
:1038D0003C46059E3788364E77522746049C196829
:1038E000344E31506D1CDBE73C713C700494E0B207
:1038F0000590022822D30598401E0023069003E07D
:103900005B1C0698834219D02A490D68284E274A25
:103910000FE00F604D60778834887480378090CADC
:10392000083A17605460401E091DB61C121D00287D
:10393000E6D04F68BD42ECDC3D46F4E70498000653
:103940001A4C059D10D0124E30464C306A00184972
:10395000FCF710FCAA000F481649FCF70BFC01CC41
:103960003070761C6D1EFAD109B0F0BD00203871A0
:10397000387009B0F0BDC04662900102A0C00000DE
:10398000149A010251AF0000CD980000A0960102E8
:103990001897010224A70102D6BD0102A06D010003
:1039A000808509000026B803DCA70102DCBC010207
:1039B000A4BD010240BD0102B0B502F079FE154C74
:1039C000E060A178002900D0B0BD21790029FBD1A9
:1039D0000121217100281AD06425281AA16881428A
:1039E00015D0A0682018007D21698847A068401C78
:1039F000A060A068642801DB0020A060E168A068E6
:103A0000022D04D36422511A6D1E8842E9D1002090
:103A10002071B0BDC095010280B5002007F0B0FB59
:103A200080BD80B5012007F0ABFB80BDB0B582B092
:103A3000602833D0622843D0642854D101A82F498C
:103A40000180EFF3108072B600242046214601F079
:103A5000F5FD2B4D002805D1012002030020294649
:103A600001F046FD103501AA02232046294602F046
:103A700041FA62B623A0FFF757FD64201B490C52A0
:103A800005F07EFF1A4800F0A3FEBFF34F8F1948E0
:103A900019490160BFF34F8F00BFFDE76020134954
:103AA00000220A5205F06CFF114800F091FEBFF3AE
:103AB0004F8F104810490160BFF34F8F00BFFDE7E3
:103AC00062200A4900220A520A8005F059FF08487C
:103AD00000F07EFEBFF34F8F064807490160BFF339
:103AE0004F8F00BFFDE702B0B0BDC0467EA201020D
:103AF000A08601000CED00E00400FA05AAAA00006F
:103B000000D00204BDF8C8EBC9FDBCB6C4A3CABD51
:103B10000D0A0000F0B581B0644FB96808291BD8C0
:103B20008A0001A39A5897464D3B0000593B00007C
:103B3000593B0000693B0000933B00009F3B0000A5
:103B4000A93B0000773B0000B33B0000552848D15B
:103B50000120B86001B0F0BDAA2838D1012936D1C2
:103B60000220B86001B0F0BD0421B9600021B97035
:103B7000787001B0F0BD39797A181073481C38712B
:103B8000C0B27978491F81422FD10820B86001B0B6
:103B9000F0BD0521B9604649087001B0F0BD0621AD
:103BA000B960B87001B0F0BD0721B960387001B0DC
:103BB000F0BD797806291AD34B1F002422463D19FF
:103BC0002D7B521992B2641C9C42F8DB10E0032852
:103BD00007D1022905D10120F8700320B86001B097
:103BE000F0BD0020B870B860787001B0F0BD002260
:103BF000101841182E4800780918BD7849193C78EA
:103C00000919FA78002A00D0C91CC9B2FF2945D188
:103C1000012819D0022841D12748401939460C31D2
:103C20002246FCF7A7FA387B012802D12846FFF785
:103C3000FDFE05F0A5FEBFF34F8F2048204901602F
:103C4000BFF34F8F00BFFDE71A4EB47103203071F0
:103C5000B070AA2070705520307068087071651DB2
:103C6000F570400014490918F01D2246FCF782FA4D
:103C7000301DE11CEAB2D21C037892B2D218401C6B
:103C8000491EF9D1A019D143C171090A0172093441
:103C9000002031462246034607F09EFD0020B87002
:103CA000B8603871787001B0F0BDC046509501021F
:103CB0001C900102999701027EA201020CED00E026
:103CC0000400FA0580B582B0002001900448C26863
:103CD000002A02D001A80021904702B080BDC04652
:103CE000F0940102F0B583B000242046FFF7EEFA0D
:103CF000FFF711FB274EB060FFF70AFB7060264FFD
:103D00000BE001A8C1888088084319D101A8408828
:103D100024180834B068844235D201AD0821284601
:103D20002246FFF7DFFA28880028EAD0B8422AD0D6
:103D300001AD0421284600F035FDA9888842E5D070
:103D40003460B06884420CD201AD0221284622467C
:103D5000FFF7C8FA2888B84203D0A41CB068844290
:103D6000F2D370682118491E4042084030600DD0DF
:103D70000024254601202946FFF78CFA03CE4D1971
:103D8000083E8542F6D3346003B0F0BD00243460B1
:103D900003B0F0BD90960102FFFF0000F0B585B0C2
:103DA0001F4604920646C8170C1844400A2C03917B
:103DB00014D301250A212046FCF78CF96D1C632CD5
:103DC0000446F7D804998D4200D329460A9C002F57
:103DD00009D00398002808D4002207E0012504999F
:103DE0008D42F2D2F2E7002205E0012204232340B3
:103DF0009B081343FA1A02232340049800280294D4
:103E000012D1002B10D0F468002C62D40398002843
:103E100025D40298400734D57068B5686F1C874276
:103E20002FD830682B2423E0E407ECD1002A0AD1F4
:103E3000E9E7376820203855B560F068441CF46025
:103E4000521E002CDFD49142DDD27768B468651C25
:103E5000BD42EED9F468521E002CF4D5D3E740429F
:103E600003907068B5686F1C87420AD830682D24AB
:103E70004455B760F068441CF4600025ED43A84247
:103E800027DB002B1CD00120029B1840049B184309
:103E900016D1002A03D113E0521E002C0ED49142F9
:103EA0000CD27068B3685D1C8542F5D83068302448
:103EB000C454B560F068441CF460EDE7002C08D4ED
:103EC0000092029801900A2230460399049B00F068
:103ED00003F805B0F0BD0000F0B587B01F461546E9
:103EE0000290012406919142009407D30124069880
:103EF0002946FCF7EFF8641CA842F9D20D980C9AF9
:103F0000BC42039700D3039400990140002A00911A
:103F100009D00029029C25D12021800705D408461C
:103F2000002F11D004E0029C1CE03020002F0BD0A9
:103F3000084609E023685854A260E168491CE16022
:103F40003246721E00290DD4039991420AD21646B8
:103F50006368A1684A1C9A42ECD9E1683246721E35
:103F60000029F1D5E068002859D40590012401E02A
:103F70007F1E6C43022FFBD2069821461646FCF7A3
:103F8000A9F83246A842F4D2029880680490069FAD
:103F90000195069738462146FCF79CF8049D691C5C
:103FA000029F7A68914206D9069F059A019D059263
:103FB000002A0ED516E01B4A125C3B685A55B960C0
:103FC000FA68521CFA600491069F019D0592002A2E
:103FD00008D460433F1A20462946FCF77BF8AC42E0
:103FE0000446D6D200980028029C059B049D16D05A
:103FF000002E14D0701C01E0002B10D4401E039939
:1040000081420CD2691C62689142F5D82268202353
:104010005355A160E268531CE3600D46ECE707B01E
:10402000F0BDC04638C3000070B5002801D00120A3
:1040300070BD0C461625284600F0F2FA284605F019
:10404000E9FA002C05D01B48183014222146FCF751
:1040500091F828211748415C002915D041680029B2
:1040600016D403220B469343144A9C588D07ED0E39
:10407000FF26AE40B4439C501F220A4001219140CC
:104080000F4A11600F4A116001210161002070BDCB
:104090008A07D20EFF2393400F220A40083A0321D9
:1040A0008A43054954589C43545001210161002022
:1040B00070BDC046209001021CED00E000E400E06D
:1040C00080E200E000E100E05A21014A50527047CE
:1040D000AC990102F0B581B013490A78002A13D0D7
:1040E000052A01D104220A709300CD18561C002322
:1040F0001C462F686F60F917DB194C412D1F761E87
:10410000012EF6DC084902E00022134614464860FE
:10411000521C0A70C11718186141D2B20023FCF773
:1041200003F801B0F0BDC046209501025C21B748FC
:104130000022425282847A2141840284C283028313
:10414000C2820282114941608260C2603D214904FD
:1041500041834182090C8183818270475C21AB4895
:104160000022425282847A2141840284C2830283E3
:10417000C2820282054941608260C2603D214904D9
:1041800041834182090C8183818270474C373737E4
:1041900070B5D9484C21016001252C02601C00F04B
:1041A000BFF9322000F014FB00F078F9284600F047
:1041B0007FF9284600F08EF800F06AF90C4800F00C
:1041C000AFF900263046314600F0BAFA28463146AB
:1041D00000F0B6FA204600F0A3F9022000F0A0F9A2
:1041E0004834204605F0C6FC05F024FD70BDC046ED
:1041F0000102000010B50446072106F0FDFB074848
:104200000460032406A22046214606F099FD0AA276
:104210000F4B2046214606F093FD10BD8896010203
:1042200048656C6C6F2066726F6D204D4B53454D29
:1042300049210D0A000000004275696C6420696E16
:10424000666F726D6174696F6E2025730D0A0000D0
:10425000D8E0000010B505200424214602F0CCFA75
:104260000620214602F0C8FA0A20214602F0C4FACC
:104270000920214602F0C0FA00240121204602F064
:10428000BBFA02212046224602F0DEFA10BD80B5BC
:10429000072002F085FA80BDB0B5094D6A68002A92
:1042A00003D01120022102F00BFA0724204602F06D
:1042B00087FA05F0BFFC2868214606F09DFBB0BDDB
:1042C000889601020248016801229143016070470B
:1042D0005800004002490A6802408242FBD1704700
:1042E00004600040B0B5494D28688107484C0ED5A0
:1042F00028797F21084022688A43101820602368AB
:104300000B4002200321434A06F01AFD286880046E
:104310000ED55E20285C7F21084062688A43101811
:10432000606063680B40022003213B4A06F008FDF1
:10433000172000F075F93948016802220A4301216B
:104340008A43026036483749016037480021C1710D
:1043500081791F2529408171817A427C837C1B02EF
:104360009A18C37C1B04D218037D1B06D2182F4B4E
:104370009A4218D1427B837B1B029A18C37B1B0491
:10438000D218037C1B06D218294B9A420BD1C27A51
:10439000037B491E122906D819028918254A914221
:1043A00001D1202101720178CA0602D110221143E5
:1043B00001701C3C20682021884320601E481F4952
:1043C000016041680029FCD503F0A6FA04460220EA
:1043D00003211BA2234606F0B3FC0A20C441032C90
:1043E00005D8022003211DA206F0AAFCFEE718480A
:1043F000C1680F229143C1600168164A0A400260F9
:1044000019200001144948600D60B0BD149A0102E2
:10441000480000402CCB000016CB000004020040F6
:104420000C060040AF6B100A6B0001404D3836504F
:10443000312E32360734000000600040FE1C008040
:10444000436869702049443A20253038780D0A00C5
:10445000C8600040FEFFC3FF0C0400404F6C6420A6
:1044600063686970206D6F64656C206973206E6F7E
:104470007420737570706F72746564206279207433
:104480006869732053444B2121210D0A000000006C
:1044900080B5172000F0BCF8002080BD10B51724AF
:1044A000204600F0BDF8204605F0B4F8002010BD0D
:1044B0000121C907014301480160704700600040C5
:1044C00010B582B003460C480168022B01DD0122C1
:1044D00004E00222D24393420CDCFF227F248A189C
:1044E000A14322408918016000920448032104A2DC
:1044F00006F026FC02B010BD480000400208000093
:104500005854414C206C6F61642063617020747555
:104510006E65202564203A2025640D0A0000000005
:1045200010B5C1B2000AC2B202290CD0012913D0C1
:10453000002930D1911E7F4802291BD20121032A74
:104540002AD0490429E07B484168002A1FD002464E
:10455000203A1143416010BD76480168D31E022BFA
:1045600010D3012A29D0002A41D101229207914378
:10457000016010BD002A16D10121490702688A4353
:10458000026010BD0123042A1FD05A041EE001223C
:1045900092079143416010BD0904194A7F32C36AF2
:1045A00013405918C16217498A699207FCD5012145
:1045B000490702680A43026010BD052212079143B1
:1045C0000246203A0A43026010BD1A04836A0C4C6A
:1045D0001C40A21882620B4A131F00241C600A4B65
:1045E0000A4C1C600D235B0214681C431460054ACE
:1045F00093695B06FCD5052212071143016010BDCB
:1046000080FFFCFF1402004004010040FF0F000087
:1046100001218140474802688A4302607047C046D2
:1046200001218140434802680A4302607047C04646
:1046300010B5052811D8C046784400794000874459
:10464000020E192434393B490A680868C0003CD579
:104650003A4820390A425DD03BE0002010BD354980
:104660000A680868C00035D534480B46203B1A421A
:1046700037D134E02F490A680868C00036D52F4882
:104680000B46203B1A424CD135E02A494C680120A8
:10469000C0030A680B46203B1C421AD00C68E40099
:1046A0003BD5264C1A423CD03AE022480068012013
:1046B000C00310BD1F490A680868C0001ED51F4806
:1046C0000B46203B1A4220D11DE01B4820390A42EC
:1046D00020D010BD18480B46203B1A4201D10120C2
:1046E000C00349688900890FC84010BD12480B46B5
:1046F000203B1A4215D10120C00312E00E480B46A0
:10470000203B1A4201D10120C00349680903890FE7
:10471000C84010BD0120C00310BD074C1A4200D094
:1047200020464A689200920FD04049680901890FDB
:10473000C84010BD20000040006CDC020026B80319
:1047400004282CD8164AC046784400794000874493
:10475000020A121A21000320000713688343880706
:10476000800818181AE0032080061368834388071E
:104770000009181812E00320800413688343880797
:10478000000B18180AE0FF20000213688343080298
:10479000181803E01068FF23984340181060704712
:1047A00024000040B0B5002200290CD0074B04784B
:1047B00095B22D0A65406C001C5B12026240491ED6
:1047C000401C0029F3D190B2B0BDC04638C10000F2
:1047D00000280AD030B407252C02CD256419604387
:1047E00040091238001FFDD830BC7047F0B583B0C7
:1047F0001F4616460D460146E8680291FBF737FD55
:1048000004460F2E11D8082E04D320462146FBF76C
:10481000D5FC09E0042E02D38120C10501E041202E
:1048200001062046FBF723FD04460999089E2B202C
:10483000C043874205DB20460F462146FBF7BEFCFE
:104840000DE03F20C04387420BDA4920C043874236
:104850000CDBFF200F4681052046FBF708FD39469B
:104860000446688A0880346003B0F0BD019153208B
:10487000C043874206DB20462146FBF79FFC0446E7
:10488000688A10E0A8690299FBF71AFF002801D195
:10489000A88B00E0E88BFBF774FF01462046FBF78E
:1048A000E6FC0446002001990880346003B0F0BDA6
:1048B000F0B581B005460120072D66D80C460029C9
:1048C00063D04A4F38680169C90736D1052630469A
:1048D000FFF7A6FE304604F09DFE03CF03690122D8
:1048E00013430361002918D403200B4683438E48E9
:1048F0001E588807C00EFF278740BE4340278740C9
:10490000374389481F501F20084082408748026073
:1049100087480260354800680FE08A07D20EFF26FC
:1049200096400F230B40083B03218B437D495F5882
:10493000B743402696403E435E506901401801212E
:1049400009024218E369DB069B0CA569ED00EDB294
:10495000EB18536062685207520B23685B075B09D0
:104960009A18A3685B079B0CD218E3685B075B0D82
:10497000D21823695B01DBB2D21863699B07DB0E97
:10498000D218802313434350002001B0F0BDC0462D
:10499000F0B581B0002A23D005460835134C2668AF
:1049A000F668EE40F50702D0022001B0F0BD069D8A
:1049B0008600A619B56040012468201800930123E1
:1049C0001D02461977680724A7437760F1603261BA
:1049D0000099B160415919434151002001B0F0BD27
:1049E00003A00AA174220DA305F04CF970920102F4
:1049F000696E636C7564652F647269766572732F76
:104A00006D6B5F646D612E6300000000646D615F1B
:104A10007472616E7366657200000000496E7661A3
:104A20006C6964207472616E73666572206473745D
:104A30002061646472000000000158490858406811
:104A40007047C046F0B581B005460120012D4CD815
:104A50000C46002949D0002D03D0012D04D10F2090
:104A600000E00E20FFF7DCFDA668012E04D0002E2A
:104A70004FD1E08900284CD1290129484358002012
:104A8000D860F507AD0F27686668B607360F761948
:104A90002569EA07920EB618022F04D0012F03D120
:104AA0000122164300E040361D4F9E60E2681A6006
:104AB00079188D606269CA604968002917D4032299
:104AC0000B469343184A9C588D07ED0EFF26AE40C7
:104AD000B4438026AE4026439E501F220A40012147
:104AE0009140124A1160124A116001B0F0BD8A076C
:104AF000D20EFF2494400F230B40083B03218B432D
:104B000008495D58A543802494402C435C5001B073
:104B1000F0BD08A00FA1492212A305F0B3F8C046CA
:104B2000B89201021CED00E000E400E080E200E049
:104B300000E100E0696E636C7564652F64726976EC
:104B40006572732F6D6B5F6475616C5F74696D6501
:104B5000722E63006475616C5F74696D65725F6F5E
:104B600070656E00636F6E66696720697320696E99
:104B700076616C69640000000001084A1058016009
:104B8000816880220A4382607047C0460001034961
:104B9000085881688022914381607047B892010271
:104BA000F0B58DB0019315460E460A901298002478
:104BB00008900480149F3C80139809900460159815
:104BC00004900480FF2081053046FBF750FB0290E3
:104BD000304603963146FBF7F1FA2B463D460690E8
:104BE000274607950B9311E01180188880002858FC
:104BF000099908600120079D2880052004990880F4
:104C00007F1CBCB21888844200D9A0E02888002804
:104C1000F6D1A0000A9D2E5830460699FBF742FDBA
:104C2000002817D030460399FBF73CFD00280B9B6A
:104C3000079DE5D1089A1780099D2E601888011BF1
:104C4000012934D11080198889000A9A51582960A5
:104C5000059035E0089A1780099806600B9B198823
:104C6000081B0128C0D00C96019825187E1CB0B2F4
:104C70008542BFD389B2B2B28A420ED880000A9967
:104C80000C5820460C99FBF7FFFC0B9B002804D125
:104C900009980460089806800C94761CB0B285428E
:104CA000A8D3198889B2B2B28A42E7D9F5E70C963F
:104CB000019962187D1CA9B216468A4205972CD22A
:104CC000059884B2A5000A9E7259002C104609D09E
:104CD000A819001F016810460C92FBF76FFA0C9A96
:104CE000062C07D80446A81941681046FBF766FA57
:104CF0000C902046079D0299FBF7E2FC00280B9BD5
:104D000007D10C980299FBF7CDFC0B9B002800D033
:104D100076E701202880032070E780B2AAB28242A1
:104D20000FD888000A990C5820460C99FBF7ACFC68
:104D30000B9B002805D1099804600898058005950B
:104D40000C946D1CA9B28E42BAD31888E5E70DB059
:104D5000F0BD0000F0B585B001273904494D686801
:104D600004918843686028684749014329603907EE
:104D7000464801604648039101600024204600F047
:104D8000BDFD4448017849B2002902D480220A437B
:104D9000027068690290A86901903F4803683F4E1D
:104DA0007360C36833603346143B1B68F36033465B
:104DB000103B1B68336133460C3B1B687361334601
:104DC000083B1B68B361331F1B68F3616C62FB0512
:104DD0002C460C3C20689843206078046A68824323
:104DE0006A6030BF6A6802436A60206818432060C6
:104DF0002B4C02980440002901D42648017007205A
:104E00006862002000F08CFD264803990160BFF322
:104E10004F8FBFF36F8F1D48016070681E49086097
:104E20003068C860002C08D08C622046019A10407F
:104E3000086320469043C862CC611B48016889061C
:104E4000FCD50A242046FFF7C3FCF80229688143F9
:104E500029602046FFF7BCFC38032968814329609C
:104E60002046FFF7B5FC2868B84328602846143868
:104E70000068C002FAD5686804990843686005B004
:104E8000F0BDC0462C000040011C000080E200E0A4
:104E900000E100E067000140042000501C010040D8
:104EA000FFFF030080E100E02C0200400A490A688D
:104EB0000A4802400A60FD214900094A1268515C13
:104EC000002908D007490A6C02400A640120000644
:104ED0000A6882430A60704700040040FFFFFF7FBA
:104EE000C89301022000004000207047F0B583B055
:104EF0000D4604467C26464350488719F869396AAE
:104F0000FBF7E8F8A84200D892E00195029401214D
:104F1000EFF31080084002D1EFF3108272B63C46E6
:104F200010343B690025062B0CD80A469A40D3065C
:104F30005B0F06D161231A4275D00D46002803D0BD
:104F400003E00225002800D162B6002D02D02846D9
:104F500003B0F0BD00943C462034384880591021FD
:104F6000C1613E46143604F05FFE05463868C069EC
:104F7000C00605D504F058FE401B31888842F5D99B
:104F80000621029D284600F02FFF20680199414329
:104F9000B869091838688160172179563C4617347A
:104FA000002909D5C16920220A43C2610121F9669D
:104FB000890502680A4302600521284600F014FFB3
:104FC000207840B200250028C1D42B4800687D24F9
:104FD000E100FBF77FF861014143029800F0D6FE43
:104FE00004F022FE04463868C069C00705D004F00A
:104FF0001BFE001B31888842F5D904F015FE0446DB
:105000003868C169890706D504F00EFE001B318897
:105010008842F5D938680121009A116053498161AD
:10502000284603B0F0BD0321216000288CD08CE716
:10503000034804A1084A09A304F024FEE0920102F7
:105040005CCB0000666C6173685F626C6F636B5F62
:1050500065726173650000005D020000626C6F6341
:105060006B20696478206973206F766572207261A5
:105070006E67650D0A000000F8B30102F0B583B059
:1050800002907C214143934A5418E56EEAB2511EC6
:1050900002291FD229040126090E18D00196009278
:1050A000022100F0A1FE2746143704F0BDFD06469C
:1050B0002068C169890606D404F0B6FD801B3988D2
:1050C0008842F5D92068007DC007019E08D030468F
:1050D00003B0F0BD032A36D100922804000E36D06A
:1050E00020466C302D0C00210191016027461437B9
:1050F00004F09AFD06462068C069C00705D004F098
:1051000093FD801B39888842F5D904F08DFD064651
:105110002068C169890706D504F086FD801B39889F
:105120008842F5D9206811498161E9B2012000293E
:1051300011D003290099019E00D006202061226F22
:10514000002A0ED1C3E70026304603B0F0BD012689
:10515000304603B0F0BD0099019E2061226F002A05
:10516000B5D002A89047304603B0F0BD000093EBE5
:1051700070B5002801D0012070BD7825CD4E705D3E
:1051800000280ED000240921204600F02DFE0F201B
:10519000FFF71EFB1520FFF73BFA745534612046DC
:1051A00070BD042070BDC046F0B581B00C460078DB
:1051B000484EF16881422CD1032C54D1706EB16EEF
:1051C000884261D900240621204600F00DFE306897
:1051D000F16D81602046214600F006FE35466035BF
:1051E0002CCDF0683168B48C414F00975B1BA34213
:1051F00000D81C46A3081431FFF7CAFBB06E001993
:10520000B066306E00193066F06D0019F06501B0BF
:10521000F0BDB168814255D1032C45D1F08CF16DC0
:105220000918F165316E09183166B16E0818B0665B
:10523000716E814238D900240621204600F0D4FD49
:105240003068F16D81600121204600F0CDFD316EA6
:10525000B068F38C3268264C009414329B08FFF738
:1052600097FB01B0F0BD30681021C16104F0DCFC97
:1052700005463068C069C00616D504F0D5FC401B51
:10528000B18A8842F5D90FE030681021C16104F07D
:10529000CBFC05463068C069C00605D504F0C4FCE7
:1052A000401BB18A8842F5D90120C10732681368D2
:1052B0008B431360F16E22040A4300021043F06630
:1052C00001B0F0BD4D200201034804A1844B04F05D
:1052D000D9FCC046E09201025CCB0000666C6173B1
:1052E000685F646D615F63616C6C6261636B000039
:1052F000A9510000F0B581B000786E4DAA688242D5
:1053000000D0D0E001263002032942D16A6DAA669E
:10531000AB6DAC6AA418EB652C66AB6C5B1CAB6424
:105320006B6E934235D95E30FFF752FA686CA96C08
:1053300002293AD3814238D1E88C696D0818686532
:105340000020062100F050FD2868E96D81602F6D76
:1053500004F06AFC04462868C069C00705D004F060
:1053600063FC001BA98A8842F5D904F05DFC044661
:105370002A68D069800706D504F056FC001BA98A6C
:105380008842F5D92A687420285C012841D0F104AC
:1053900040E0F2072B681C6894431C60EA6E090425
:1053A00011430143E96601B0F0BD0229FBD38142FC
:1053B000F9D2E88C696D09186965A96D0818A865A6
:1053C0000020062100F010FD2868E96D8160EF8C57
:1053D00004F02AFC04462868C069C00705D004F020
:1053E00023FC001BA98A8842F5D904F01DFC044661
:1053F0002A68D069800706D504F016FC001BA98A2C
:105400008842F5D92A687420285C012822D0F1044A
:1054100021E03105334B3B405918012802D01920B7
:10542000400601E00720C00608182F4940185060C8
:10543000002F0DD004F0F8FB04462A68D0698007DD
:1054400006D404F0F1FB001BA98A8842F5D92A682A
:105450002B6D1FE03105234B3B40C918012802D0BA
:105460001920400601E00720C00608181E49401810
:105470005060002F0DD004F0D7FB04462A68D06995
:10548000800706D404F0D0FB001BA98A8842F5D916
:105490002A68EB8C296EA868144C00941432FFF72C
:1054A00077FA01B0F0BD044804A10C4A0C4B04F09B
:1054B000E9FBC046E09201025CCB0000666C6173C0
:1054C000685F646D615F77726974655F6E6279743D
:1054D00065735F63616C6C6261636B0072040000F2
:1054E00043CB0000FF3F000000808000F552000029
:1054F000F0B587B004460126880E14D01546002A60
:1055000011D00F468120C004401B88420BD37C2061
:105510006043F04908180590818C38460691FAF7E7
:10552000D9FD002902D0304607B0F0BD28460699C3
:10553000FAF7D0FD0029F6D1059880693E1A304669
:105540000699FAF7C7FD0746039670190190069E63
:105550003146FAF7BFFD0546C01B04900598006A66
:1055600002903146FAF7B6FD049981420FD2002627
:10557000BD42D8D92046394600F03CFB2046FFF713
:105580007DFD0028FAD17F1CAF42F3D3CBE700901A
:105590000398029D2946FAF79DFD0646284670436A
:1055A0000399081A019800D0761C2946009D75437E
:1055B000FAF790FD0590029941430198401A039033
:1055C0000699FAF787FD0490AF420BD22046394680
:1055D00000F010FB2046FFF751FD0028FAD17F1C98
:1055E000AF42F3D305988642069D009F0CD2204619
:1055F0003146FFF77BFC2046FFF740FD0028FAD13B
:10560000761C05988642F2D30398A84203D200265E
:10561000304607B0F0BD059847430025E9192046FC
:1056200000F0E8FA2046FFF729FD0028FAD16D1CAA
:10563000002604988542F1D375E7C046F0B585B0E1
:10564000002803D00124204605B0F0BD7822A14FE8
:10565000B85C002803D00024204605B0F0BD0492B9
:10566000002905D0384614300CC90CC01CC91CC018
:105670000020F86615242046FEF7D2FF204603F0EE
:10568000C9FF38681021C16104F0CEFA04463868B9
:10569000C169C90607D504F0C7FA001BB98A884258
:1056A000F5D9386800E0B98ABA7D1207120B521892
:1056B000F97DCB07DB08D2188B07DB0F5B05D2180F
:1056C000CB06DB0FDB05D2184B07DB0FDB06D2184E
:1056D0008B06DB0F5B07D2180907C90F8907114337
:1056E000016000240A21204600F07EFB3220FFF7F3
:1056F0006FF80821204600F077FB04F095FA054684
:105700003868C169890606D404F08EFA401BB98A4C
:105710008842F5D93868017D0A46C23A534253415E
:1057200074257B550904027D12025118007D0B1867
:105730000220032668A2314605F002FB785D0128AD
:10574000039619D1F87D029000260621304600F01C
:105750004BFB0721304600F047FB012102988143B3
:10576000785D012847D13868890101750675752172
:10577000795C012938D048E00020032100F034FB97
:1057800004F052FA06463868C169890606D404F066
:105790004BFA801BB98A8842F5D93868007D4608E3
:1057A0000122F87D014631431640C90701D030403F
:1057B00036D00295002506212846019200F014FB00
:1057C00007210095284600F00FFB019846400298FB
:1057D000385C012813D13868B10101750099017551
:1057E0007521795C012910D114307621795C4A4207
:1057F0004A41510008E038680675490003E03868FE
:1058000000990175710014300170374800687D21DE
:10581000C900FAF75FFC28214143002000F0B6FAE6
:105820007720385C012803D102200021FEF788FF91
:1058300004F0FAF906463868C069C00705D004F0DC
:10584000F3F9801BB98A8842F5D904F0EDF90646D0
:105850003868C169890706D504F0E6F9801BB98A62
:105860008842F5D93868E249816117203856002806
:1058700029D57868002816D40146039A91431C4A1A
:105880008B588507ED0EFF26AE40B3438026AE4011
:105890001E438E501F210140012088401549086099
:1058A000154908600FE08107C90EFF228A400F23C7
:1058B0000340083B039883430C481D5895438022BE
:1058C0008A402A431A5001200499785438612046AE
:1058D00005B0F0BDE09201026A656465635F6964CA
:1058E0002025780D0A000000F8B301021CED00E04D
:1058F00000E400E080E200E000E100E080B57C210F
:105900004143A64842187823D25C002A05D040586B
:10591000024941600F20FEF75BFF80BD008020B987
:1059200080B57C2141439D4842187823D25C002AEF
:1059300005D04058024941601E20FEF749FF80BD56
:10594000008020ABF0B593B07C270A904743934882
:10595000C619980704D0F07D4024044000D017E118
:105960000125880E2ED0002B2CD08120C004C01A17
:10597000884227D309920122EFF31084144002D108
:10598000EFF3108072B63046103005903069002574
:1059900006280891069310D8079414468440E1061F
:1059A000490F04D161210C4203D0154604E00225C1
:1059B00002E00221059B1960079C002C00D162B611
:1059C000002D02D0284613B0F0BD3446173473487A
:1059D000C05910210491C1613746143704F024F9ED
:1059E00005463068C069C00605D504F01DF9401BA6
:1059F00039888842F5D92078400665D40297B78C5B
:105A0000069C20463946FAF765FB07903946414324
:105A1000601A039035462435A74200D894E00398D5
:105A200000281CD006210A9C204600F0DDF92888B9
:105A30000799484308994018316888600027204634
:105A4000039C394600F0D0F9079B099A28885843EF
:105A5000C0193168097D11547F1CA742F6D3306804
:105A60000499C16104F0E0F80446029D3068C06901
:105A7000C00605D504F0D8F8001B29888842F5D95E
:105A800004F0D2F804463068C069C00705D004F0BD
:105A9000CBF8001B29888842F5D904F0C5F80446E4
:105AA0003068C169890706D504F0BEF8001B298853
:105AB0008842F5D930680121059A1160B2498161A7
:105AC0000025284613B0F0BD03200025089FF76588
:105AD0000999316606997166B566F0660120C007BE
:105AE00031680A6802430A6006210A9C204600F0D9
:105AF0007BF9306887602046294600F075F93A4FF7
:105B00000BAA0A921BCF1BC21BCF1BC2B48CF0681E
:105B10000A99FEF7CDFEF0683168344A0092069A81
:105B2000944200D31446A3081431099AFEF730FFBB
:105B3000B06E0019B066306E00193066F06D001955
:105B4000F065284613B0F0BD002404E0641C0798FB
:105B5000844200D363E706210A9800F045F92888BB
:105B60006043089940183168886000270A983946D0
:105B700000F03AF928880028099AE7D06043101805
:105B80003168097DC1557F1C28888742F6D3DDE73F
:105B9000034804A1064A07A304F074F8E092010246
:105BA0005CCB0000666C6173685F726561640000C5
:105BB000C603000054686520444D4120726561644D
:105BC000206C656E6774682073686F756C64206202
:105BD0006520746865206D756C7469706C65206FE4
:105BE0006620340D0A000000B8C30000A95100006F
:105BF000000093EBF0B583B00D4604467C26464387
:105C000051488719F869B98CFAF764FAA84200D8A4
:105C100094E0019502940121EFF31080084002D135
:105C2000EFF3108272B63C4610343B690025062B18
:105C30000CD80A469A40D3065B0F06D161231A425C
:105C400077D00D46002803D003E00225002800D1BC
:105C500062B6002D02D0284603B0F0BD00943C4649
:105C60002434394880591021C1613E46143603F06E
:105C7000DBFF05463868C069C00605D503F0D4FFD0
:105C8000401B31888842F5D90621029D284600F044
:105C9000ABF8208801994143B869091838688160D8
:105CA000172179563C461734002909D5C1692022AD
:105CB0000A43C2610121F966890502680A4302604C
:105CC0000421284600F090F8207840B22C460025A8
:105CD0000028C0D42B4800687D21C900FAF7FAF9E2
:105CE00020492D314143204600F050F803F09CFF3D
:105CF00004463868C069C00705D003F095FF001B53
:105D000031888842F5D903F08FFF04463868C169AD
:105D1000890706D503F088FF001B31888842F5D932
:105D200038680121009A116017498161284603B043
:105D3000F0BD0321216000288AD08AE7034804A12E
:105D4000084A09A303F09EFFE09201025CCB000029
:105D5000666C6173685F736563746F725F657261AF
:105D6000736500002B020000736563746F72206915
:105D70006478206973206F7665722072616E676542
:105D80000D0A0000F8B30102000093EBF0B583B0F8
:105D900001917C220290424353498C1825461435C8
:105DA00003F042FF06460221029800F01DF803F0BE
:105DB0003BFF07462068C169890606D403F034FF1B
:105DC000C01B29888842F5D92068007DC00708D00B
:105DD0006420FEF7FDFC03F027FF801B0199884239
:105DE000E1D903B0F0BDC046F0B585B004910446DA
:105DF0007C2060433C490F183D46143503F014FFE6
:105E000006463868C069C00705D003F00DFF801B47
:105E100029888842F5D903F007FF06463868C0692B
:105E2000800705D503F000FF801B29888842F5D93B
:105E30001421049B5943DC2060432C4A1018039022
:105E400002914018018A8268C47C7426BE5D012ECE
:105E50000DD10191012B02990CD0012B0DD075268B
:105E6000BE5D012E0ED0019E072B0ED10EE00E4618
:105E700002990BE00222012BF1D138247526BE5D78
:105E8000012EF0D10326072B00D0019E184B334082
:105E900024069207D20A1219D218039B5958C9072F
:105EA000490C52184168CB071B0CD218837C5B0746
:105EB0005B0BD218C0684007000A10183A6850609F
:105EC000002E0ED001290CD103F0AEFE0446386836
:105ED000C069800705D403F0A7FE001B298888420B
:105EE000F5D905B0F0BDC046E092010200C5000042
:105EF000FF3F0000F0B59DB00D460126890E2FD062
:105F0000002B2DD011928121C9041093C91AA942E6
:105F100026D30121EFF310840C4002D1EFF310825D
:105F200072B67C220F904243E74814928718384695
:105F300010303B690026062B0DD80A469A40D3063E
:105F40005B0F07D161231A4200D16FE30E46002C8C
:105F500003D003E00226002C00D162B6002E02D04E
:105F600030461DB0F0BD0290BD65002113917965EA
:105F70001098401E12904019B964B9690D916E1ABB
:105F80001199B962FD6238637E63F98C0E913046D7
:105F9000FAF7A0F80446B863129830180E9E3146FE
:105FA000FAF798F8109B011B4A1CF86339647A646D
:105FB000139A0029194608D0704359190D9BC91A24
:105FC0000A1A7443581B80190119384648300E903C
:105FD000384644300D90384640300B9038462630D5
:105FE0000590384658301390384654301290F96472
:105FF0003A651498B44908581021C16138461430E4
:1060000014903846503004903D464C3503F00CFE59
:1060100004463868C069C00606D503F005FE001BBB
:10602000149909888842F4D9F87D40060C9500D56A
:1060300074E201230E9803600D98016800290F98FF
:1060400000D1CDE23A4674320A92DA0407921A0578
:1060500009921922520606920722D206089216E0E9
:106060009A4800687D21C900FAF734F81099414335
:106070000F9C2046FFF78AFE20460C9D0E9A116861
:106080004B1C13600D9909688B4200D9A8E20B9A4A
:106090001268012A55D0002A00D0A8E02E68129973
:1060A0000C6813990D6806211091FFF79DFE386862
:1060B00085601198051903F0B7FD04463868C0697A
:1060C000C00706D003F0B0FD001B14990988884270
:1060D000F4D903F0A9FD04463868C169890707D5DA
:1060E00003F0A2FD001B149909888842F4D938688E
:1060F0000A990A78012A089900D00699012A099A72
:1061000000D0079A3346724C234013430B43714926
:106110000B434360002EA3D003F086FD044638688D
:10612000C069800706D403F07FFD001B149909881D
:106130008842F4D93868297801756D1C761EFAD129
:106140008EE7012B00D0C7E02E6812990C681399D6
:106150000D6806211091FFF747FE38688560119899
:10616000051903F061FD04463868C069C00706D010
:1061700003F05AFD001B149909888842F4D903F0F2
:1061800053FD04463868C169890707D503F04CFD03
:10619000001B149909888842F4D938680A990A784A
:1061A000012A089900D00699012A099A00D0079A75
:1061B0003346474C234013430B4346490B4343604C
:1061C000002E69D003F030FD04463868C0698007AE
:1061D00006D403F029FD001B149909888842F4D9DC
:1061E0003868297801756D1C761EFAD154E0012BB0
:1061F00000D0C9E02E6812990C6813990D68062129
:106200001091FFF7F1FD386885601198051903F0CA
:106210000BFD04463868C069C00706D003F004FDD2
:10622000001B149909888842F4D903F0FDFC044648
:106230003868C169890707D503F0F6FC001B14997B
:1062400009888842F4D938680A990A78012A089995
:1062500000D00699012A099A00D0079A33461C4CAF
:10626000234013430B431B490B434360002E13D0C1
:1062700003F0DAFC04463868C069800706D403F0EE
:10628000D3FC001B149909888842F4D9386829780E
:1062900001756D1C761EFAD10C4800687D21C9007D
:1062A000F9F718FF109941430F9C2046FFF76EFD48
:1062B00020460C9D2A68139B196889181960129B47
:1062C000196889181960D9E6E0920102F8B3010251
:1062D000FF3F0000008080008B4200D0CEE6049992
:1062E0000E6812990C6813990D6806211091FFF73A
:1062F0007BFD386885601198051903F095FC04460C
:106300003868C069C00706D003F08EFC001B1499E2
:1063100009888842F4D903F087FC04463868C169CB
:10632000890707D503F080FC001B1499098888426F
:10633000F4D938680A990A78012A089900D0069990
:10634000012A099A00D0079A3346D44C23401343BC
:106350000B43D3490B434360002E00D180E603F08A
:1063600063FC04463868C069800706D403F05CFC0F
:10637000001B149909888842F4D938682978017576
:106380006D1C761EFAD16BE6129A1268119CA61843
:10639000139A15688B425FD104990C68062103910A
:1063A000FFF722FD3868856003F03EFC054638683B
:1063B000C069C00706D003F037FC401B1499098858
:1063C0008842F4D903F030FC10900C9D3868C16904
:1063D000890708D503F028FC1099401A14990988F8
:1063E0008842F3D938680A990A78012A089900D0B6
:1063F00006991091012A099A00D0079A2346A749C5
:106400000B40134310990B43A5490B434360002CE9
:1064100014D003F009FC10903868C069800707D4D5
:1064200003F002FC1099401A149909888842F3D9A4
:10643000386831780175761C641EFAD19A48006874
:106440007D21C900F9F746FE039941430F9C204680
:10645000FFF79CFC204611E605990C880621039164
:10646000FFF7C2FC3868856003F0DEFB054638683C
:10647000C069C00706D003F0D7FB401B14990988F8
:106480008842F4D903F0D0FB10900C9D3868C169A4
:10649000890708D503F0C8FB1099401A1499098898
:1064A0008842F3D938680A990A78012A089900D0F5
:1064B00006991091012A099A00D0079A2346774934
:1064C0000B40134310990B4375490B434360002C59
:1064D00014D003F0A9FB10903868C069800707D476
:1064E00003F0A2FB1099401A149909888842F3D945
:1064F000386831780175761C641EFAD16A480068E4
:106500007D21C900F9F7E6FD039941430F9C204620
:10651000FFF73CFC204605990A88CCE65E4815A9A1
:106520000A4678C878C278C878C20125E8073A6870
:10653000136803431360B868FEF7BAF90220002617
:10654000139C2168BA6AF9653A6610997966BE6645
:10655000F8660C980068129A1168091811600E9B71
:1065600019684A1C1A60226810182060002900D09F
:10657000F6E410953846603013903C465C3438465B
:106580000830129006210F98FFF72EFC386821681A
:1065900081600C980068119003F046FB044638684F
:1065A000C069C00706D003F03FFB001B149909889F
:1065B0008842F4D903F038FB0446109D3A68D0694C
:1065C000800707D503F030FB001B14990988884227
:1065D000F4D93A687420385C01282DD0E9042CE005
:1065E00003F022FB04463868C069C00706D003F0F8
:1065F0001BFB001B149909888842F4D903F014FB93
:1066000004463868C169890707D503F00DFB001BF4
:10661000149909888842F4D938680121029A1160D6
:1066200022498161002630461DB0F0BD0421016081
:10663000002C00D191E491E42905119C174B2340D3
:10664000591801280C9D02D01920400601E00720AE
:10665000C0060818124940185060002C0ED003F0F4
:10666000E3FA04463A68D069800707D403F0DCFAFD
:10667000001B149909888842F4D93A682B6813984A
:10668000016812980068074C00941432FEF780F9F4
:1066900030461DB0F0BDC04678C30000FF3F00008B
:1066A00000808000F5520000F8B30102000093EB77
:1066B0003120C000014909680858704770920102F2
:1066C000F0B5032920D8C0467944097949008F44A0
:1066D00001080F15012181403D4B1B685963D962A8
:1066E00012E0012181403A4B1B681963D9620BE02B
:1066F00001218140364B1B68596304E00121814030
:10670000334B1B681963996283003149CB18DA60F7
:106710008A68002A29D14A68002A16D4032314461D
:106720009C43174BE5589607F60EFF27B740BD432D
:106730008027B7402F43E7501F23134001229A4080
:10674000104B1A60104B1A600FE09307DB0EFF2509
:106750009D400F241440083C03229443074AA65846
:10676000AE4380259D403543A550012282400868F4
:106770000262886810438860F0BDC0461CED00E0EE
:1067800000E400E080E200E000E100E010B5012458
:106790002046FDF745FF204602F03CFF002010BDDB
:1067A000012181400A48006842688A43426070477C
:1067B000074909680968C140012008407047C04680
:1067C000012181400248006842680A4342607047E4
:1067D0006093010210B505480468054800686043ED
:1067E0000449F9F78DFC201A10BDC0467400004022
:1067F00074A8010240420F00124A072809D88000FD
:106800000F2383408140194010689843084310606B
:1068100070470F280AD8800020380F23834081401A
:1068200019405068984308435060704780004038D2
:106830000F2383408140194090689843084390603B
:106840007047C04634000040F0B54307DC0E072611
:10685000A640C3089D000E4BEF187D68B5433E1D52
:10686000002908D035600122824001290CD1186826
:1068700010431860F0BD01218140186888431860FA
:10688000A24015433560F0BD186890431860F0BD14
:106890000C01004010B582B014460A460146049827
:1068A000009301900820234600F092F802B010BD3A
:1068B000B0B584B014460A460146089802250095F2
:1068C000019302900720234600F052F904B0B0BDB6
:1068D00070B500285BD031490A783149002A03D1CC
:1068E0004A68012313434B60428803881B049A18AB
:1068F0000B46183B1A60828883891B049B180C4640
:106900000C3C23600B46083B84681C6044690323ED
:106910002340057CAD00EB188569AD072D0D5B1993
:10692000457C2D035B19C569AE07B60A9B19867CA9
:10693000B6059B190E1F3360036A122B04D107247E
:106940000C60541EA2410AE0032C05D1012D03D88E
:1069500007220A60012202E006220A600122114C8D
:10696000002525700F2464012034C57C6D0225406C
:106970001B069B0BD218C3791B07DB0ED21880793C
:106980000007C00D101840191439086070BD064882
:1069900006A1862209A303F075F9C046DCA6010210
:1069A00018100050DEA601023ACE00006C73705F32
:1069B000656E67696E655F72756E00005061726129
:1069C0006D65746572206973206E756C6C000000D3
:1069D000F0B58BB0109E34043ED00D46D64C21400D
:1069E000012701977F06B9423CD111462140B942A7
:1069F0003FD11C40BC4243D1119902AC0027E78132
:106A0000E780668027802782A774E1749908A181B6
:106A1000A908A1800A90099708970797900880B263
:106A200004902046FFF754FFAA480078002801D0C0
:106A30000BB0F0BDAB480168C90708D10168C907B0
:106A400005D10168C90702D10168C907F3D07F48A1
:106A5000019901700BB0F0BDB8480D49AF22C14B90
:106A600003F010F90095B5480949B022754B03F0C1
:106A700009F90092B1480649B122724B03F002F9BC
:106A80000093AE480249B2226E4B03F0FBF8C046B9
:106A900010CE0000F0B58DB00392139E340446D0A2
:106AA0000A46A54C2140012502956F06B94244D102
:106AB00003992140B94247D11C40BC424CD11499A2
:106AC000129D04ACE174294921820027E781E78007
:106AD000668027809908A1819108A1800B95012DDE
:106AE00001D16121CF43A7740C9002200A90099034
:106AF0000398800880B206902046FFF7E9FE7548AB
:106B00000078002801D00DB0F0BD76480168C907B3
:106B100008D10168C90705D10168C90702D1016818
:106B2000C907F3D04948029901700DB0F0BD834800
:106B30000D49FB228B4B03F0A5F800927F480A49D0
:106B4000FC22404B03F09EF8039800907B480649D6
:106B5000FD223C4B03F096F8009378480249FE2250
:106B6000384B03F08FF8C0461DCE00008E8E00001B
:106B7000F0B58BB0119E340447D00D466E4C2140C9
:106B8000012701977F06B94245D111462140B942FC
:106B900048D11C40BC424CD11299109F02ACE17408
:106BA000294921820021E181E180668021809908C4
:106BB000A181A908A1800997012F01D0712100E0CE
:106BC0006121C943A1740A9003200890079090089E
:106BD00080B204902046FFF77BFE3E4800780028F4
:106BE00001D00BB0F0BD3F480168C90708D101686A
:106BF000C90705D10168C90702D10168C907F3D0E7
:106C00001248019901700BB0F0BD4C480C49D522D7
:106C1000544B03F037F8009548480949D622094BF0
:106C200003F030F8009245480549D722054B03F0A0
:106C300029F8009341480249D822024B03F022F878
:106C40002CCE00005ACE000086860000DEA601028F
:106C500010B582B014460A46014600200093019008
:106C600004202346FFF7B4FE02B010BD10B584B077
:106C700014460A4601460020009001930290042029
:106C80002346FFF707FF04B010BD000070B50D46A6
:106C9000064604242046FDF7C3FC204602F0BAFC59
:106CA0000B4805600B480670002E0ED00A4801689C
:106CB00080220A437F218A430260012000030749A2
:106CC00008600749086007480460002070BDC0469E
:106CD000E0A60102DCA601020CE400E080E200E094
:106CE00000E100E01C100050B0B582B0144602462E
:106CF0001148204001256D06A8420DD1180413D07B
:106D00001748016000200093019006201146234699
:106D1000FFF75EFE02B0B0BD0094FF228C32074840
:106D2000074908A302F0AEFFFF208C30421C034845
:106D300003490C4B02F0A6FF0300FCFF3ACE000013
:106D400002CE000044737420616464726573732022
:106D5000257820697320696E76616C696400000093
:106D60000810005078CE000080B582B00B46014676
:106D700000200092019003200A46FFF729FE02B08E
:106D800080BD0000002801D0042100E00221C34A98
:106D90005172411E8841800103490A6840239A4389
:106DA000101808607047C04650A00050F0B583B07E
:106DB00002912E49CD7A0E7B771987424FD90899D7
:106DC0000191182545434126F604BF00BE19745BA6
:106DD00034490C4057033C199B07D90C6418324BBB
:106DE0001B681B7A745375196C880326B6032640FA
:106DF0009B079B0C9B193F2404401819029CA30677
:106E00001B0DC0186880012A184E13D8707B1422FD
:106E10004243307B5023434324011B199A18F37AD1
:106E2000C0181C234343D01880081E4A1040074353
:106E30000F432F800198686001F0C4FEA860E868E5
:106E40001A4908403030E860286908402721715C01
:106E50004018286100F016FE686103B0F0BDFF2203
:106E60008832034803A108A302F00CFFE8A6010240
:106E7000C9CE00006D61635F63735F636F6E73748F
:106E80007275637400000000435320696E64657876
:106E9000206973206F7665722072616E67650D0AD6
:106EA00000000000FF070000C89301020000F0FF8F
:106EB000F0B581B0009314460D46074606263046CD
:106EC000FDF7AEFB304602F0A5FB26211D484754D6
:106ED0000021017041708171017181704171C17037
:106EE000C17102224272C162016341638163047312
:106EF0004273C572009A561C134A168001724120D3
:106F0000C00401214903F9F74EF9502060432901DB
:106F1000081861198A00801818224A438018B2B2F2
:106F20004A438018094940180949884204D200F0B0
:106F3000B7F8002001B0F0BD064807A19A2209A3C6
:106F400002F0A0FEE8A60102E4A601022800080261
:106F500001200802C9CE00006D61635F696E69742B
:106F600000000000454D206F766572666C6F770DEE
:106F70000A000000BC48C179002901D001207047F7
:106F8000007A411E88417047F0B583B002912A49CA
:106F90004B7B834248D9CB7A0C7BE31818245C43A3
:106FA0009B00E3184124E4041A19142401900546B7
:106FB00065430026565100925519EE882E4F0B4618
:106FC0007A1C32402D4E3688497A711A2C4E0E406A
:106FD000B618EE803740997BEF80AA88294F17407A
:106FE0004A424A4191007918274A8918A980274FB7
:106FF0000F402D1D029801280AD125490E40092174
:10700000C902711869800121C9037918298000E03B
:107010002F800198444300980019074A918C4182BF
:10702000118C018203B0F0BD3520C200034804A1D9
:1070300009A302F027FEC046E8A60102C9CE00005F
:107040006D61635F6C696E6B5F646573635F636FD3
:107050006E737472756374004C696E6B2064657333
:107060006320696E646578206973206F766572208D
:1070700072616E67650D0A00FFFBFFFFE4A6010267
:10708000FF03000003D0FFFFE80F0000EF1F000028
:10709000FF830000D54A506391637047E8A6010260
:1070A000F0B581B04348CC21016003214160CF4954
:1070B0000A7BD304404C1B19CC7AA218541E1C43E3
:1070C0001823534392009A184B7B14255D435219A1
:1070D000920122430124630613434361002282622A
:1070E000C262026342638263C26342650267334BDA
:1070F0001A605A609A60324B1A601A619A61DC61B8
:10710000304C1C62304C251D1D6325460C3D5D63D3
:107110002546283D9D632D4EDE631C645C642C4D2A
:107120002F461C379F642746143FDF64103C1C65C4
:10713000284C5C65284C9C650C369E67274CA563E3
:107140004035E563DA651A665A669A66DA661A6742
:10715000234DDD6702258561224DC561C325AD0341
:10716000CD620A63D2435A601F4A1368FF25AB43BE
:1071700026254D5DAD072D0EEB1813601B4A10231D
:1071800013601B4A1360272260238B5419498160C6
:10719000C160016121607D210901016641661649D6
:1071A000C164164941641649016400F05BFC01B0FA
:1071B000F0BDC04604A000500000F8FF94A00050AD
:1071C00034A10050FF185A00300400400410004061
:1071D0001C2000405430004060400040B8A10050E6
:1071E00014001400FF3F3FFF04E400E080E200E0F1
:1071F00000E100E0DC05DC053F0270020133D0074E
:10720000D007D00770B5182002F004FA192002F058
:1072100001FA0624204602F0FDF92046FDF700FAA7
:10722000D54C002525706570A5712571A570657117
:10723000E570607B14214143207B50224243E37A76
:107240001E0192195118C0181C224243891841206E
:10725000C004F8F7A8FFE5712572FFF721FF70BDA4
:107260002921C54A50547047E8A60102F0B58BB0F9
:10727000079208910146C04FB8780991FFF784FE44
:1072800078793A7B79790691824200D89FE0FB7A3F
:107290009A181823534392004124E1040491521890
:1072A000D2187B7B14214B43D218502460431558CD
:1072B00001230A93DB022E469E4316504E4B2B4071
:1072C00005937D7B03914D433E7B7443F97A0B011B
:1072D0001B195B1971181C24029461435918A74BA0
:1072E0001B88069C5C430919C904490D059BC918F4
:1072F000115010180799416038787979089A0092EE
:107300000322099BFFF752FDF87A397B0918387878
:10731000814263D983000993049AD45C0894F721CD
:107320002140D154D1184D788E7836027619CB7819
:107330001B04F31807900A9886051E43330CCB7084
:10734000FB7A387BBC784D709E4D3540039E66437A
:10735000C018029B4343981940029B4B03405C19A1
:10736000200A8870200CC870F023089D2B401B1D3C
:107370003D7B0895FE7A099D5355C8700620079AF3
:1073800050438019089A801848701F22D202224068
:107390000243100A88707879401C7871387B7979BB
:1073A000814201D3002179713978491C3970F97A09
:1073B00008183978884201D80020387028200A99A6
:1073C0003954387A401C3872387A0BB0F0BDA72097
:1073D0004200D1480649074B02F054FCA720420066
:1073E0007A32CD487249734B02F04CFCE8A6010298
:1073F000E9CE000092CE000000F0FFFF032000065F
:1074000005490A6882430A600A6802430A60034821
:10741000012101607047C0461C0000401CA00050C4
:1074200080B50120FDF7B2FB80BD0000F0B587B04C
:1074300006930646504C607A504B1B88181A0C9DD8
:10744000A84200DC89E00F460592012E06D156487D
:107450000021C1620169554A89180160A07831464E
:10746000FFF792FDE078E178069A2B4600F0AEF83F
:107470002078E1780097002206923346FFF796FCC9
:10748000E07A217B0818217888426ED94120C20415
:1074900004918800815C0391F7250D400292855488
:1074A0004549455C4549465C360276194449475C86
:1074B0003F04F6190127BF0537433E0C4654E67AD0
:1074C000217BA3783C4A85543E4D3D4014275F43C1
:1074D00089191C234B43D91949023B4B0B405D19B9
:1074E000290A364BC1542E0C35494654F0270399CE
:1074F0000F400599002900D13F1D217BE37A029AB4
:1075000087542F4A86540622049E7243D21851187B
:10751000294A81541F22D20215400D43290A274AC5
:107520008154E078401CE070E07AE178814201D338
:107530000699E1702178491C2170217B0818217877
:10754000884201D806982070E079401CE071A07A4A
:10755000401CA072E07907B0F0BD3920C20016329D
:10756000074808A109A302F08DFB3920C200044896
:107570000F49104B02F086FBE8A60102E4A60102C7
:10758000C9CE00006D61635F747800004D414320F7
:107590005458206C656E206973206F766572207276
:1075A000616E67650D0A00000804004090D003007A
:1075B000FFCE0000B0CE0000010008020200080269
:1075C00003000802FF07C0FF00F83F00F0B589B0D4
:1075D0000893019204914F4DEF7A874200D891E0D1
:1075E000297B502632464A434124E3040693D218AD
:1075F000CC19A10051181822059254430A19697B2D
:107600001423079359435318029000011958044654
:107610000390504A0A40A97AC90251180898820575
:10762000D2088A181A514C4911402A7B00965643B9
:10763000384CE57A2C0106982418A719354E5419B0
:10764000A5007D19059844432819747B079D6C4358
:107650000519049FD2194148048854432A19089CEB
:10766000D204520D51181D460398195000F014FA17
:107670000146707A001902043E460CD080B2C00068
:10768000002900D1801E029FA5214900F8F722FDA4
:107690001F21014001E00021029F38012818427992
:1076A00083791B029A18C3791B04D2182C4B134000
:1076B000437109045918090CC171002C20D01548D8
:1076C00035460646007B009B4343F17A0A01069F3C
:1076D0003A43D21841188B00D218059B4B43D1185E
:1076E000727B079B5343C91840191C4A12884243B6
:1076F00088180199884203D001992246F8F73AFD8B
:1077000009B0F0BDFF225C32034804A109A302F0D6
:10771000B9FAC046E8A60102C9CE00006D61635FF8
:1077200074785F646573635F636F6E73747275639F
:10773000740000005458204445534320696E64652A
:1077400078206973206F7665722072616E67650DAF
:107750000A000000FF0700E000F8FFFFE4A60102B6
:10776000EFFFE0000168044A1160416851608168E0
:107770009160C068D060704780A0005082B0FCF774
:1077800007FD052000252946FFF736F80620294683
:10779000FFF732F80A202946FFF72EF8092029467C
:1077A000FFF72AF80124204603F0F2FB284603F0F5
:1077B000EFFBFCF74FFD2846FCF71CFD01F0AAFE8D
:1077C00001F0A2FE47480168474800688903019418
:1077D00008D40321090708402107884202D0FCF79A
:1077E000A5FC06E0FCF77EFAFCF7B8FC0020FDF7EC
:1077F000BFFCFCF777FD0025284604F0EBFBFEF705
:10780000C5FF3A483A49016000F09AF8754FB888C8
:10781000384C2080FF2002307880B87A36490870D2
:107820007D20C000F988F8F755FC344E307023688D
:107830000324334A2046214603F082FA7888C1B2F5
:107840000091030A2F4A2046214603F079FA2E4977
:1078500064222E4B284603F099FE01F039FC2C4A95
:10786000019C2046214602F0C5F8A00302F0F2F880
:10787000284F09E00024204601F0DAFB642220466C
:107880002149224B03F082FE7878002802D07D70D7
:10789000FBF7CCFEFCF790F80B20FEF789FF397858
:1078A000002804D0002905D10198387002E0012990
:1078B00000D13D7070780028E6D002F03DFEEFF375
:1078C0001080C007D6D1EFF3108072B60024204696
:1078D00001F0AEFB642220460B490C4B03F056FE30
:1078E00062B6D1E71800004030000140D095010297
:1078F000153B0000CC960102A19601029697010269
:10790000F3CD0000D6CD0000D4950102C1B7000030
:10791000CD99000014900102014800687047C046EC
:107920000C00004081B080B581B0039303AB00939D
:1079300002F07EFE01B080BC02BC01B0084700002E
:10794000F0B581B0002630463146FDF777FE0125BF
:10795000AC022349234F30463A462346FDF7F2FF57
:1079600039882148814238D064217E5262217E527A
:1079700060217E5244217E5250217E52FD87BD8778
:1079800078217987022139874321F986BE83FD81D9
:107990001649B9817E810A2139811549B98038801B
:1079A000FE831420B8827D208000F880EFF31080E1
:1079B00072B630463146FDF741FE00280CD12A034D
:1079C00000263046064D2946FDF792FD054A304611
:1079D00029462346FEF78EFA62B601B0F0BDC046D6
:1079E00000E002047EA20102AA550000E1FF0000AF
:1079F000341200000020704710B50024002809D080
:107A0000002905D003464A0003481946F8F7B2FB9F
:107A1000204610BDE04310BDD8920102014600206F
:107A20000A2901DAC0437047014A11807047C046F5
:107A30005C9301020020704780B50188064A1180DE
:107A40008178064A1170C178054A11700079FCF7F7
:107A50003BFB002080BDC046B4930102B6930102F7
:107A600098A70102044805490160152109044160F5
:107A7000034981607047C0469C30004041000800C7
:107A8000340007000748006840697047FD20400047
:107A900004490968085C7047024800686221405C3C
:107AA0007047C046C893010210B5064804680648EE
:107AB00000686421F8F724FB0221C94341430819F7
:107AC00010BDC0469CA70102A0A701020A491A22C4
:107AD0000A600A4948704878FF210902084A136879
:107AE0008B43800380B2C0181060064820210160DB
:107AF000054801600020704770200040B8930102E3
:107B000004E400E080E200E000E100E0F0B5A9B0AC
:107B100016460F460546C648002B024600D01A46B8
:107B20003921CC003D21C90051181191824218928F
:107B300006D001204202BE491898F8F71BFB189A9C
:107B40006120111913910E21119C0A91A170002F2F
:107B50000D9501D00A2100E00921592317938300D4
:107B6000E170784278411399087030781090107065
:107B7000F17AE17471785170B7789770F178D170BB
:107B80003579157174795471B1799171F179D17137
:107B9000317A1172717A5172B17A91727E1EF0B29D
:107BA00000210328169106D870B28000A1A21058B7
:107BB0006A00805A1690179882001898C01814907E
:107BC000F81E022804D3012E084604D89D4800E080
:107BD0009D48031918781290189DA81817902846E8
:107BE000303015902C4656346D2080002950974A2D
:107BF000974B149E33627262B362F2623176F18205
:107C0000139B597009229A70281841608160C160E5
:107C10000161109880008F490858F8F76BFE012F1A
:107C200010900F9104D0022F05D17F217E2004E017
:107C30007C217B2001E05B215A20159DA9842070C6
:107C400003200C90A080012666701F200B90A88254
:107C50001820A8740A46083A179BDA76169B129ADF
:107C6000D2184A439100189A9163B702791E8B4249
:107C70000E9109D97848608034206884774828823A
:107C800077481399088339E07F2B10DD802B18D0BB
:107C900031028B421BD071028B4227D16E49618029
:107CA00068846F4813990883CF20C00025E0202BFB
:107CB00017D0402B1AD16848608004206884694836
:107CC0001BE06548608006206884674815E06248CC
:107CD000608010206884624813990883C520C00022
:107CE0000BE0624860800220688404E0042068841D
:107CF000812040006080FF2002302882104600F082
:107D000005FF1298102806D0402808D108201499A1
:107D1000C876072000E004201799887002E01798C1
:107D20000C9981701898169A8078C11E02290CD37C
:107D3000022811D001280CD12672BA4200D900269F
:107D40006672BA4213D8F44812E00D20000211996D
:107D500008800120800201E00C9800022081BA42D4
:107D600001D8EE4800E0FA20179988600EE0FA206A
:107D700017998860139800780028119901D0E84875
:107D80004880E848139A1083E7480880A88CF8F7E1
:107D900013FD0026E54B3246F8F796FB02460B46EC
:107DA000E3493046F8F7F8FBE24B3246F8F78CFB34
:107DB000F8F754FD0746E080DF493046109A0F9BE4
:107DC000F8F7EAFBDD4B3246F8F77EFBF8F746FDA5
:107DD00078434042800B608116990E98814208D901
:107DE0000C20149FB872D648179988831220189ACD
:107DF0000EE0480A189A149F01D00D2003E0080AEB
:107E000000D1DBE20A98B872CE4817998883122015
:107E1000F872D078052844D8784400794000874427
:107E20000227402C3339C848B881C8482FE0C046E3
:107E30007090010248C3000048C3000058C300000E
:107E400058C30000A6C00000ADC00000307500009F
:107E500010270000F8C0000005020000FF06000027
:107E6000040800000A0400003604000003020000B9
:107E7000B748F881B748388013E0B748F881B74869
:107E80003882B74838600CE0B448B881B5481799D3
:107E9000C88306E0B4487882B448B8800B980006DE
:107EA0009064AE483881A748F880B14802882A8497
:107EB000B0480078E874B0480078119F7875387D34
:107EC000139000285ED0AD490A681023DA413A6069
:107ED0000A794B79CF8867801B029A186A840A7ADC
:107EE0004B7A8F7AC87A0D7B65701B029A183B0417
:107EF000D21800061018179FF860487B8A7BCB7B4E
:107F00003B77120210186081087C7877487C149ABD
:107F10009072887CD072C87C159B1874087D587448
:107F2000487D11909874C87D0A7E120212181A8436
:107F3000887DD87418464B7EC375887ECD7E2D0211
:107F40002818B880087F4D7F2D022818F880887F78
:107F5000B877C87FF8772020085C149D287321200B
:107F6000085C68732A20085C2A314D782D02281895
:107F70008D782D044019C97809064018189988642D
:107F8000119801E0EB7DA87C7D498B700A80800010
:107F90001F38C882C883139800281FD02222774830
:107FA000825C034622335B781B029A180A842422DF
:107FB000825C034624335B781B029A18CA8426220B
:107FC000825C034626335B781B029A188A83282238
:107FD000825C283040780002801888846948032534
:107FE00069A2294602F0ACFE189F387814907B787D
:107FF000B8780F90FA78B8791390F8791190387AA8
:108000001090787AB97A0890099100930F980190AE
:108010000292169803901298049013980590119864
:10802000069010980790FAA2F8482946149B02F08F
:1080300087FE3D46643580212846F8F7B4F8B878C5
:10804000C11E02290ED3012800D18FE1022800D0E1
:10805000ABE11691149078787F225043F74940188D
:10806000F74907E01691149078785B225043F14964
:108070004018F14941182846F8F77CF80D9D1898EA
:10808000C6870E34324602E0641C0F2A0ADA2178D1
:108090000029F9D0491C8907C90F91400E43C687B2
:1080A000521CF1E71699022907D31499491E012998
:1080B00000D97DE14279D24901E04279CF4989185E
:1080C0000C78002D00D177E1C1790E91032900D9F8
:1080D0004AE14279062A00D979E14921890041180B
:1080E0001191E43010900E98401E129019A80019BA
:1080F0000F9000231392149403E01898290600D1DE
:108100005AE1052A5AD8C0467A4412795200974457
:10811000455C728598ABC04688130000E2040000FD
:108120000C080000060A0000040F000000001041C7
:1081300030C1BD41000070400000F0400000D0415F
:10814000120C0000140B000012120000140E0000AC
:108150000E160000130D0000121600000E12000093
:10816000140B0E0A12080000101600000E0B00007F
:10817000B4930102B693010298A70102A4A70102D9
:108180002094010201080000436173652070617250
:10819000616D65746572733A200D0A001693DFB243
:1081A000002F04D019A801223946F7F7F5FF002C5B
:1081B00000D191E019A8C019BB498AE0E8B20228B1
:1081C00067D00027022867D06BE00E98022872D192
:1081D000E8B2022800D103461693DFB2002F04D084
:1081E00019A801223946F7F7D7FF002C74D019A837
:1081F000C019ACA16DE0E8B2022800D104231693A7
:10820000DFB2002F04D019A801223946F7F7C4FFC6
:10821000002C61D019A8C0199FA15AE0E8B2022829
:1082200000D106231693DFB2002F04D019A8012233
:108230003946F7F7B1FF002C4ED019A8C01992A10A
:1082400047E0E8B2022800D10C231693DFB2002FDA
:1082500004D019A801223946F7F79EFF002C3BD025
:1082600019A8C019874934E0E8B2811E4A424A4140
:108270009700022804D119A801223946F7F78CFF8C
:10828000002C16D019A8C0197CA12246F7F772FF5E
:108290000FE00627022804D119A801223946F7F772
:1082A0007BFF002C05D019A8C01980492246F7F79A
:1082B00061FF169710E01693DFB2002F04D019A8C3
:1082C00001223946F7F768FF002C05D019A8C0191C
:1082D00073492246F7F74EFF3C193F2C05D80F98FB
:1082E000C0194021091BF7F75EFF12980228189861
:1082F00001D2002002E0C078411E88411599087023
:10830000611E2E46E8B202280CD1179A517019A9A5
:10831000119AB8C9B8C2B8C9B8C2B8C9B8C2B8C940
:10832000B8C20DE0179A117019A9109AB8C9B8C24D
:10833000B8C9B8C2B8C9B8C2B8C9B8C2C10709D1AA
:1083400080073546149C139A169B00D4D5E602206C
:108350008543D2E6FE20354605401898149C139AB2
:10836000169B290628D0CCE637A231E0169114904E
:1083700078780B994143334808181F386F21C94357
:108380000D9D7A180378D427D3554378D827D35531
:108390008378DC27D355002900D170E6C378E02725
:1083A000D3551031001D189FEBE70120404A10E023
:1083B0000024002D00D087E629B0F0BD80290ED31F
:1083C0000F20B872104817998883102020E525A245
:1083D0000120014602F0B4FC189829B0F0BD10202D
:1083E000402904D3B8720849179B998310E5B872E5
:1083F00004481799888314200AE5C046ADC00000E0
:10840000A6C00000150F0000140B000001080000BA
:1084100025642025642025642025642025642025EA
:10842000642025642025642025642025642025649B
:108430000D0A000085D800001DF7FFFF9DCF00004A
:1084400089FBFFFF8DD700007472785F6D6F6465E4
:1084500020706172616D65746572206572726F72F1
:108460000D0A00004E73666420706172616D657460
:108470006572206572726F720D0A0000FFFFFFFFC8
:1084800001FF0000D8C30000FFFFFFFFFF0101FF55
:10849000FF01FF01FFFF01FFFFFFFF01FFFF01FFE2
:1084A000DCC50000FFFF01FFF8C3000068C3000047
:1084B0003BCF0000002800D101481D4908607047EB
:1084C0007090010210B5002801D0044601E0184860
:1084D0000468204600F006FC204600F021F80B4816
:1084E00041780B4A1A23136041704078FF2109023A
:1084F000084A13688B438007000CC01810600648B8
:10850000202101600548016010BDC046B8930102FA
:108510007020004004E400E080E200E000E100E0C0
:10852000F0B586B0002805D10148006802E0C046D9
:10853000C89301023121C900049141188A791F238F
:108540001A40CD79ED06AD0DAA180D7AED066D0C29
:1085500052194D7AED062D0B52198D7AED06ED0963
:108560005219CD7AED06AD0852194D7CED0752191E
:10857000BD4C22600A7B1A404E7BF606B60DB2183F
:108580008E7BF606760C9219CE7BF606360B921988
:108590000E79F606F60992194E79F606B608921982
:1085A00062604A6AB14D2A40A2608A6A2A40E2604B
:1085B0002D22D20087183A7E1A4003937E7EF6065B
:1085C000B60DB218BE7EF606760C9219FE7EF60641
:1085D000360B92193E7FF606F60992197E7FF60653
:1085E000B60892190E7CF60792192261BA7F1A40DA
:1085F0000597FE7FF606B60DB218049BC35CDB063A
:108600005B0CD2184B78DB061B0BD2188B78DB0681
:10861000DB09D218CB78DB069B08D2186261CA69E5
:108620002A40A2610A6A2A40E2618A7C01252A4026
:10863000CB7CDB079B0F9A180B7DDB075B0FD218F7
:108640004B7D9B07DB0ED2188B7DDB079B0ED21870
:10865000CB7D1B079B0D9A180B7E1B079B0CD2181A
:108660004B7E5B06DB0A13438A7E520612091A43CD
:10867000CB7E5B075B0813432362CA6A62620A6BA4
:10868000A2624A6BE2628A6B22633922D200835C67
:108690001E462E4066635E425E41B304AE04744FD4
:1086A0003C68B443E3183B6083185A782A409C78AE
:1086B0002407E40EA2188C8F6401A2186D4C14409C
:1086C000C98FC905490A0919DA78D207120A891827
:1086D0001A791207120989185A79D207D20889180B
:1086E000FB4EB1639968F163997904952940DA7971
:1086F000D207920F51181A7B5207D20E89185A7B53
:10870000D206920D51189A7B5207D20C8918DA7B47
:10871000D206920B89181A7CD206520A89185A7C02
:10872000520792090A43997CC906490851183164D5
:10873000D97C039A11401A7DD206920D51185A7DA8
:10874000D206520C89189A7DD206120B8918DA7D4E
:10875000D206D20989187164197E0F2421405A7EED
:10876000120151189A7E12038918DA7E1207120A32
:1087700051181A7F1207120989185A7F120789188F
:10878000B164997F01942140DA7F1207120E5118CB
:108790003D22D200835C5B075B0D59188418627818
:1087A0001207520C8918A278D206120B8918E278A7
:1087B000D206D2098918F164217907220A40617929
:1087C000C9008918A2795206920B5118E2799207D2
:1087D000120B8918227AD2078A18BF490A60627A76
:1087E000A37A1B029A18E37A1B04D2184A60E28922
:1087F000BA4B13400394228AD2049209D2188A6099
:1088000003463033598CB64A114002939A8CD205F4
:10881000D20A51185622825C12068918B14D29607D
:10882000014656314A788C782402A2188C88640557
:108830006409A218CC78240712196A60CA880C7AD5
:10884000A407A40BA2184C7A6407E40A1219AA60C0
:108850004989E960492189004118FF22663282185E
:1088600000921035002207E000300040FFFFFF00BB
:1088700004040040FF3F000084186427E65D0327DE
:108880003E406523E35C9B071B0F9B196626A65D94
:10889000B607B60EF3186726A65DB601F318DBB26D
:1088A0006826A65DB607B60DF3186926A65DB6075D
:1088B000360DF3186A26A65DB607B60CF3186B26BC
:1088C000A65DB607360CF3186C26A65DB607B60B88
:1088D000F3186D26A65DB607360BF3186E26A65D57
:1088E000B607B60AF3186F26A65DB607360AF31860
:1088F0007026A65DB607B609F3187126A65DB60701
:108900003609F3187226A65DB607B608F318732663
:10891000A45DA407E31808C51032802AACD1019ADF
:10892000D243704EB4180B783B404D78AD072D0FF5
:10893000EB188D78AD07AD0EEB18CD78AD01EB18C7
:10894000DBB20D79AD07AD0DEB184D79AD072D0DEF
:10895000EB188D79AD07AD0CEB18CD79AD072D0C6B
:10896000EB180D7AAD07AD0BEB184D7AAD072D0B5B
:10897000EB188D7AAD07AD0AEB18CD7AAD072D0A4D
:10898000EB180D7BAD07AD09EB184D7BAD072D093D
:10899000EB188D7BAD07AD08EB18CD7BAD07EB1861
:1089A000A3641031121DBDD1009B19785A7852076B
:1089B000520D51189A78D207120D8918B164059B8F
:1089C0001968F164D97D5A681202511831659968A5
:1089D000454A0A40998A490589187165D9683D4C0C
:1089E0002140B16519692140F165029E3178049DED
:1089F000294082785207120F5118C2799207920EBD
:108A00008918427A9207920D5118827A9207120DB4
:108A10008918C27AD207920C89189A7DD207520C13
:108A2000891872789207D20B8918B2781207D20A85
:108A30008918F2781207D2098A182C490A60327C08
:108A4000737C1B071B0D9A18B37C9B069B0BD218DB
:108A5000F37C1B079B0AD218337DDB065B09D21817
:108A6000737DDB071B09D2184A60B27D2A40C38F91
:108A70005B009A188A60826CCA60C26C22400A61EC
:108A8000F27D7F231340328C5204520AD2184A617D
:108A900002698A614269CA6182690A62C2694A627C
:108AA000026A8A62426ACA62826A0A63C26A4A6364
:108AB000039A927CD201121D0A64027A3A40CA6576
:108AC000808F074A10400866002006B0F0BDC046FF
:108AD00000300040FFFFFF009C300040FF1F0000FF
:108AE000FF03000000400040FFFF1F000020004087
:108AF00004480068806B80080349096849004018F1
:108B000009307047C89301021004004010B52D21B0
:108B1000C9004118027A032A04D10079002807D03D
:108B2000082006E08378DA1E022A05D2032412E028
:108B3000142088601C203DE0012B02D1C8228A60ED
:108B400012E00479042C01D3462404E0032C01D163
:108B5000322400E014248C605B1E022B04D3022A12
:108B600010D24279154B01E04279154B9B181B78C6
:108B7000402B04D0102B06D11423442405E02A23D3
:108B80003E2402E04279342348244B800C80022AA0
:108B900006D0062A08D0052A08D118224C2301E065
:108BA000142250230B8000E01C224A80C078042845
:108BB00003D1142048806420088010BDADC000009F
:108BC000A6C00000424800687047C04610B53F4A42
:108BD000107091703E49002813D05068086104203D
:108BE00048619078FF2212023A4B1C68944380033C
:108BF00080B20019186001204007054A1060364A0B
:108C0000106000200860354901220A6010BDC0468E
:108C100080E200E03148002101602D4801680268CF
:108C20008A420BD0016802688A4207D00168026854
:108C30008A4203D0016802688A42EFD17047C04679
:108C4000F0B581B021480178214D002911D08178FB
:108C5000FF2212021F4B1C689443890389B2091931
:108C60001960012149071C4A1160406828610420ED
:108C700068610127EFF310803840009002D1EFF3D4
:108C8000108072B6154807602E682868B04208D177
:108C90002868B04205D12868B04202D12868B042A5
:108CA000F3D0FDF797FD0446F7F76BFD0C49F7F796
:108CB000DEFAF7F7BEFD3018B843286000980028A8
:108CC00000D162B6204601B0F0BDC046B8930102A3
:108CD000180400401CE400E000E100E070000040E7
:108CE00080096E45F0B591B0002801D1C0480068F8
:108CF0008778F91E022913D3012F21D0022F3CD1EE
:108D00001021CA4344782146193991423DD8009731
:108D10000125B94A28462946234602F011F853E1B5
:108D20000821CA43447821462139914218D8009736
:108D30000125B14A28462946234602F001F843E1BD
:108D40000821CA43447821460939914234D8009712
:108D50000125A94A28462946234601F0F1FF33E1BF
:108D6000032F3CD0042F43D1C3780125042B00D01E
:108D70002DE106462A02042343E00125A6A2284647
:108D800029463B4601F0DCFF1EE1C3780125052B97
:108D90000AD806462A02284698401B21084230D1AC
:108DA0000021052B08462ED002200090914A28462B
:108DB000294601F0C5FF07E10646C3780021022BD2
:108DC0001ED3032B1CD0042B08460A461BD00125BA
:108DD0000095884A2846294601F0B2FFF4E0C3789E
:108DE0000125032B00D0FAE006462A02032308E0FF
:108DF000012583A2284629463B4601F0A1FFE3E076
:108E00000A46012148020F91592189007518FD2158
:108E1000490071180291314662313F05D219641E32
:108E20001F2727405C013C19144304433279520741
:108E3000D20C22432B789B065B0BD218B379DB074D
:108E40001B0B13436D4D2B60F279032310931A40D3
:108E5000737A9B079B0E9A18B37A5B07DB0D9A18FF
:108E6000F37ADB079B0DD218337BDB075B0DD2183F
:108E7000737B1B075B0CD218AA603269EA607269C7
:108E80002A61B2696A61F269AA61326AEA61726A48
:108E90002A62B26A6A620F980870F06AA8623F207C
:108EA000C4432C353046E4300F903046E5300E9008
:108EB0003046E6300D903046E7300C903046E830D2
:108EC0000B903046E9300A903046EA30099030463F
:108ED000EB3008903046EC3007903046ED3006908D
:108EE0003046EE3005903046EF3004903046F0309A
:108EF00003903746F1373046F230F3360F990A19AE
:108F00004021525C109B1A400E9B1B195B5C9B0717
:108F10001B0F9A180D9B1B195B5C9B079B0E9A18E5
:108F20000C9B1B195B5C9B019A18D2B20B9B1B1903
:108F30005B5C9B079B0D9A180A9B1B195B5C9B074C
:108F40001B0D9A18099B1B195B5C9B079B0C9A18BD
:108F5000089B1B195B5C9B071B0C9A18079B1B1932
:108F60005B5C9B079B0B9A18069B1B195B5C9B0722
:108F70001B0B9A18059B1B195B5C9B079B0A9A1895
:108F8000049B1B195B5C9B071B0A9A18039B1B190C
:108F90005B5C9B079B099A183B195B5C9B071B0951
:108FA0009A1803195B5C9B079B089A183319595C44
:108FB0008907891802C51034A0D1029800780421CD
:108FC00001430E48C1630025284611B0F0BD0420BE
:108FD0000090084A2846294601F0B2FEF4E7032033
:108FE0000090044A2846294601F0AAFEECE7C04654
:108FF000C893010210CF000056CF000000100040BF
:10900000556E646566696E6564206D65616E20509D
:1090100052462025640D0A00496E76616C69642011
:109020006D65616E205052462025640D0A000000D7
:10903000B0B584B00446FBF72AF91F4801680091D7
:109040004168019181680291C0680390FFF7E2FDD9
:1090500000F03AFD1948016804220A430260184DE5
:109060006868A021002C01D1884300E008436860B3
:10907000FF200230FBF754FAFBF76CFE0020FFF7ED
:1090800021FAFEF7BFF86846FEF76CFB0D48016851
:10909000C907FCD0012080022968814329600A4861
:1090A000FBF73EFAFFF7CCFD4B49086000F02AFDC4
:1090B000FBF7F2F804B0B0BD80A0005010ED00E066
:1090C0002C0000402C020040010200007047704755
:1090D00080B50E490E480246083A1268920000D444
:1090E000603142680A4342600A490A6808239A4389
:1090F0000A60091F012252040A60032189040268E0
:109100008A430260FBF7DEF880BDC0462000008085
:109110002800004004020040B0B5032000072D499C
:109120000A68824301256807101808600024204659
:10913000FFF7CDFF2046FFF7C9FFEFF3108028406F
:1091400002D1EFF3108172B68021C943224A5368DD
:109150000B40536093680B409360D3680B40D3601F
:1091600013690B40136153690B405361002800D110
:1091700062B6B0BD70B50C4603210907154A1368E5
:109180000B4313600122EFF31081114002D1EFF382
:10919000108272B68025EA430F4B5E6816405E600F
:1091A0009E682E439E60DD681540DD601D69154098
:1091B0001D615D6915405D61002900D162B600281E
:1091C00002D00120FFF783FF002C02D00120FFF71F
:1091D0007DFF70BD00040040389501020D4A002952
:1091E00007D001290BD1012181401068884310600C
:1091F00007E00121814010680843106001E001216F
:109200008140101F02680A430121C9071143016010
:109210007047C04644000040032804D84000064977
:10922000085A00B27047002000B27047032802D8E5
:109230004000014A11527047D2A701029E490870AE
:109240007047C04670B58AB00C460546FF20FC301A
:10925000A8490E68315C59208000335CB2783078C0
:1092600008AE069609AE05960C4E049621267606A3
:1092700003960B4E0296012601960E2600965B1C65
:10928000DBB2F9F7BDF80998F7F7BAFA2870089831
:10929000F7F7B6FA20700AB070BDC0460000204152
:1092A00000000443F0B58BB00446457C824800784A
:1092B0008249002822D000200880814A1080814BFA
:1092C00001269E761E830A907F4800787F4E36786E
:1092D0006DB205957E4D04957E4D03950AAD0295C0
:1092E0007D4D01950096F8F7C9FD0A9D1120205685
:1092F0007A497B4A00F0D8FB064626E000260E801D
:109300006F4A16806F4B01209876188309966E4835
:1093100000786E4F3F786DB205956D4D04956D4D9B
:10932000039509AD02956C4D01950097F8F7A6FDE0
:10933000099D112021567F20C005009001900296C2
:10934000664A674B3046F9F7EDFE43200106284692
:10935000F6F78DFFF7F754FA089062480078002876
:1093600024D05120800060494A7D42438D185F48D7
:109370000068A8642F46403750480078B8745048B9
:109380000078F87455480078387555480078787535
:1093900057480078F87550480069F7F731FAB87502
:1093A00052484069E8644C4800686864FF20FE3019
:1093B00050490968085C3922D2008918022812D362
:1093C00003D04E48007801280DD14B480660434831
:1093D00000883A4A108042480088394A10800920A3
:1093E0000790089605E04448089A02603548C08B0B
:1093F00007900B780022002B01D0114600E0D143EA
:109400000125002B01D0042300E0EB43A67AAD1B1D
:10941000EE175B1971416568AE0F277AAD00ED1943
:109420005641677A3F1FF817ED1970414000EE0F63
:1094300080196D00EB1848418001990E4118980180
:1094400027239B02C31A91411D4805881B480088A9
:10945000854201D00798421B10202056C001194DAB
:109460002D8C032D07D1E468E5176D0A6419E41506
:109470000519EC170FE0E468E5176D0A6519EC179C
:10948000ED15C6174519744197B2002F00D0344628
:10949000002F00D00546581BA141130409D012B279
:1094A000D2015242D31780185941089BDA17C01ACB
:1094B00091410BB0F0BDC0465E93010288A6010247
:1094C00086A60102209401026190010260900102CF
:1094D000749C0102749A01028CA60102D6A60102B4
:1094E000D4A6010240A00102789D01026420004040
:1094F00084A60102C893010280A60102D8A6010237
:10950000C10D4002803070470120C0071B49086030
:109510007047C04610B519480068C10710D18107CF
:1095200011D4410712D4010713D4C10614D4810603
:1095300015D4410616D48021084016D031A215E07A
:1095400001240FA213E0022411A210E0032414A2AC
:109550000DE0042416A20AE0052419A207E006245F
:109560001CA204E0072421A201E0254A04090220EC
:10957000032101F0E5FB204610BDC0465C00004021
:10958000526573657420627920504F520D0A0000B5
:10959000526573657420627920424F520D0A0000B3
:1095A00052657365742062792050494E0D0A00009F
:1095B0005265736574206279205744540D0A000087
:1095C0005265736574206279204C4F434B55500DA2
:1095D0000A00000052657365742062792053572099
:1095E0005265626F6F740D0A00000000526573656A
:1095F00074206279205359535245510D0A000000DE
:10960000BACB0000526573657420627920445644D9
:10961000440D0A0001218140044A1F2802D010682D
:109620008843106010680843106070471C000040B9
:10963000F0B583B0029104469949F6F74BFD054613
:10964000984901942046F6F745FD974946189749F1
:10965000714300956F189649441864212046F6F727
:1096600039FD3818A108471A92492046F6F748FDF7
:10967000381891494518914F05D464213046F6F7C2
:1096800029FD0C4614E0A6B264213046F6F722FD0F
:10969000B7204000A20701D1002907D1884B7343AE
:1096A0000422D341874A934200D3401E0C464519F9
:1096B0000098474302980680192001013046F6F7CA
:1096C00009FD2A461F3A284600DB1046019BFF1879
:1096D000B30705D1002C03D01F2D05DA0120C5E00A
:1096E0001F2D0BDA0120C1E005461D3D034600DBBE
:1096F0002B461C2808DC02201546B7E000290CD0B8
:109700001C21451A0CD50CE019461F39184600DB00
:1097100008461F2B1DDA0320A8E01D21451A00D49E
:109720002846002D08D401461F39024600DB0A46B0
:109730001F2804DA032099E00220154696E015461A
:109740001E3D104600DB28461E2A0CDA04200D467A
:109750008CE005461E3D024600DB2A461E280BDA39
:1097600004200D4682E001461F39024600DB0A460E
:109770001F280ADA052079E011461F39104600DB60
:1097800008461F2A0BDA052070E015461E3D1046DC
:1097900000DB28461E2A0CDA06200D4666E0054648
:1097A0001E3D024600DB2A461E280BDA06200D4627
:1097B0005CE001461F39024600DB0A461F280ADA30
:1097C000072053E011461F39104600DB08461F2AC8
:1097D0000BDA07204AE015461F3D134600DB2B46F7
:1097E0001F2A0CDA08200D4640E005461F3D0246C0
:1097F00000DB2A461F280BDA08200D4636E0194602
:109800001E39184600DB08461E2B0ADA09202DE017
:1098100011461E39104600DB08461E2A0BDA0920C5
:1098200024E01F28054601DB05461F3D1F280CDAF2
:109830000A200D461AE01F28054601DB05461F3D9C
:109840001F2806DA0A200D4610E01E2D05DB0C202D
:1098500004E01E2D06DB0C2005E00B201E2D05DB91
:109860001E3D03E00B201E2D00DB1E3D029EB0704E
:10987000681CF070E12001013846F6F72BFC3071CE
:10988000C0B211494143CC193C212046F6F722FCD5
:1098900070713B21C94341430819B07103B0F0BD59
:1098A000805101008033E101B207000093FEFFFF09
:1098B000B107000070FEFFFFA7FA0A0080AEFEFFAE
:1098C000295C8FC20BD7A300F0F1FFFF70B50446EF
:1098D000FFF722FCA08A244EB082B18A002908D06A
:1098E000F0820220B07100207082FFF76BF9F06106
:1098F00070BDE08A7082A169728A1C48F6F73AFC52
:109900002046FFF7CFFC05460C461948007BFFF7C1
:1099100083FC81B2C90B401800B2C1174010281A4D
:1099200030678C417467FFF74DF9B061F06D401CF2
:10993000F065FEF7B9F8F064FAF7CCFB0446306541
:109940000C48406AF6F7D6FF0B4A0C4BF6F7BCFD05
:10995000F6F784FF01462046F6F7D2FBFAF7B0FD92
:109960000120B07170BDC046A0960102DCA70102C3
:1099700062900102F8C000008DEDB5A0F7C6B03EC0
:10998000F0B581B0EFF3108072B600200146FBF70E
:1099900055FE0446002803D062B6204601B0F0BD53
:1099A00001273A030025074E28463146FBF7A0FD64
:1099B000BB02054A28463146FCF79CFA62B62046AF
:1099C00001B0F0BD00E002047EA2010207488178E8
:1099D000491C8170C9B2782903D10121417000214D
:1099E00081700348012141707047C046969701027B
:1099F0001490010270B514460D4606461120FAF780
:109A00000FFE2248042101600C4804601E480560D6
:109A10008660002E0DD0FF20000609490A688243A7
:109A20000120C00710180860064808210160064898
:109A300001601A200221FFF7D1FB70BD78A8010256
:109A400000E400E080E200E000E100E00C49086092
:109A50007047C04610B5044609480068604309498C
:109A6000F6F74EFB001908494860084800220260DA
:109A700002460C3A4B6813600968016010BDC0468D
:109A800074A8010240420F00089001022C1001400E
:109A900000480047C100000080B502490968C96D4F
:109AA000884780BD0090010280B582B013460A4607
:109AB00000900348011D0348F9F7E0FA02B080BDA9
:109AC000B4A80102AC9901023B4800210160816801
:109AD0004068401C534A13685B0104D400290246C5
:109AE00009D00A4607E04D490B685B1C0B60012159
:109AF00049061160024649494860801ACA688018C0
:109B0000C860704770B5454E71682748821C914205
:109B10002AD2491E284A516028490B680340032075
:109B200084071B190B60002191601060FCF752FE46
:109B3000054674682146F6F7CDFAF16849192246C0
:109B40004243891AF160A14204D3091B401CA1427F
:109B5000FBD2F160316809183160002803D0306908
:109B6000002800D0804770BD10481149E622114BF3
:109B700000F088F810B50C498A1C90420DD2401EA6
:109B80000D4A50600D4803680B4003218C071B19D8
:109B9000036000209060116010BD04480449E62273
:109BA000044B00F06FF8C046FFFFFF0091CB0000B0
:109BB000ABCB000077CB000010E000E020ED00E030
:109BC000B0B50120EFF31081014002D1EFF3108214
:109BD00072B6124A1368124C2268646885061148EE
:109BE00000682840850E5D192923DB006B43002C9B
:109BF0001D4606D1002809D11E20684300290AD03D
:109C0000B0BD121BD218551C0028F5D01D461E20D1
:109C100068430029F4D162B6B0BDC046E4B3010286
:109C200014E000E004ED00E080B50020FAF704FF46
:109C3000404280BDB0B586B0104869460A4638C873
:109C400038C238C838C200242046FAF7FBFE039910
:109C50002046FAF791FF0198012803D00824002834
:109C600004D102E00424002800D104460220FAF7BF
:109C7000DFFCE0400249086006B0B0BDB4C000009F
:109C8000F8B3010290B01C4605AB07C3EFF3108098
:109C9000C00702D1EFF3108072B6EFF310800B9083
:109CA00068460E907046089010AB0F93CF4F3E1D44
:109CB00001200490C50230462946224600F0B8FC37
:109CC00000213154EFF303800990EFF308800C90EA
:109CD000EFF309800D90EFF314800A9000F02CFC54
:109CE0003868012833D80028C14F00D0C14F2A203E
:109CF000C1497A69920703D50A783A60401E491C27
:109D00000028F6D1B948041D2046FFF7C5FE0028FB
:109D100007D079698907FAD521783960401E641C1B
:109D2000F5E70220B5497A69920703D50A783A60C7
:109D3000401E491C0028F6D12A20AF497A699207B3
:109D400003D50A783A60401E491C0028F6D1FFF777
:109D500037FF0346AA4A30462946FDF7E3FD04468D
:109D60003018291B089F3B1F049A9343A5A2FDF7B7
:109D7000D9FD9E490968012966D8001900299C4C23
:109D800000D09C4C00280AD09849091D62699207AE
:109D900003D50A782260401E491C0028F6D10A200B
:109DA0009F496269920703D50A782260401E491CC8
:109DB0000028F6D10598FFF76FFE002809D06169E9
:109DC0008907FAD5059A11782160401E521C059228
:109DD000F3E7022089496269920703D50A78226075
:109DE000401E491C0028F6D10A208EA16269920704
:109DF00003D50A782260401E491C0028F6D1069837
:109E0000FFF74AFE002809D061698907FAD5069A4A
:109E100011782160401E521C0692F3E70220774918
:109E20006269920703D50A782260401E491C002807
:109E3000F6D10A207EA16269920703D50A782260D2
:109E4000401E491C0028F6D17CA230462946079BBB
:109E5000FDF768FD6549096801290E9B1BD800299B
:109E6000634900D0634900280AD0604A121D4C693A
:109E7000A40703D514780C60401E521C0028F6D1AC
:109E800002205E4A4C69A40703D514780C60401E7A
:109E9000521C0028F6D16AA230462946FDF742FD41
:109EA00004463018291B694A3B46FDF73BFD4F49E4
:109EB0000968012911D8001900294D4900D04D49E0
:109EC00000280AD0494A121D4B699B0703D5137815
:109ED0000B60401E521C0028F6D15D4A30462946D0
:109EE000099F3B46FDF71EFD0446F800C00FB90070
:109EF000C90F7A00D20F0092019102903019291BEC
:109F0000FB0F544AFDF70EFD04193019291B3F239E
:109F10003B40514AFDF706FD34490968012911D833
:109F200020180029324900D0324900280AD02F4A8F
:109F3000121D4B699B0703D513780B60401E521C02
:109F40000028F6D1454A304629460B9BFDF7EAFC2E
:109F500004463018291B424A0A9BFDF7E3FC2349BB
:109F60000968012911D800190029214900D0214987
:109F700000280AD01D4A121D4B699B0703D5137890
:109F80000B60401E521C0028F6D1364A3046294646
:109F90000C9BFDF7C7FC04463018291B324A0D9B69
:109FA000FDF7C0FC114909680129114A0DD80019B3
:109FB000002908D00F4A06E05169890703D5317896
:109FC0001160401E761C0028F6D128490E98091A07
:109FD000A94200D32946890800F03CFE24480068C5
:109FE000002800D0804700F045F8C046C8B4010200
:109FF0000090014000A00140EBCB00007ACF0000B0
:10A00000D4CB00000D0A232323204153534552543F
:10A01000204020307825303858202323230D0A0093
:10A02000AECC000046554E4354494F4E3A200000F6
:10A030004C494E45202020203A2000002564000095
:10A040000D0A53503D253038580D0A0073CC0000DE
:10A0500089CC000095CC00007DCC000032CC000003
:10A0600041CC000050CC00005BCC000000F80202A4
:10A07000C4B40102F7480068012811D8002801D0B3
:10A080000B4800E0FC480C210A4A01E0002907D0F7
:10A0900043699B07FAD513780360491E521CF5E704
:10A0A0001E20FFF7B7FA00BF00BF00BF00BFFAE7EE
:10A0B00000A00140DECB00008AB00646E448B0664E
:10A0C00000F03AFAFFF77CFD0346E248041D012048
:10A0D0000590C502E04A20462946FDF723FC0746C5
:10A0E00008942018DB4C0995E91BF36C3F2206927B
:10A0F0001340DAA2FDF716FC2168012910D8C01917
:10A100000029DD4900D0DD49002809D0221D4B6916
:10A110009B0703D513780B60401E521C0028F6D114
:10A12000F36BD7A2089C2046099D2946FDF7FAFB50
:10A130000746291A2018336C069A134007D1D8A273
:10A14000FDF7F0FBC34C2168012907D917E0CEA227
:10A15000FDF7E8FBBF4C2168012910D8C019002980
:10A16000C54900D0C549002809D0221D4B699B076D
:10A1700003D513780B60401E521C0028F6D100272F
:10A18000CBA5B80030580090089809992A463B465C
:10A19000FDF7C8FB216801290FD80029B64900D076
:10A1A000B649002809D0221D4B699B0703D51378B7
:10A1B0000B60401E521C0028F6D17F1C0D2FE0D1F1
:10A1C000736BBFA2089C2046099D2946FDF7AAFB98
:10A1D000074620189F4CE91BB36BBC4AFDF7A2FB56
:10A1E0002168012910D8C0190029A34900D0A3492A
:10A1F000002809D0221D4B699B0703D513780B60FB
:10A20000401E521C0028F6D1336CB14A089C2046EF
:10A21000099D2946FDF786FB0746326CD000C00F2A
:10A220009100C90F5300DB0F009301910290E019D8
:10A23000E91BD30FA74AFDF775FB3246C619A019D3
:10A24000A91B1546136C069A1340A34AFDF76AFB37
:10A2500080490968012911D880190029864900D050
:10A26000864900280AD07B4A121D4B699B0703D5FB
:10A2700013780B60401E521C0028F6D12E466B6CE2
:10A28000964A089C2046099D2946FDF74BFB074648
:10A290002018E91B0796B36C914AFDF743FB6D4A02
:10A2A0001168012910D8C0190029734900D07349D9
:10A2B000002809D0121D4B699B0703D513780B604A
:10A2C000401E521C0028F6D10798426E04236021DC
:10A2D0005C2004931A400B4600D003460693002AE4
:10A2E00000D00846079E33587E4A089C2046099DA8
:10A2F0002946FDF717FB074606983358E019E91B76
:10A30000794AFDF70FFBC619A019A91B079A536ECE
:10A3100076A2FDF707FB4F490968022911D280197F
:10A320000029554900D0554900280AD0494A121D34
:10A330004B699B0703D513780B60401E521C002805
:10A34000F6D10798C36C06466DA2089C2046099D6D
:10A350002946FDF7E7FA07462018E91B336D6B4ADB
:10A36000FDF7E0FAC619A019A91B079F7B6D68A22B
:10A37000FDF7D8FA8619A019A91BBB6D67A2FDF7D6
:10A38000D1FA344909680129059C11D8801900299E
:10A39000394900D0394900280AD02E4A121D4B698C
:10A3A0009B0703D513780B60401E521C0028F6D182
:10A3B0000798476B5D4A974237D2032087430026B0
:10A3C000059CB00039580246049B1A43BA5808232A
:10A3D0000343FB580C2505437D59009101920293DC
:10A3E00003953B1808980999514AFDF79BFA1949BA
:10A3F000096801290FD800291F4900D01F490028EA
:10A4000009D0089A4B699B0703D513780B60401E4F
:10A41000521C0028F6D11B2E444A06D80798406BE0
:10A42000361DB10040189042CBD30798406B111AEB
:10A43000099A914201D8890800E0610200F00AFC03
:10A440003C480068002800D08047FFF713FEC04654
:10A4500022224B4DC8B40102D4CB00000D0A0D0AD4
:10A4600023232320455843455054494F4E2025640B
:10A47000202323230D0A00000090014000A001408A
:10A4800050433D25303858002C2045786365707462
:10A49000696F6E4E756D6265723D25640D0A000030
:10A4A0002C205468726561644D6F64650D0A00006C
:10A4B00052252D32643D253038580D0A0000000029
:10A4C00053503D253038580D0A00000073CC000071
:10A4D00089CC000095CC00007DCC000032CC00007F
:10A4E00041CC000050CC00005BCC00004558435FDD
:10A4F00052455455524E3D253038580D0A00000043
:10A50000494353523D253038580D0A0066CC0000AF
:10A510005343523D253038580D0A00004343523D05
:10A52000253038580D0A0D0A0000000000F802021C
:10A5300016CC0000C4B40102F0B583B0344D2C68D1
:10A54000012C06D8601E8441204601F0ABFA002899
:10A55000FAD10120EFF310810140019102D1EFF314
:10A56000108072B62B48285A2B49695A814245D02F
:10A570002A68002A01D02A4E00E0284E1F23DB0261
:10A580000293284C022A27D205E01046214AA852FD
:10A5900082B2914232D087B2B9420A4600D8621CD8
:10A5A000131A21482B5218040DD0E819001D9FB230
:10A5B00001E0002F07D073699B07FAD50378336059
:10A5C0007F1E401CF5E7A242DFD902981018DDE794
:10A5D000304683B299420CD0024680B281420E4688
:10A5E00000D8661CA642F3D90298301883B299426B
:10A5F000F2D108496852B01A0B4968520B48002141
:10A6000029540198002800D162B603B0F0BDC046BD
:10A61000C8B401020A0800000808000000900140C8
:10A6200000A00140FF0700000C0800000F08000018
:10A63000F0B58DB00793174600240C9409AA13C2F5
:10A6400015E006986849F5F712FEF6F7D9F8C11734
:10A65000401848406549F5F73DFD009509A80622D8
:10A660003346F9F79BFBBDE0002C00D5BEE13878FE
:10A670007F1C25280DD0002800D1B7E10B9A511C72
:10A680000A9B9942F0D8099B9854641C0C940B9136
:10A69000EAE708940025397823390D2914D80120D8
:10A6A0007944097949008F44090F0F0F0F0F0F0FDD
:10A6B0000B0F060F0F0D05437F1CECE70820FAE790
:10A6C0000420F8E70220F6E7387801463039002404
:10A6D000092902D9264639460BE000260A21714392
:10A6E0000E18303E791C78780246303A0A2A0F4616
:10A6F000F4D32E2817D14A1C48780146303909294D
:10A7000005D911464F1C2538532811D96AE0002479
:10A710000A2161430C18303C511C50780246303AF3
:10A720000A2A0A46F4D34F1C2538532800D959E089
:10A730004000C0467844808840008744A000530011
:10A740005300530053005300530053005300530071
:10A750005300530053005300530053005300530061
:10A760005300530053005300530053005300530051
:10A770005300530053005300530053005300600034
:10A780005300530053005300530053005300530031
:10A790005300530053005300530053005300530021
:10A7A00053009800530053005300530053005300CC
:10A7B0005300530053005300AD00B6005300600037
:10A7C00053005900530053005300590053005300E5
:10A7D0005300DE0053005300BD005300D30053006C
:10A7E000530098000C9C3FE70024744940420F003E
:10A7F000791C38780F4625385328F3D898E70799FD
:10A80000C91D07208143086807914968F6F786F853
:10A8100000210690F5F754FF00280BD10B99481C36
:10A820000A9A904206D8099A2D2353540899491C34
:10A830000C910B900798083007900698F5F7E0FF09
:10A840000095C2178118514009A822463346F9F7EE
:10A85000A5FA0B98411C0A9A914200D9F1E6099A8F
:10A860002E2313540B910C98401C0C90E9E607988A
:10A8700002C807900096019509A8102239E00B98AC
:10A88000411C0A9A9142ADD8099A252313540B9181
:10A890000C98401C0C90A5E70B9A511C079C201D9E
:10A8A0000A9B994239D907909CE7079802C80790FC
:10A8B000009509A82246D3E6079901C9079109998D
:10A8C0000A9A089E02E0401C002E8BD40378002BCD
:10A8D00088D00B9D6C1C9442F5D84B55761C0C9679
:10A8E0000B94F0E7079802C807900096019509A815
:10A8F0000A222346F9F7F0FA74E7079B10CB102CD5
:10A90000079308D300202146401C0A09FF2911465D
:10A91000FAD806280AD8082009E02368099CA3541D
:10A92000089A521C0C920B9107905BE7401C069012
:10A9300009230C980B9D099905910A9E04940DE03A
:10A94000202104463046059E715506462046049C4B
:10A95000401C15460146089100290AD45B1E069941
:10A96000994206D26A1CB242EAD908990891002994
:10A97000F4D50C900B950898002800D532E70126F5
:10A98000082501E06D1E3601022DFBD2204631461E
:10A99000F5F7A0FB0F28F6D80C98059009980390BE
:10A9A0000A9806900B9D20463146F5F793FB691CEB
:10A9B000069A914204D90899089100290CD511E012
:10A9C0000C4A125C039B5A55089A521C0D4605927C
:10A9D00011460891002905D47043241A3009102E1D
:10A9E0000646E0D205980C900B95FBE620460DB08C
:10A9F000F0BDC04638C3000070B588B000220328FF
:10AA000003D9D243104608B070BD804CC44D2A51C2
:10AA10000F4B104EEE5081231E010123AB552860D1
:10AA20002C1962600128EDD8079300220692059246
:10AA3000049203230393029201920091411E8841E4
:10AA4000694600F0CFFC0246104608B070BDC04613
:10AA500004080000FFC0FFC0F0B583B00C4600231F
:10AA6000D943012C56DB074602910126EFF31085EE
:10AA7000354002D1EFF3108072B65849584A505C05
:10AA8000002800D0A3E056545F48115A5F48105A7E
:10AA90000196F202161A814240D832465218A2425A
:10AAA00040DB00930295A642354600DB25464C4923
:10AAB0000818001D39462A46F5F75CFBA642484EA9
:10AAC00004DA7919621B301DF5F754FB4F48305AF0
:10AAD000001981B24E4A914201D94E494018029D57
:10AAE000009B4A49705230464B4E805D002865D12C
:10AAF000EFF310850198054002D1EFF3108072B694
:10AB0000374A4148115A4148105A884232D1434885
:10AB100013524FE00C46204603B0F0BD424252189B
:10AB2000A242BEDA3C4A2E4EB25C002A0CD03B4A0E
:10AB3000B25A51188AB2364CA242284C029F01D90F
:10AB4000344A8918314A02E0244C304A029F335576
:10AB5000B152421A89B2884202D22D488018421C52
:10AB600093B23048012130A200F0EAF83C46002DB3
:10AB7000D1D128E0019F9755884201D82448401C34
:10AB8000421A90B2800A01D0019882022348144FE1
:10AB90003A52386801280DD8431E9841104B591875
:10ABA000091D92B21E4B00F017FE009B002801D039
:10ABB0000B488355002D029D00D162B60748084915
:10ABC0000B54002DA7D162B6204603B0F0BD054856
:10ABD00005A1094A09A3FFF755F8C0460E08000071
:10ABE000C8B401022ACD000074726163655F6F759D
:10ABF00074707574000000000E020000545241434E
:10AC000045204255535900000A080000080800007A
:10AC1000FF07000000F8FFFF0F0800000C0800000D
:10AC20006DAE000002FF00000D0A547261636520E2
:10AC30006275666665722069732066756C6C2C207F
:10AC40006469736361726473202575206279746529
:10AC5000730D0A00F0B587B00546002606960596E6
:10AC6000049603960296800701D007B0F0BD0191CB
:10AC700002A8142126A2FCF755FE294909680129DA
:10AC800011D80029274900D0274900280BD002AA53
:10AC900001E0002807D04B699B07FAD513780B60B9
:10ACA000401E521CF5E701990029DED0204C3746A2
:10ACB000B8002B58D80724D0581EA04204D31B48F4
:10ACC00018181C4A90421CD802A814211AA2FCF79A
:10ACD00029FE13490968012911D80029114900D01A
:10ACE000114900280BD002AA01E0002807D04B69C7
:10ACF0009B07FAD513780B60401E521CF5E7761CB3
:10AD000001997F1C8F42B0D2322ED1D3ADE7C0461D
:10AD10000D0A4261636B74726163653A200D0A002B
:10AD2000C8B401020090014000A00140FFFFFFFCF9
:10AD3000FFFF0200FEFF0100253038580D0A000019
:10AD400081B0F0B5C4B00E4607464993812000019A
:10AD50002F49085C002845D002920120050204A872
:10AD60002946F5F720FAFCB20021C8430C2C3AD84A
:10AD7000721E032A37D82748005DB042084632D3F6
:10AD8000F80535D50021B8050DD404A80190401868
:10AD9000691AA20022A39B582E4AFCF7C3FD019812
:10ADA000FEF77AFE014678050ED404AF7818691ACA
:10ADB000B20029A3D218121F1368264AFCF7B2FD6D
:10ADC0003846FEF769FE0146029A04AE70180C463A
:10ADD000691A49AB0393FFF72BFC01193046FFF7C3
:10ADE0003BFE00E0002044B0F0BC02BC01B00847CC
:10ADF000FEF7E6FE034604A8019007A22946FCF7E9
:10AE000091FD0198FEF748FE0146B805BDD5CAE799
:10AE1000C8B401025DDB000025313075207C2000C4
:10AE2000CECC000024CD00001ECD0000FDCC0000E3
:10AE3000C8CC0000E9CC000017CD000010CD000008
:10AE40000BCD0000C1CC0000D4CC0000E4CC00004D
:10AE5000B9CC000045CD000003CD0000EFCC0000D0
:10AE6000F6CC0000DACC000000000000F0B581B0A4
:10AE70000B460120EFF31084044002D1EFF3108160
:10AE800072B6990F07D0022001212DA2FFF758FFBB
:10AE9000002C3DD141E02249224D00276F54224A27
:10AEA000AB5A224AAE5AF3189EB2F60A01D0204E8F
:10AEB0009B19AB52EFF31086064002D1EFF31083DB
:10AEC00072B6AA5A1C4BEB5A934202D116482F5223
:10AED0001AE06854934201D8164B5B1C9B1A99B236
:10AEE000890A00D0830210482B52286801280BD809
:10AEF000411E8841A918091D9AB2104B00F06CFC44
:10AF0000002801D006482F54002E03D0002C04D076
:10AF100001B0F0BD62B6002CFAD162B601B0F0BD4E
:10AF20000F080000C8B401020C0800000A08000065
:10AF300000F8FFFFFF070000080800006DAE0000EA
:10AF400055415254204572726F722025780D0A00C7
:10AF500010B50446FEF7E0F8A08A002800D010BD26
:10AF60000A4CA06D401CA065FDF72CFE6062606D70
:10AF7000002805D0FDF726FE60660020606510BD44
:10AF8000A06920660120606510BDC046A096010240
:10AF900070B5012801D9012070BD48224243734B8E
:10AFA0009C58A5691F218D43A5610625A5600F2525
:10AFB00025629C18A27C002A05D1627C002A02D15D
:10AFC000227C002A14D06368002B11D4251D0B406D
:10AFD000012216469E400C4B1E60BFF34F8FBFF3FD
:10AFE0006F8F2B68002B03D40B409A4007490A60EF
:10AFF000002803D0012804D1092000E00820F9F737
:10B0000007FB0020A06170BD80E100E080E200E06D
:10B01000F0B585B00D460278E348C368934219D075
:10B02000446D944216D08368934203D0016D9142DF
:10B0300000D07FE09B1A591E8B410493482159434D
:10B04000032D46D14418E16900294ED01C3400205C
:10B0500020606DE09B1A5A1E93410493032D1AD170
:10B06000039548225A438418A26B0121EFF31085FF
:10B070000D4002D1EFF3108772B6A7691026B743CF
:10B08000A761A669002E01D118342160002D00D1DE
:10B0900062B6039D0CE04821594342189169183269
:10B0A000302902D0116810294CD180211160002272
:10B0B0004821594340180021816301628162243094
:10B0C00000210160002A33D004A82946904705B02A
:10B0D000F0BD421891691832302902D01168202938
:10B0E00039D180211160002216E00395E26B012620
:10B0F000EFF31085354002D1EFF3108172B6A169EC
:10B100002027B943A161A169002901D11834266023
:10B11000002D00D162B6039D4821594340180021FB
:10B12000C163C1624163303000210160002ACBD18C
:10B1300005B0F0BD00920E4A2E329C480D490E4BD0
:10B14000FEF7A0FD10680093019098480949084A4D
:10B150000A4BFEF797FD106800930190044A2432D1
:10B1600092480449054BFEF78DFDC04660940102EC
:10B17000B1020000A9CD00007ECD000062CD00002C
:10B18000F0B585B0049048210A464243864B9C584E
:10B19000E6690F2535409A18167C002E31D04F20D5
:10B1A00040026169014200D185E0A0690421884321
:10B1B000A06102202062012081076918D161D36B50
:10B1C000EFF31084044002D1EFF3108572B6956955
:10B1D0002026B54395619569002D00D173E0104696
:10B1E0003C30002C00D162B600240460D462546369
:10B1F000303200201060002B63D004A8984705B0BF
:10B20000F0BD0C2D5DD8C0467D442D796D00AF4456
:10B2100067586B580658A1635858585806009569E6
:10B22000202D04D0154618352D68302D49D1156BC9
:10B23000566B3432AE4217D26669360714D564684D
:10B2400015686E1C166048431818C06A4455049867
:10B250000C4644431A19156B566B3432AE4203D276
:10B260001C5966693607EAD41268AA4229D14143BB
:10B27000585882690524A24382615A18D36B012170
:10B28000EFF31080084002D1EFF3108472B6946996
:10B290002025AC4394619469002C02D114461834E3
:10B2A000216014463C34002800D162B600212160A0
:10B2B000D16251639CE70C2D00D176E7012D00D1BE
:10B2C00073E705B0F0BD15461835286010463C30D0
:10B2D000002C00D187E787E70420206205B0F0BD8D
:10B2E0000120206205B0F0BD0825256216461836FB
:10B2F0009569102D02D03568302D4BD10396566AD2
:10B3000015462835976AB74228D1A069022188439B
:10B31000A061936B0121EFF31080084002D1EFF39D
:10B32000108472B6039E34681027BC4334603468BE
:10B33000002C00D1316014463834002800D162B6A8
:10B340000021216029601162243200201060002B4E
:10B35000B7D052E70220206205B0F0BD2A68B242A1
:10B36000AFD262699207ACD52A68561C2E6048435A
:10B370001818006A805C206004980A4642439D18B1
:10B38000AC6A6E6AB4429CD228359C5862699207B6
:10B39000EAD496E7316800900191044804A1094A73
:10B3A00009A3FEF76FFCC0466094010248CD00007F
:10B3B000756172745F6972715F68616E646C6572E9
:10B3C000000000003D0300005561727420256420D8
:10B3D000737461746520676F65732077726F6E6731
:10B3E00020256400F0B585B00E460546022804D33A
:10B3F000002E02D1012005B0F0BD002D03D0012D9B
:10B4000008D1092400E008242046F9F709F920466C
:10B41000FEF700F948216943E74A505883691F2421
:10B420000294A3438361062383600F230193036285
:10B4300057180023BB62BB63FB633B627B62FB620A
:10B440003B63317F3974727F7A74B27FBA7404932C
:10B450007B637368B268F468920022435B1E032B1F
:10B460000ED8C0467B441B795B009F44010503074F
:10B47000082304E0282302E0182300E038231A43BD
:10B48000C260C907090F72699201D2B28918B26904
:10B490009207920E8918491C8160796131690129EE
:10B4A00001D122210161012D5CD831680E2959D2C8
:10B4B0003846123003900324002D01D0204600E0CE
:10B4C00004204C432D490E19B178F9F739F9396840
:10B4D000CA68802510462843C8602848005D7378F4
:10B4E0001B021818C862AA43CA60F9F771F90398D9
:10B4F0000078002809D1384611300078002804D19E
:10B50000384610300078002827D07868002815D4F5
:10B51000032102468A431B4953588407E40EFF2641
:10B52000A640B343A5401D43555002990140012058
:10B530008840A2490860144908600EE08107C90EDE
:10B54000FF228A40019C0440083C032084430C48AD
:10B55000235893438D401D4325500120B861049822
:10B5600005B0F0BD02480349DA22034BFEF78AFB1F
:10B5700048CD0000BBCD000098CD0000CCC000003D
:10B580001CED00E000E400E000E100E0F0B58FB069
:10B590000E900125002900D14BE003930491059200
:10B5A000002A00D145E00121EFF3108201910A4009
:10B5B00002D1EFF3108172B64827029747437E49C4
:10B5C000CE19B5690023302D23D831461831C04635
:10B5D0007D442D796D00AF4420242626262626267C
:10B5E00026262626262626265E26262626262626C3
:10B5F00026262626262626261826262626262626F9
:10B60000262626262626262618000223002A0CD0C7
:10B610000CE0402D01D0802D05D10123002A04D05B
:10B6200004E020240C60002A00D162B61D46002BE5
:10B6300002D028460FB0F0BD002575630399F16371
:10B640000499F162059931635B4CE35959691322FE
:10B65000D202114205D0062199600F211962716949
:10B660009960317C00290CD0F56109950895079502
:10B6700006950D950B9502210A91012810D01720EF
:10B680000FE0717C9A6900292CD0952002439A61C1
:10B6900028460FB0F0BD30240C60002AC5D0C5E7A5
:10B6A0001920049F0C907068002805D41F210840C1
:10B6B000019981404148016014209861B06806A951
:10B6C000F9F7F6F80E9802994143601880686158BE
:10B6D000F34A0092091D3A46059BF9F759F92846A5
:10B6E0000FB0F0BD3436110602D580218A439A612D
:10B6F00031680025059A91422DD205955D694F214B
:10B700004A0215421BD1E90502D4029CEC4F0AE023
:10B71000596833685C1C3460029C6043E84F3818F9
:10B72000C06AC1540E98214641437E18736B346B36
:10B73000A34238D234367B585D691542E3D00221EA
:10B740001962019EB10729433546DD4CEFF31082A3
:10B75000324006D008E02946019EEFF310823240C5
:10B7600002D1EFF3108372B6029B4343E018836962
:10B770002024A34383618369002B05D0002A08D0CD
:10B78000C26B002A0AD154E7034618331E60002A10
:10B79000F6D162B6C26B002A00D14AE70EA89047E4
:10B7A00028460FB0F0BD2946059D019E3C46EFF3AB
:10B7B00010823240D5D0D7E76094010280E200E0E9
:10B7C00080B5012002496422024BFFF7DFFE80BDF5
:10B7D000D4950102C1B70000F0B591B010900126D8
:10B7E000002900D19BE003930591002A00D196E047
:10B7F00007900121EFF310800291084002D1EFF38E
:10B80000108172B604924823069307994B43AC49C2
:10B81000C9188D690026302D6ED80C461834AD003D
:10B82000374602A675593E46AF46C04601B90000EC
:10B8300009B900000DB900000DB900000DB90000F4
:10B840000DB900000DB900000DB900000DB90000E0
:10B850000DB900000DB900000DB900000DB90000D0
:10B860000DB900000DB900000DB90000F1B80000DD
:10B870000DB900000DB900000DB900000DB90000B0
:10B880000DB900000DB900000DB900000DB90000A0
:10B890000DB900000DB900000DB900000DB9000090
:10B8A0000DB900000DB900000DB900009FB90000EE
:10B8B0000DB900000DB900000DB900000DB9000070
:10B8C0000DB900000DB900000DB900000DB9000060
:10B8D0000DB900000DB900000DB900000DB9000050
:10B8E0000DB900000DB900000DB90000F1B800005D
:10B8F000022600280CD00CE0402D01D0802D05D16F
:10B900000126002804D004E010252560002800D17D
:10B9100062B6002E069D6A4F049C079802D03046FE
:10B9200011B0F0BD00268E62039A8A63059A0A62FE
:10B930004C620A7C002A0BD00C960B960A9609964C
:10B9400008960E9602220D9201282DD018202CE088
:10B950008A7C2831002A3BD00A68A24216D22B46A4
:10B960004343FA585469A40710D50868441C0C6076
:10B97000F918096A085C10601098294641437A1842
:10B9800011462831936A526A9342E8D34543785965
:10B99000816982220A438261304611B0F0BD3025B0
:10B9A00025600028B4D0B4E71A200F90C86808A911
:10B9B000F8F77EFF109845437A597819C0683849DE
:10B9C000009105992346F8F7E3FF304611B0F0BD2A
:10B9D000FB589A69140602D58024A2439A610A682A
:10B9E0000026049882422ED25D694F2252021542EF
:10B9F00007980AD002211962029EB10729431FE06D
:10BA000028315D6915423E46F4D137465C69A4078A
:10BA100002D406992A4E0AE00C68661C0E6006994C
:10BA20004843274E3018006A005D18601098414363
:10BA3000735871188C6A4E6AB442E1D329463E4667
:10BA4000069D1F4F01E0314607985A6A002AFCD133
:10BA5000EFF31082029B1A4002D1EFF3108372B60B
:10BA60004543781983691024A34383618369002BBC
:10BA700005D0002A09D0826B002A0BD14FE703467C
:10BA80001833029C1C60002AF5D162B6826B002A32
:10BA900000D144E710A89047304611B0F0BDC04631
:10BAA00011B0000048214143054842189269D2066E
:10BAB00001D4002070474058416901200840704778
:10BAC0006094010205480068202803D00548064913
:10BAD0000860704702480449086070470C00004045
:10BAE00024D6010330CF010300900102F0B587B0E6
:10BAF00001460127022505283A4600D02A460020A3
:10BB00000929014600D01146C900374A54180E21B0
:10BB10000591615EFDF78AFB1026A15F3846FDF7AF
:10BB200085FB1227E15F2846FDF780FB069514256B
:10BB3000615F03200490FDF779FB0598235EA05F09
:10BB4000E15F625F00AD07C528A2069F3846049DED
:10BB50002946FFF7F5F82046263004263146FBF744
:10BB60004BFF2620235E2820205E2A21615E2C22A6
:10BB7000A25E00900191029224A238462946FFF766
:10BB8000DFF827463E3738463146FBF753FF3E2065
:10BB9000235E06983C5EB95F0622BA5E009401916E
:10BBA000029221A207462E462946FFF7C9F85624DD
:10BBB0000D4D285FFBF732FF2B5F2C4621A2384644
:10BBC00031463546FFF7BCF8264658363046FBF777
:10BBD00011FF5820235EF05F00901FA238462946CF
:10BBE000FFF7AEF807B0F0BD149A0102546F46207B
:10BBF000616E742064656C6179732025642025640E
:10BC00002025642025640D0A0000000050446F4187
:10BC10002064656C61797320256420256420256487
:10BC20002025640D0A00000050446F4120676169BF
:10BC30006E732025642025642025642025640D0A68
:10BC40000000000050446F4120616E7420737061E9
:10BC500063652025640D0A0050446F4120616E67C2
:10BC60006C65206F66667365747320256420256497
:10BC70000D0A0000F0B587B01546774B1A680F24FF
:10BC8000A2432F783A431A60744C23462C3B744AE3
:10BC90001A60049003462246283A12681207FAD521
:10BCA000704E092F0291039306D972493160716079
:10BCB0000C2F09D171480FE0042F07D96C4931606E
:10BCC0006C497160092F06D36D4805E06648306005
:10BCD0007060664800E068486A490860EB7AFF2BAC
:10BCE00002D10020B0620AE003210B406648C05C2C
:10BCF00040220243B2620220644AFFF721F8039F08
:10BD00000021384605952A460B46FBF7FFFE0646FE
:10BD1000022503215EA2284601913346FFF710F861
:10BD200006963046FCF7C6FB0121049800910840B6
:10BD30002CD13D4033D15C4900283AD1002D1ED092
:10BD40006048A062E062206360635F4860625F48B1
:10BD50000860152085046E1C8E608D60642420466A
:10BD60000F46F8F735FD3E603D602046F8F730FDA0
:10BD7000281D38605648032156A2FEF7E1FF0598BA
:10BD8000007BFAF7FFFF069807B0F0BD2E46054688
:10BD90000698FCF7A7FF284635463D40CBD02E46F7
:10BDA00005460698FCF7BCFB284635463E49002868
:10BDB000C4D03E4808613E4848613E48886115202D
:10BDC000C8613D48016840220A4302600721080318
:10BDD000244B5A6982430098400310185861052289
:10BDE000029842432748036898182F4E766B47788D
:10BDF0000F40995C0907490EC919CA032F4B3340FC
:10BE00009A18C90151182E4A8918274A51632649A0
:10BE1000896B3822914382785207920E8918042246
:10BE20000A4321498A630F4E31690279019B1A4006
:10BE3000C0784007C00E80181F2291430818306157
:10BE400055204003411C216020606420F8F7C0FCAD
:10BE50001549002D93D073E7040400402C60004086
:10BE600000040080000600400F040F044DC70000CE
:10BE700003040304000400047EC800001CC6000084
:10BE8000AFC90000CC930102E0CA0000C9CD000098
:10BE900050485920706172616D732073657473200E
:10BEA000253038780D0A00009060004012A83E004E
:10BEB0009DD79B5AD579BD49340200403F0080FF91
:10BEC000404000002008820002D50F000202550009
:10BED000020800007577625F72785F696E69740DA1
:10BEE0000A000000B0B51820FDF794FB1920FDF7FB
:10BEF00091FB002420462146F8F796F8204621467B
:10BF0000FAF7C4FE012503217F2328460A46FAF7E3
:10BF1000CFFF2846FBF7A4F90220FBF7D7FD284600
:10BF20002946FCF753FE2046B0BDF0B581B0164659
:10BF300000910446002001273946FDF71BF9EFF375
:10BF400010853D4002D1EFF3108072B627204001EA
:10BF500070430A21F4F7BEF80246002C02D00020FC
:10BF6000009901E002200021FBF780F90446FBF76D
:10BF700045FA002D00D162B6204601B0F0BDF0B503
:10BF800081B01D460E460446022A09D101273846D3
:10BF90003946FDF7EFF800960022384629460FE0B3
:10BFA000174601200021FDF7E5F8012F04D1009686
:10BFB00000202946024603E00096022000210A469E
:10BFC0002346FBF733FA0446FBF718FA204601B084
:10BFD000F0BD000070B5002801D0012070BD032520
:10BFE000A9020F4802680F4B5350002494600122AD
:10BFF00053030D4E3360BFF34F8FBFF36F8F0B4E64
:10C00000336003685A50847204811020F8F700FBF3
:10C01000022007A22946FEF793FE204670BDC046C7
:10C02000F094010251E5CC1A80E100E080E200E0EA
:10C0300057445420636C6F73650D0A002021020C75
:10C0400001D010211046020A01D010460839020919
:10C0500001D01046091F820801D01046891E4208EF
:10C0600001D0881E7047081A704702E008C8121FE6
:10C0700008C1002AFAD170477047002001E001C1D1
:10C08000121F002AFBD17047000084C1000008C1C4
:10C090000000C03F000038410000AC410000D44126
:10C0A00028000400000008400800000810080408E8
:10C0B000102000000000000000000000010000004F
:10C0C000FFFFFFFF000000000000000059062014E1
:10C0D000032145012882003241003219004113003A
:10C0E000390300B506002D03002D020022010022B5
:10C0F00001003E01002000008009EE4D5048504FE5
:10C1000080096E4F58E5854F80096E4FB867C14F63
:10C110005048D04FB867C14FE828DF4F8009EE4F35
:10C1200018EAFC4F8009EE4F58E50550A4550D5014
:10C13000F0C51450A4550D5000002110422063306A
:10C140008440A550C660E770088129914AA16BB16F
:10C150008CC1ADD1CEE1EFF1311210027332522217
:10C16000B5529442F772D662399318837BB35AA3BF
:10C17000BDD39CC3FFF3DEE36224433420040114E7
:10C18000E664C774A44485546AA54BB5288509950F
:10C19000EEE5CFF5ACC58DD55336722611163006B7
:10C1A000D776F6669556B4465BB77AA7199738875F
:10C1B000DFF7FEE79DD7BCC7C448E5588668A77877
:10C1C0004008611802282338CCC9EDD98EE9AFF9AF
:10C1D000488969990AA92BB9F55AD44AB77A966A57
:10C1E000711A500A333A122AFDDBDCCBBFFB9EEBFF
:10C1F000799B588B3BBB1AABA66C877CE44CC55C27
:10C20000222C033C600C411CAEED8FFDECCDCDDD4E
:10C210002AAD0BBD688D499D977EB66ED55EF44EF6
:10C22000133E322E511E700E9FFFBEEFDDDFFCCF9E
:10C230001BBF3AAF599F788F8891A981CAB1EBA1F2
:10C240000CD12DC14EF16FE18010A100C230E3206E
:10C250000450254046706760B9839893FBA3DAB316
:10C260003DC31CD37FE35EF3B1029012F322D232BE
:10C270003542145277625672EAB5CBA5A8958985E6
:10C280006EF54FE52CD50DC5E234C324A01481040E
:10C290006674476424540544DBA7FAB79987B897B6
:10C2A0005FE77EF71DC73CD7D326F2369106B0165E
:10C2B00057667676154634564CD96DC90EF92FE976
:10C2C000C899E9898AB9ABA94458654806782768AE
:10C2D000C018E1088238A3287DCB5CDB3FEB1EFB56
:10C2E000F98BD89BBBAB9ABB754A545A376A167AFE
:10C2F000F10AD01AB32A923A2EFD0FED6CDD4DCD26
:10C30000AABD8BADE89DC98D267C076C645C454C4D
:10C31000A23C832CE01CC10C1FEF3EFF5DCF7CDFF5
:10C320009BAFBABFD98FF89F176E367E554E745E9D
:10C33000932EB23ED10EF01E3031323334353637C3
:10C340003839414243444546100040008000000116
:10C350000002000400080010100018002000300047
:10C360004000600080000001FFFFFFFF01FF01FFB0
:10C37000FF0101FFFF0100000000000000000000BD
:10C3800000000000000000000000000002000000AB
:10C390000000000014000000020000000700000080
:10C3A0000200000002000000000000000200000087
:10C3B0000000000014000000020000000100000066
:10C3C0000200000002000000020000000000000067
:10C3D0001400000000000000FFFFFFFFFFFFFF014F
:10C3E000FFFF01FFFF01FF01FF01FFFFFF0101FF51
:10C3F000FFFF01FF0101FFFF000100FF010000FF3F
:10C40000000064009E00C800E800020119012C0130
:10C410003D014C015A01660172017D0187019001C5
:10C420009901A101A901B001B701BE01C401CA016E
:10C43000D001D601DB01E101E601EB01EF01F401DE
:10C44000F801FD010102050209020D0211021402A8
:10C4500018021B021F022202250228022B022E02B2
:10C460003102340237023A023D023F0242024502E3
:10C4700047024A024C024F0251025302560258022E
:10C480005A025C025F02610263026502670269028E
:10C490006B026D026F0271027302750276027802FE
:10C4A0007A027C027E027F0281028302840286027B
:10C4B000880289028B028C028E028F029102920204
:10C4C00094029502970298029A029B029D029E0294
:10C4D0009F02A102A202A302A502A602A702A9022C
:10C4E000AA02AB02AD02AE02AF02B002B102B302C9
:10C4F000B402B502B602B702B902BA02BB02BC026C
:10C500000000000000000000020000000400000025
:10C51000001003EB0000000001000000010000001B
:10C5200004000000000100320000000000000000D4
:10C5300000000000010000000100000500000000F4
:10C5400000000000000000000100000001000035B4
:10C5500000000000010000000000000004000000D6
:10C5600000000020000000000100000000000000AA
:10C5700004000000000000D80000000001000000DE
:10C5800000000000010000000000000600000000A4
:10C590000100000000000000010000000200000196
:10C5A000000000000000000000000000010000008A
:10C5B0000300009F000000000100000000000000D8
:10C5C00001000000000000B90000000001000000B0
:10C5D0000000000001000000000000AB000100FFAF
:10C5E000010000FF000100FF010000FFFF0000014B
:10C5F00000FF00010001000000FF00FF00FF00003D
:10C600000100FFFF00FF010000000001010000FF2A
:10C61000FFFF01FF01010000000001010003020112
:10C6200000000502010000010301000003030100F6
:10C6300001000301000102030100020003010002E6
:10C6400002030100030203010003040301000402CA
:10C6500003010000000302000003030200000603C0
:10C6600002000100030200010303020001060302AD
:10C670000002010302000204030200020703020099
:10C680000303030200000107030000060703000183
:10C690000004030001000703000104070300010771
:10C6A0000703000200070300020407030002070754
:10C6B0000300030207030003060703000402070345
:10C6C0000004060703000501040300050207030038
:10C6D000050607030006000703000604070300061B
:10C6E0000707030007030703000707070300080203
:10C6F00007030008060703000902070300090607ED
:10C7000003000A020703000A070703000B050703DB
:10C71000000C030703000C070703000D07070300C5
:10C720000E070703000E060704000E070704030E9A
:10C73000070704030E070704030E070704030E0789
:10C740000704030E070704030E070704030007008E
:10C7500002020100000202000401020200070102BD
:10C7600002020200020201010102020106010202AC
:10C770000305000202040200020202060102020393
:10C780000001020203050102020503000202040582
:10C790000102020204020202020702020205030170
:10C7A000020205060102020600010202060301025E
:10C7B000020205030202020603020201060402024B
:10C7C0000106070202020304020202030702020238
:10C7D000060702020302070202030507020203071B
:10C7E0000702020407040202050104020205010710
:10C7F00002020503070202050607020206020702FB
:10C8000002060507020207010702020704070202E7
:10C8100008010402020802070202080507020209D1
:10C820000304020209040702020A000702020A02C4
:10C830000702020A050702020A070702020B0307A2
:10C8400002020B060702020C010702020C04070297
:10C85000020D010702020E000702020E0407020287
:10C860000F010702020F050702020E040703030F60
:10C87000030703030F070703030F07070303000062
:10C88000000202000000020200000002020000009C
:10C890000202000000020200000002020001000289
:10C8A000020004000202000700020201010002026D
:10C8B0000104000202010700020202030002020159
:10C8C0000401020201060102020305000202020441
:10C8D0000102020301010202030301020204010139
:10C8E0000202040401020202060202020302020220
:10C8F000020106030202020203020201020702020F
:10C9000001040702020303030202020404020202FA
:10C9100005070202030107020203050402020401E3
:10C9200007020204030702020506030202050007CC
:10C9300002020502070202050407020206000702BE
:10C9400002060207020206050702020607070202A4
:10C95000070407020207070402020802070202088E
:10C9600005070202090107020209040702020A0080
:10C970000702020A030702020A060702020B020765
:10C9800002020B050702020C010702020C05070256
:10C99000020D020702020C010703030C0607030342
:10C9A0000D020703030E020703030E07070303002C
:10C9B000000002020000000202000000020200006B
:10C9C0000002020003000202010000020201020054
:10C9D000020200050102020202000202030100023B
:10C9E0000202010102020204010202010202020229
:10C9F0000104020202030401020202020202020214
:10CA000005020202000207020200040702020006F9
:10CA100007020201020702020104070202010607DF
:10CA200002020203070202020507020203020702D2
:10CA300002030407020204020702020404070202BE
:10CA400004060702020501070202050307020205A8
:10CA50000507020206020702020604070202060692
:10CA60000702020704070202080107020209000781
:10CA70000202090107020209030702020A00070273
:10CA8000020A020702020B000702020B020702025F
:10CA90000C000702020B060702020C040702020C3C
:10CAA000060702020D030702030C000703030C0232
:10CAB0000703030C050703030C070703030D050712
:10CAC00003030D070703030D070703030D07070300
:10CAD000030D070703030D070703030D07070303F0
:10CAE0000E0D0B07696E636C7564652F6472697651
:10CAF0006572732F6D6B5F6164632E6300696E6393
:10CB00006C7564652F647269766572732F6D6B5FE7
:10CB10006165732E630033324B206C6F6164206358
:10CB200061702076616C2025640D0A005854414CD8
:10CB3000206C6F6164206361702076616C202564D5
:10CB40000D0A00556E657870656374656420646DC8
:10CB500061206368616E6E656C0D0A00696E636CBE
:10CB60007564652F647269766572732F6D6B5F668D
:10CB70006C6173682E630052656C6F61642076612E
:10CB80006C756520696D706F737369626C650D0AF1
:10CB900000696E636C7564652F6472697665727383
:10CBA0002F6D6B5F6D6973632E63007379735F74B0
:10CBB00069636B5F7374617274005265736574208E
:10CBC000627920756E6B6E6F776E20736F7572630E
:10CBD000650D0A0025313064207C200D0A00437267
:10CBE00061736865642121210D0A002D2D2D2D2DE5
:10CBF0002D2D2D2D2D2D2D2D2D2D2D2D2D2D2D2D65
:10CC00002D2D2D2D2D2D2D2D2D2D2D2D2D2D2D2D54
:10CC10002D2D2D0D0A00253038583A202530385852
:10CC20002025303858202530385820253038580DE8
:10CC30000A005052494D41534B3D253038580D0A9A
:10CC400000434F4E54524F4C3D253038580D0A008A
:10CC50004D53503D253038580D0A005053503D2556
:10CC60003038580D0A0041495243523D253038585A
:10CC70000D0A004C523D253038580D0A00495053DA
:10CC8000523D253038580D0A00785053523D25301A
:10CC900038580D0A004E3D25642C205A3D25642C41
:10CCA00020433D25642C20563D25640D0A0046494D
:10CCB0004C45202020203A20005B53435030335D08
:10CCC000005B464952415D005B5557425D005B4D3C
:10CCD00041435D005B4343435D005B564552424F19
:10CCE00053455D005B53455D005B5543495D005B0B
:10CCF0005741524E5D005B494E464F5D005B4150CF
:10CD0000505D005B4552524F525D005B4F535D00DA
:10CD10005B424F4F545D005B544553545D005B4490
:10CD200052565D005B5048595D00696E636C7564D6
:10CD3000652F647269766572732F6D6B5F747261B3
:10CD400063652E6300257300696E636C7564652FDF
:10CD5000647269766572732F6D6B5F756172742E84
:10CD60006300556E657870656374656420756172E3
:10CD70007420256420737461746520256400556EE9
:10CD8000657870656374656420646D6120636861B3
:10CD90006E6E656C20256400506172616D74657201
:10CDA00020696E76616C696400756172745F646D90
:10CDB000615F63616C6C6261636B00756172745F6B
:10CDC000626175645F736574004F70656E20414EDB
:10CDD0005425640D0A00B9CCBCFEB0E6B1BE3A558C
:10CDE00057422DB1EAC7A9205625642E25642E206E
:10CDF0000D0A00C9E8B1B849443A202578202E0D23
:10CE00000A006C73705F7363616C655F6633320038
:10CE10006C73705F675F6F705F663332006C737046
:10CE20005F675F6F705F696E743136006C73705F3F
:10CE3000675F6F705F696E7438002E2E2F2E2E2F55
:10CE40002E2E2F2E2E2F2E2E2F6472697665727342
:10CE50002F6D6B5F6C73702E63004F706572616E27
:10CE6000642061646472657373202578206973207F
:10CE7000696E76616C6964004E656564206174203A
:10CE80006C65617374206F6E65206F706572616E82
:10CE900064005258204445534320696E64657820ED
:10CEA0006973206F7665722072616E67650D0A0086
:10CEB000455420696E646578206973206F766572C9
:10CEC0002072616E67650D0A002E2E2F2E2E2F2EDA
:10CED0002E2F2E2E2F2E2E2F647269766572732FB1
:10CEE0006D6B5F6D61632E63006D61635F72785F70
:10CEF000646573635F636F6E737472756374006DE2
:10CF000061635F65745F636F6E73747275637400E1
:10CF1000556E646566696E6564206269742072612D
:10CF2000746520256420666F72206D65616E2050E7
:10CF30005246206F662025640D0A004D45414E2063
:10CF400050524620706172616D6574657220657221
:10CF5000726F720D0A00436F646520696478202542
:10CF60006420616E64206D65616E205052462025FC
:10CF70006420636F6E666C6963740D0A002E2E2F39
:10CF80002E2E2F2E2E2F2E2E2F2E2E2F64726976C0
:10CF90006572732F6D6B5F7068792E6300010000FE
:10CFA00001000000FF00FFFF0000FFFF0100010083
:10CFB000010000FF01FF010100010000000001016C
:10CFC000FF000000010000FF0000FFFF00FF010064
:10CFD0000100FFFF00FF010101000101000000014D
:10CFE000FF00010000FF000101FF0001010100003E
:10CFF000FF01000001000100FF000101FF01FFFF30
:10D0000001000000000000010000000000FF01001E
:10D01000000000FF00FF000000FFFF010101000011
:10D020000100FF01000001000001000000000000FD
:10D03000FF000000FF0000FFFF000000FF0001FFF5
:10D040000100FF0001FF00FF01000000000001FFE0
:10D050000000010100FF00010000FFFF01000001CE
:10D0600001FF010001FF000100000000FF00FF00C0
:10D07000FF00FF0101FF01000100000100010000AD
:10D0800000FF0100010101000000FFFFFFFF01019F
:10D09000010000000001010100FFFFFF01FF00008F
:10D0A0000000010000FFFF0000000000FF00010081
:10D0B000010001FF000100000100000100FF00006D
:10D0C000FF010101000001000000FF01000100FF5D
:10D0D000000000000101010101FF010001FFFF004C
:10D0E00001FF000101FFFF00FF0000000100FF0140
:10D0F0000000010001FFFFFFFF000000FF00000033
:10D10000000000FF01000001FF000101000000011C
:10D1100001FF00000101FF00FF00FF01000101000D
:10D120000000000000FF000100FF0100FFFFFF0101
:10D13000FF01010000FF01000101000100010001E9
:10D14000000000FF0000FF0000FF01000001FF01E0
:10D1500001000000FF01FF00FF010100FF000101CD
:10D16000010100FF0000FF000101000001000100BB
:10D17000000101FF00000100000001FF000000FFAE
:10D1800000FFFF0100000000FF00000000FFFF00A3
:10D1900001000000000001FFFF01000000FFFF0090
:10D1A000000000FFFF010100FF0101010100FF007D
:10D1B0000101000100FF0000FF010001010000016A
:10D1C00001FF0001010001FF0100FF00000100005C
:10D1D000FF00FFFF000000FF01FF00000100000052
:10D1E00000FF000101FF000000000001FF00FF0040
:10D1F0000000000000FF0000FF01FF0101FF01002F
:10D200000000FF0001000100010101FF0000FFFF1D
:10D21000000001000100000001000000010100FF0A
:10D22000000100FF000001FF00FF0100FF000001FE
:10D23000000100000000010001FF000000000101EA
:10D24000000001000101010101FF0100FF0001FFD9
:10D2500000FFFF01000101FFFF000000FFFFFF00D2
:10D260000100000001000100FF01FF0000000000BC
:10D270000001FF01FF00FFFF00000101000000FFAF
:10D2800000000100000101FF0000FFFF0101FF009D
:10D2900000FF00000000000001FF00000100FF008F
:10D2A0000000FF010100000000FFFFFF010100007E
:10D2B00000010001FF00FF010000FF01000000FF6E
:10D2C000FF00FF0000FFFF00FFFF010101FF010061
:10D2D000FF0101000001FF0101000100000000004A
:10D2E0000100FF00010101FF00000100000100003A
:10D2F00000FF00000000010000FFFF01000101002D
:10D3000001000100FF0000FF00FF01FF000100011C
:10D310000100000000000101000000000100000009
:10D3200001000001FFFF0001FF010100FF000000FC
:10D33000FFFF000001FF00010000010100000001EB
:10D340000101000001000100FF00FF01FF00FF00DC
:10D3500001000001000001000101FFFFFFFF0100CB
:10D36000000101FFFF010001FF00FFFF01000000BD
:10D37000000000FF00FF00000000FF0100FFFF00B1
:10D380000001000000000001FF0101000000FF009B
:10D39000FF0100010001FFFF000000FF00FF00008F
:10D3A000000001FF0000000000010000000000007C
:10D3B00001FFFF01FF010100FF000100010000016A
:10D3C000FF000001010100FF010100FF000001005A
:10D3D000FF01000000010100010101FF00FFFF004B
:10D3E000010001FF00FFFF0000FF0000010000003E
:10D3F000FF01010000000001000101FF01FF00002A
:10D400000100010001FFFF0000FFFF00FF0000001E
:10D4100001000001FFFF0001010100000000010107
:10D4200001FFFFFFFF0000000101010001FF0000FC
:10D43000000100010000010001FF0101FF00FF00E9
:10D44000FF00FF000000000100FF010001FF0101DB
:10D45000000001FFFF00000100FF0001010000FFCC
:10D4600001000000000001FF00FF0100FF0001FFBC
:10D470000100FF000000FFFF0000FF000000FF00B0
:10D48000000000000001000001000001FF00010099
:10D49000000101FF00FF01010000FF010100000089
:10D4A000010100FF01000001FF000000000000FF7B
:10D4B000000000FFFFFFFF010001000001FF00016D
:10D4C000000000FF00FFFF010100FF0100FFFF015E
:10D4D0000001FF010101010100000000FF00010047
:10D4E00001FF000000010000010101FF0000FF003A
:10D4F0000100000100000100FF010001000100FF28
:10D500000000000000FFFF00000100000000FF011C
:10D51000FF00FFFF0100000000000100FFFF00000E
:10D520000000FF0000000001FFFF00FF000000FFFF
:10D5300001000000010000FF0101000001000100E6
:10D5400000010100FF0000FF000101010100FF00D8
:10D550000101FF00FF01FF0000000101FF010000C9
:10D5600001FF0000FF0000FF0000000100010001BA
:10D570000001010001FF00000101FF01FFFFFF00AA
:10D5800001FF000100FF0000000000000101000198
:10D59000FF0100010000FFFF0000FF010101000189
:10D5A000000100FF00000001FF0101FF01FF00007A
:10D5B000FF000000000000FF00FF0100000000006D
:10D5C000FF010100FF00000000010000FF01FF005B
:10D5D0000000FFFF00FF0000010000FF0001FF014D
:10D5E00000010100FF0101000001010001FF000036
:10D5F000FF000100010100FF0001010101FF000126
:10D6000001FFFF00000000FFFF000000010000001C
:10D6100000FF0000FF0101FFFF0000FF010100000B
:10D62000010000FF00000001010000FFFF00FF01FA
:10D63000FF01000000000000FF01FF0001000100E9
:10D6400000000100FFFFFF000000FFFF01010001DB
:10D65000FFFF00FF0100FF0001FF010101010100C8
:10D66000010000010100000000FF010001000000B6
:10D67000000100010000FF0001FF00FF010000FFAA
:10D68000000100FF00010100000001000000000097
:10D6900000000101000100FF01FF00FF0000FF008A
:10D6A0000100010001010001FFFF00000100000076
:10D6B00000FF000000010000010000FF0101010067
:10D6C000FF0001000000000001000101FF01000057
:10D6D0000101FF0001FF010101FFFF00FFFF00004A
:10D6E000FF00FFFF00000001FF000001FF00FF013D
:10D6F00000010000000101FFFFFF00000000010128
:10D70000FF000000FF00010000FF01000000010019
:10D7100001FF00FF0000000101FF01000000000008
:10D72000010000FFFF0001FF00000000FF00FF00FC
:10D73000000000000001FFFF00FF010001FFFF01EA
:10D7400001000001FFFFFFFF0101000100000100D7
:10D75000000100FF00FF01FF00FF000100010000C9
:10D76000010101000000010100000100FF010000B3
:10D77000FFFF000000FF000101FF0100FFFF0100AB
:10D7800000010000000100000000010100FF000096
:10D7900000000100FF000101010001FF0000000185
:10D7A000FF0101010000FF0100FF00000001000176
:10D7B000FF00010001000000FF010100FF01FFFF69
:10D7C000FF00000100000101000000FF0100010155
:10D7D000000000FF01FF0101000001010001000045
:10D7E000FF00000000FF000100FF0000000001FF3B
:10D7F0000000FF0000FF010101010001FF01000026
:10D80000000100FF00010100FFFF0001FF00000117
:10D810000101FF01000000FF010001010100FF0004
:10D820000100000000FF000001010000010000FFF6
:10D83000FFFF01FF000101FF00000001000100FFE8
:10D8400001000100000000010000000001FF0001D4
:10D85000000100000100000001000101FFFFFF00C6
:10D86000FF010000FF0100010000FF00FF000101B7
:10D8700000000000FFFF010000FF01000101FF01A7
:10D880000100010000FF0001010101FFFF01FFFF96
:10D8900001FF01010101FF01FFFFFF0101FFFF0186
:10D8A0000101010101FF0101FF01000001FFFF0172
:10D8B00000FFFF01000101010101FFFF010101FF64
:10D8C000FF00FFFF0001FF01FFFFFFFF00FF01FF5F
:10D8D00001FF010001FFFF0101FF01FF0101010044
:10D8E00001010001FF01FFFFFF0101010101FF0133
:10D8F000FF0101FFFF01FFFF0101FFFFFF01FF002B
:10D9000001010100FF01010101FF01000100FFFF12
:10D910000001FF0101FF010101010101FFFF01FF02
:10D9200001010000010101FFFF0001FFFFFFFFFFF8
:10D9300001FF0001FF01FF01FFFFFF010101FFFFE8
:10D94000010101FFFFFF01FF01FF00FF01FFFF00D9
:10D950000101FF01FF0100FF0101010101010101BE
:10D960000101FFFF01FFFF0101FF0101000101FFB4
:10D9700001FF01FFFF01FFFF010101FFFFFF00FFAA
:10D98000010101FF00010000FFFFFF0101FF01FF96
:10D99000FF00FF0101000101010101FFFF01010181
:10D9A000FF0101FFFFFF01FF01FFFF000101FFFF7A
:10D9B000FF01FF010001FFFFFFFFFF010001010167
:10D9C000FFFF01FF01FFFF01FF0101FF0101010155
:10D9D00000FF00FF0101000001FF010101FF010143
:10D9E000FF0100FF0100FFFF01FFFFFF0101010038
:10D9F0000101FF00FFFF01FF0101FFFF0001010026
:10DA0000000101FF0101FFFFFFFFFF010101010113
:10DA100001FF0001FFFF01FF0101FFFF01FF010105
:10DA200001FFFF01010101010101FF0101010001ED
:10DA3000FF01FF00FF00FF0101FFFFFF0100FFFFEB
:10DA4000FF010100FF01FF01FF0101FFFF010100D4
:10DA5000FFFF000101FF0000FFFF0101FF0101FFC7
:10DA600001FFFF0101010101FFFFFF010101FF01B2
:10DA7000FF0001FF01FF01000101010101FF0101A0
:10DA800001FF010101FF0100FFFFFFFFFFFF010197
:10DA9000FF0101FF0100FFFFFFFF01FF01FF000188
:10DAA0000001FF010101FFFF01FF01010001010170
:10DAB000FFFF0101FF0001010000FFFF0101FFFF67
:10DAC000010101FF01FFFFFFFFFFFF00010101FF57
:10DAD0000101010101FFFF01FF0101FFFFFF01FF44
:10DAE00001FFFFFF01FF0100FF01FFFF0001000137
:10DAF000FF0101FF01010001FF01FFFF0001010122
:10DB00000101FF0101010101010101010101FFFF0B
:10DB1000FF01FF0101FFFF01010000FF01FF010004
:10DB2000FF01FF00FF0101FFFF010101FF010101F2
:10DB300000FFFF000101FF01FF01FF00FFFFFF01E8
:10DB400001FF00FFFFFFFF01010101FF01FF0001D5
:10DB500000FF01FF0101FF0101FFFF01FF040000C1
:10DB600004040404040404040000000090DB00002A
:10DB700008900102F8040000800B000060DD000046
:10DB8000009501026C2900007AC00000000000002E
:10DB90005203328042014301015526B803014590EA
:10DBA0000050084202C203001515C0C1C2C3C4C55B
:10DBB000C6C7C8C9CACBCCCDCECF000101014B012D
:10DBC000800305090203020501330203650902030C
:10DBD00001420257140019412717901D070605043A
:10DBE00003020100F29798DDC89D5CB81CC0DEA757
:10DBF000DB615BCA010200035240480510040601C4
:10DC00000001522D2C280004007C007B010502033A
:10DC100008FF5B0F010065F901417B070701016007
:10DC2000002000881333E0536420ACFF501B0D0725
:10DC30000E080E080E080E080C030D050B050D0747
:10DC40000D070D070D0701012E010402004003FF1F
:10DC5000FF7F00FFFF7F0816FFFFFF00FFFFFF3A77
:10DC6000010001000A00010106401E4005120512D4
:10DC7000000515040201020301024004020103032E
:10DC8000020C0E0900087A0232413428002A82036D
:10DC900003455006C570014013E620700140144C46
:10DCA00007001000D6FF00B000500B42028203456F
:10DCB000FFFF0F20320442083201045510000134E6
:10DCC000B400030550200050079D28000400010205
:10DCD0000100FFFFFFFF3770900102AFC90051152F
:10DCE0001EC135BF80F3E2BDC0B464BF871699BDC5
:10DCF000AD178DBF941799BD33A876BFC4780DBDFD
:10DD00002BC162BA0CB0AFBEA9F6E9BAFC567BBE15
:10DD100007254CBBEC8823BE5DC0CBBB0CCE20BD21
:10DD20007BA095BCD40F3A3E2D5EACBD5913073F86
:10DD300064010042420944030006320145100140DB
:10DD40000FC20E520145900140184204023D0545A4
:10DD5000A00140194206023D07454001400D8201E5
:020000040000FA
:10E09000A5A54B4D0000001000000002AAAA5A7F5F
:10E0A00090E00000000000000200000000000000FE
:10E0B0000000000000000000000000000000000060
:10E0C0000000000000000000000000000000000050
:10E0D00028E10000000000000A56656E646F7209B6
:10E0E0003A204D4B53454D490A43686970093A201F
:10E0F0004D4B383030300A44617465093A2053651D
:10E100007020313920323032340A56657273696FAB
:10E110006E093A2056302E362E32000000000000E4
:08E120000000000000000000F7
:04000005000000C136
:00000001FF
